:020000040000FA
:040000006FD00400B9
:101000006F00D0350000000000000000902000209C
:10101000A4220020A9BDF9F55C23002000000000F7
:10102000000000005C230020902000200000000051
:101030000000000090200020000000009020002010
:101040000000000090200020902000209020002030
:101050009020002090200020CC2A00204E24002048
:10106000000000009020002090200020F4230020A9
:1010700090200020C22300209020002090200020FB
:101080009020002090200020902000209020002020
:101090009020002001A04111B7170040985F3AC688
:1010A000945F3247E39CE6FE3245410182800111A4
:1010B00013078008F337078093F787083EC20100C3
:1010C0000100B7170040930570052380B70413068D
:1010D00080FA2380C7040100010083C6B70493F699
:1010E000F60DA385D704238007049246F3A6068055
:1010F0000100010093760502D5CEF336078093F602
:10110000860836C4010001002380B7042380C70489
:1011100001000100B70614007D89558D88C70100C4
:1011200001000100010023800704A246F3A6068007
:101130000100010073370780137787083AC6010062
:1011400001002380B7042380C704010001000100CF
:1011500001003727004093061005A303D7802380A2
:101160000704B247F3A70780010001009307800836
:10117000F3B7078093F787083ECE01000100B71749
:101180000040130770052380E704130780FA2380CB
:10119000E7040100010003C7B70413670708A3852C
:1011A000E70423800704F247F3A70780010001004A
:1011B0000561828093760504BDC6F336078093F6F9
:1011C000860836C8010001002380B7042380C704C5
:1011D00001000100B7061400938606047D89558D31
:1011E00088C7010001000100010023800704C246F6
:1011F000F3A6068001000100733707801377870884
:101200003ACA010001002380B7042380C70401000B
:1012100001003727004093062005A303D7802380D1
:101220000704D24781B773370780137787083ACC12
:10123000010001002380B7042380C70401000100DE
:1012400098471367070C98C723800704E24719BF24
:101250000111814601468145114506CE2923930798
:101260008008F3B7078093F787083EC601000100A6
:10127000B7170040130770052380E704130780FAAF
:101280002380E7040100010003C767041367170008
:101290002383E70423800704B247F3A707800100F4
:1012A0000100F2400561828041118146014681457D
:1012B0001145552913078008F337078093F78708EE
:1012C0003EC401000100B7170040130670052380DB
:1012D000C704930680FA2380D70401000100FD555E
:1012E0002396B70223800704A245F3A505800100D9
:1012F000010073370780137787083AC601000100A1
:101300002380C7042380D7040100010003C76704BA
:10131000136717002383E70423800704B247F3A76A
:1013200007800100010001A0BD473305F50201005F
:101330007D1575FD8280411122C426C206C6AA848D
:10134000014463179400B2402244924441018280D8
:1013500005041305803E4204C13F4180DDB7000013
:101360009305000273A04580824573901534924026
:101370002242B2424243D2436244F2440255925561
:101380002256B2564257D2576258F25806499649E9
:10139000264AB64A464BD64B664CF64C065D965DE1
:1013A000265EB65E465FD65F09617300203041114C
:1013B000B7170040985F3AC6945F3247E39CE6FE59
:1013C000324541018280B71700401307000323888C
:1013D000E7028547171700002322F7AA7300203081
:1013E000411122C406C637040020973000E0E78090
:1013F000A0161C408297D5BF37370040834747006F
:101400009146BD8B6389D70099466394D700834783
:101410005740730020309716000083C6A6A6938716
:10142000160017160000230FF6A40347870097271E
:1014300000009387674BB6972380E700B7E7040067
:10144000BC4F09468945171500000345B59E829794
:10145000C9B7B787004003C76700098B6309071046
:1014600003C777009306000313770703630DD708BC
:1014700017180000034818A5171600001306C6A386
:101480000547B30606012380E60083C577001717DA
:1014900000001307E7A2429793F5F50F2300B7006A
:1014A00003C5870097150000938545A1C295137564
:1014B000F50F2380A5000347070089451377F7033D
:1014C000630CB70C63E7E50A6306071A8545630CEE
:1014D000B7129717000083C7F79E3307F60003473C
:1014E00007001377F70F19CB850793F7F70F0D4711
:1014F0006363F71A17170000A306F79CB78700402D
:1015000009472383E700B787004083C77700E207D6
:10151000E18763DE07049717000083C7B79A1717A0
:101520000000130767993E9785462300D7001717D9
:1015300000001307E7983E97930600032300D700A7
:1015400017170000130787973E97A14685072300CA
:10155000D70093F7F70F0D476364F71417170000D0
:10156000A302F796B787004009472383E70073007B
:101570002030930610026300D70E93062002630505
:10158000D70693060002E316D7F403C727021377A2
:10159000C70F13672700D5A803C767001377070491
:1015A00065CB03C7A702172800001308E85E1725BC
:1015B000000013056556134707082385E70203C794
:1015C000A7021377370F136787002385E702814748
:1015D00013070004B305F5008C41B306F80091072A
:1015E0008CC2E399E7FEF5B503C7A70213470704CA
:1015F0002385E70203C7A7021377C70F13672700E6
:101600002385E702F9B503C767001377070449C3C9
:1016100003C76702172800001308084C17250000AD
:1016200013058543134707082383E70203C76702AF
:101630001377370F136787002383E7028147130768
:101640000004B305F5008C41B306F80091078CC285
:10165000E399E7FEBDBD03C7670213470704238371
:10166000E70203C767021377C70F136727002383B7
:10167000E70285B503C767001377070411CB03C7DB
:1016800027021377370F136787002381E70291B58D
:10169000238006003DBD97170000A3850782B9BDD2
:1016A00097170000A380078275BD230304801547A8
:1016B0002303E48001002302A480828083076480E6
:1016C000E3CE07FE23030480828083076480E3CE99
:1016D00007FE03454480828083076480E3CE07FED3
:1016E0002302A4808280411126C44AC24EC006C68D
:1016F0001377F50BAD47AA892E8995446306F70049
:1017000019456537653F8D444E854537FD59FD14B4
:1017100063983401B240A244124982494101828057
:10172000135509011375F50F453F2209CDB7011176
:1017300026CC06CEB704080051371545BD377137A2
:1017400069372AC6A53F32459377150089EB1365A3
:1017500015001375F50FF240E24405618280FD1417
:10176000E9FC0145CDBF397126DC4ADA4ED852D6A4
:1017700056D45AD25ED006DE62CE66CCB7E700E021
:101780007D5783AA070022C603AA470023A0E718B3
:1017900023A2E718B7170040130770052380E7045A
:1017A000130780FA2380E70483C74704930B75FF70
:1017B000B684E20793FBFB0F8546AA892E8B3289FC
:1017C00037240040E187015763FA76016308D500AA
:1017D0008946130700026313D5000157D98F93F789
:1017E000F70FB71C00402382FC0411472303E48059
:1017F0001305F00F5D3D094CD135636D7C11B705C4
:101800000700DA9537870700795563F2E504B38757
:101810009500636EF702370B0800A94733EB6501AB
:101820006399F90689E48144513D26850DA0DA8546
:101830000945553D05090345F9FFFD14050B693DB3
:1018400081C49377FB0FFDF7DD3569FD7D55B71733
:101850000040130770052380E704130780FA2380F4
:10186000E70403C74704418B2382E704F250B7E73C
:1018700000E023A0571123A24711E25432445259E9
:10188000C259325AA25A125B825B724CE24C2161FD
:101890008280A5476395F90685691309F00FB306A1
:1018A0009900B3742B01B6941349F9FFB3749900EE
:1018B000856B33796901416B9387F9FFB3F7270192
:1018C00099E363FC340193D94900C147E3E637FF4C
:1018D00099BF0569C1697D19D9B71305800D638862
:1018E0006901130500026384790113051008CA8594
:1018F000DD3B353D21DD4E99B3843441D9B7DA85DE
:101900002D45D533CA94E30099F205097D3BA30F19
:10191000A9FED5BF9387F9FF93F7F70F6361FC0C1E
:1019200083C71C0413073008631FF7043707080038
:10193000636BEB04B3079B00B706100063F5D70495
:10194000334BEB0089476393F9068980D549E38CD3
:1019500004ECDA850945413B11090327C9FF91478A
:101960002320E48003076480E34E07FE23033481D1
:10197000FD17EDFBFD14110B81C49377FB0FE9FFFD
:101980007D3371F5E1B5B717004003C75704B707BA
:1019900008001377070219E3B78707007955E37842
:1019A000FBEA33079B00E3FFE7F855B58547E38281
:1019B000F9F2DA852D45053B9389F4FFE38504E6CA
:1019C000293393F7390091EB83260480032709001C
:1019D00093074900E39AE6E43E89CE84F1BFB54718
:1019E0006396F9001305900BC93135BDB147130556
:1019F000B00AE38BF9FE99476391F904B705080033
:101A0000B365BB002D45C53181448D4BA149753966
:101A100063967401832704802320F9008504E398EA
:101A200034FF8327048013172B016355070023120B
:101A3000F900D5BB2322F900FDB39D476399F90254
:101A400081451305B0044531BD44232009002322FC
:101A50000900FD599D3993F77400CA9703C7070021
:101A6000FD14398D2380A700E39634FF6DBBA14799
:101A70006392F9046D398144630D0B008D47930423
:101A8000C0036308FB009304000563048B01930407
:101A900040041375C507E30895D81945393139391C
:101AA0000545213126850D3909453D314931E31C74
:101AB00005D669BB91476399F90013056006F536B1
:101AC000F53E130590090DB7E38F09D4F154A9BB76
:101AD000197106C212C416C61AC81ECA22CC26CE56
:101AE0002AD02ED232D436D63AD83EDA42DC46DE7E
:101AF000CAC0CEC2D2C4D6C6DAC8DECAE2CCE6CEEE
:101B0000EAD0EED2F2D4F6D6FAD8FEDA9705000083
:101B1000938545368841E700050092402242B24253
:101B20004243D2436244F244025592552256B25681
:101B30004257D2576258F25806499649264AB64A41
:101B4000464BD64B664CF64C065D965D265EB65E01
:101B5000465FD65F096173002030000097210020A6
:101B60009381414A175100201301C1C917F5FFFFA6
:101B700013058549970500209385C5481716002051
:101B80001306C6FD63FAC5008322050023A0550095
:101B900011059105E3EAC5FE177500001305C58C14
:101BA00097150020938585FB171600201306062A3B
:101BB00063FAC5008322050023A055001105910595
:101BC000E3EAC5FE171500201305452897350020C8
:101BD000938545196377B500232005001105E36D52
:101BE000B5FEFD42739002BC8D4273904280B722D5
:101BF00000009382828873900230970200209382C3
:101C0000624093E232007390523097220000938238
:101C10004233739012346FC0A43E730020303D43B2
:101C20002A876373C3029377F700BDEFADE5937620
:101C300006FF3D8ABA960CC34CC30CC74CC741077C
:101C4000E36BD7FE11E28280B306C3408A06970297
:101C5000000096966780A6002307B700A306B7008A
:101C60002306B700A305B7002305B700A304B700F8
:101C70002304B700A303B7002303B700A302B700F0
:101C80002302B700A301B7002301B700A300B700E8
:101C90002300B700828093F5F50F93968500D58DCC
:101CA00093960501D58D61B79396270097020000A2
:101CB00096968682E78086FA9680C1171D8F3E969B
:101CC000E374C3F8A5B7B717004003C777051377C8
:101CD000E70FA38BE704130700F8A38DE7043D4744
:101CE000238CE70413075003A38CE70403C7A7055D
:101CF0001377D70F238DE7048280B717004003C7FF
:101D0000E7020D8941111377C70F498F93068008A9
:101D1000F3B6068093F6860836C6010001009306E6
:101D200070052380D704930680FA2380D70401002E
:101D300001002387E70223800704B247F3A7078047
:101D4000010001004101828041112A83014E930E5E
:101D5000407E130F0019930F400663E56E1293083F
:101D6000001913034006B3781503854E0D4FA14F9C
:101D7000337365020D891335150063EFBE12130826
:101D8000F6FF794672984208135808013307C702D4
:101D900013D61700BE0732976146B3F6C602130684
:101DA0008070B386C6023697A166F58F42075D8FB5
:101DB000B716004083C7F60293F70708A303F100A4
:101DC0000346710083C7F60293F70708E394C7FE42
:101DD00083477100B716004093F7F70F6388071227
:101DE00093078008F3B7078093F787083EC4010084
:101DF0000100B7170040930670052380D7049306AF
:101E000080FA2380D7040100010023AA070383C6B8
:101E1000170393E60608A388D70223800704A24786
:101E2000F3A70780010001001166B71700407D1677
:101E3000D45BC85F93854703A98EF18EF5FA9306AC
:101E40008008F3B6068093F6860836C601000100C6
:101E5000930670052380D704930680FA2380D70465
:101E60000100010098C103C7170313670704A38883
:101E7000E70223800704B247F3A7078001000100AF
:101E8000410182807D133368E3039308E016630EFB
:101E900008003368F3039308D016630808009378AA
:101EA000330093B818009388D81633081E01131E08
:101EB0000801135E0E0155B56393E503054863867B
:101EC00008000148630303002A8871087298FD1511
:101ED000131E0801C205135E0E01C18179BD13F8FE
:101EE000150063F4BF007908D5B713381800E5BFB3
:101EF00083C7F60293F70708A303F10003467100B6
:101F000083C7F60293F70708E394C7FE834771007F
:101F100093F7F70FF1DFE9B531714AD966CB06DFE8
:101F200022DD26DB4ED752D556D35AD15ECF62CDB5
:101F30006AC96EC7AA8C02D8EF00901C2A89930741
:101F40008008F3B7078093F787083EDA01000100A5
:101F5000B7170040130770052380E704130780FAC2
:101F60002380E7040100010003C7F7021377770F0E
:101F7000A387E70203C7F70213678700A387E70277
:101F800023800704D257F3A707800100010005450D
:101F9000AD33130780C13347E902116A93070AE89A
:101FA00093065002BD69930BA004814A014B1304B0
:101FB0008008930470057D1AB347F9023307D702EE
:101FC0003EC0FD873ECC938709A69309803E3347E8
:101FD000F7023AC27D873AC4334739038549B3993A
:101FE000990193D93940B306D702B30B7703B3C62F
:101FF000F602B3CBFB0236C6FD8636C893D6FB414C
:1020000036CEB7460F00938606243349D90285663B
:10201000938606FAB3969601B389E90213076055D1
:102020003309D90293060010B389E9023349D90272
:10203000B3C9F9029316390036CA37190040FD8634
:1020400036D0930D090493D7F9413ED2F33604807C
:1020500093F6860836DC01000100930770052380A3
:10206000FD00930680FA2380DD0001000100834615
:10207000390593F6860FA309D9048346390593E6FB
:102080001600A309D90423800D00E256F3A60680AA
:1020900001000100130C80FA116DF336048093F6F1
:1020A000860836DE01000100930770052380FD00DD
:1020B00023808D010100010083463905216693E6E6
:1020C0000602A309D90483560905B3E6A60123181D
:1020D000D90483560905D18E2318D90423800D0015
:1020E000F256F3A60680010001008346390593F6F7
:1020F0000602638A061803463905218A6DDE081830
:10210000EF0010047336048013768608B2C2010013
:10211000010023809D0023808D0101000100B7177D
:10212000004003C637051376F60DA389C70403C61E
:10213000370513660602A389C7048356090521667D
:10214000B3E6A6012318D90483560905D18E2318B6
:10215000D90423800D009646F3A6068001000100F5
:102160008346390593F606026386061483463905CD
:10217000A18AEDFE97000020E780E0F1AA8636D420
:1021800097000020E78020F1A256E30AD5FE83568F
:1021900009054255B3E6A6012318D904C127834691
:1021A0003905A18AEDDE03560905834629058247D4
:1021B0003376CA00B306DA0293D5F641B296B388F5
:1021C000F640E24733B8C6002E983308F840A247DD
:1021D000B3B616013308D84063C70701631DF80082
:1021E000924763FA1701C247634DF80E63950701E2
:1021F000B24763E8F80E894663E7660FF246931527
:10220000180013D3F8015E8613951800B365B30068
:1022100042D646D4EF30703F3258050B137BFB0F8C
:102220006347000163120838A258638F0836130809
:102230001500B336A800B69513D6F5013298B3361B
:10224000C800AE9613581800FE06B3E606017336B2
:10225000048013768608B2C60100010023809D0029
:1022600023808D01010001000356C902B296C20607
:10227000C1822316D90223800D00B646F3A606803C
:102280000100010019BDF336048093F68608B6C03C
:102290000100010023809D0023808D0101000100C9
:1022A0008346390593E60602A309D90423800D006D
:1022B000864605BDF336048093F68608B6C4010051
:1022C000010023809D0023808D01010001008346D1
:1022D000390593E60602A309D90423800D00A6461A
:1022E000A5BDE30D0BF0F336048093F68608B6C85F
:1022F00001000100930680FA23809D002380DD0009
:10230000010001008346390593F5FC0F93F6860F13
:10231000A309D90483463905CD8EA309D9042380A6
:102320000D00C646F3A6068001000100130580FAE1
:1023300003463905930639051D8A631496297336B9
:10234000048013768608B2CC01000100130680FADF
:1023500023809D002380CD000100010003C60600FC
:102360001376F60D2380C60003C606001366060228
:102370002380C600835609051166D18E2318D9041F
:10238000835609052166D18E2318D90423800D00B8
:10239000E646F3A6068001000100130680FA834694
:1023A000390593F606026388062483463905130C23
:1023B0003905A18AFDDA08186123F336048093F603
:1023C0008608B6D001000100930680FA23809D00A4
:1023D0002380DD000100010083460C00116693F6A6
:1023E000F60D2300DC0083460C0093E60602230072
:1023F000DC0083560905D18E2318D90483560905BC
:102400002166D18E2318D90423800D008656F3A6A9
:10241000068001000100130680FA8346390593F611
:1024200006026385062083463905A18AEDFE9700E2
:102430000020E78040C62A8C97000020E780A0C5D6
:10244000E30C85FF8356090511664255D18E23188A
:10245000D90429238346390513063905A18AFDDAF3
:10246000F336048093F68608B6D401000100930683
:1024700080FA23809D002380DD0001000100834657
:10248000060093F6F60D2300D60023800D00A65615
:10249000F3A60680010001008356090503462905BD
:1024A000D247B376DA003306CA021305800C93557F
:1024B000F6413696330DF6408257333CD6002E9CBB
:1024C0003336A601330CFC40330CCC403308850373
:1024D00092564E86B335A5033305A503C295EF305A
:1024E000D01263468001631E0C16630C0D16130692
:1024F00015003335A6002E959356F5013696B33563
:10250000D600AA959396F50105828585D18E6346FE
:10251000B000639D051A638B061A0356C902158223
:102520003305D6003336C500B2956348B0006391D9
:1025300005241306F00F637DA622894663F3561522
:1025400093078008F3B7078093F78708BED601008A
:10255000010037170040930770052300F704930725
:1025600080FA2300F704010001008356C70289673F
:102570008117D58FC207C1832316F70223000704F2
:10258000B657F3A7078001000100FA506A54DA54E5
:102590004A59BA592A5A9A5A0A5BFA4B6A4CDA4C87
:1025A0004A4DBA4D296182801308F5FF3335A800E2
:1025B000FD152E951356F5013298B336C800AA962C
:1025C00051B1F336048093F68608B6CA01000100C3
:1025D00023809D002380AD00010001008346390562
:1025E000CD8EA309D90423800D00D646F3A606801C
:1025F0000100010035BBF336048093F68608B6CEA1
:102600000100010023809D002380CD000100010016
:102610008346390593E60602A309D90423800D00F9
:10262000F646F3A606800100010095BBF336048050
:1026300093F68608B6D20100010023809D00238016
:10264000CD00010001008346390593E60602A30987
:10265000D90423800D009656F3A6068001000100E0
:102660006DBB9306F5FF33B5A600FD152E9593556A
:10267000F501AE96B3B5B600AA951396F50185821D
:1026800069B5F336048093F68608B6D801000100D8
:10269000930680FA23809D002380DD000100010065
:1026A0008356C9020566011693F6F60FD18EC2064F
:1026B000C1822316D90223800D00C656F3A60680D8
:1026C00001000100850A93FAFA0F49B233E6B60019
:1026D00045C20356C9023305D0403338A000B305C4
:1026E000B040B385054115826345B000D1E1637107
:1026F000A608894663F0560593078008F3B707805C
:1027000093F78708BEDA01000100B71700401307EE
:1027100070052380E704130780FA2380E704010093
:10272000010003D7C7027D8B2396E70223800704AD
:10273000D65781BDF336048093F68608B6DC0100D7
:102740000100930680FA23809D002380DD000100B4
:1027500001008356C9020566011693F6F60FD18E65
:10276000C206C1822316D90223800D00E656B9B7EE
:1027700093078008F3B7078093F78708BEDE010050
:10278000010037170040930770052300F7049307F3
:1027900080FA2300F704010001000356C702939753
:1027A0005600B297C207C1832316F702230007041D
:1027B000F657C1BB914763EEB702175700001307E6
:1027C000A72D8A05BA959C41BA978287B717004012
:1027D00003A7470B1345F5FF698F23AAE70A03A751
:1027E000070B698F23A8E70A03A7070A798D23A09F
:1027F000A70A8280B717004083A6470B1347F5FF4F
:10280000F98E23AAD70A83A6070B558D23A8A70AFA
:1028100083A6070A758F23A0E70A8280B7170040B6
:1028200003A7470B498F23AAE70A03A7070B134502
:10283000F5FF45BFB717004083A6470B1347F5FFC9
:10284000758F23AAE70A03A7070A598D4DB7B71753
:10285000004003A7470B498FEDB7914763EEB702DE
:1028600017570000130787248A05BA959C41BA9729
:102870008287B717004003A7470D1345F5FF698FFF
:1028800023AAE70C03A7070D698F23A8E70C03A76A
:10289000070C798D23A0A70C8280B717004083A670
:1028A000470D1347F5FFF98E23AAD70C83A6070D12
:1028B000558D23A8A70C83A6070C758F23A0E70CC2
:1028C0008280B717004003A7470D498F23AAE70C62
:1028D00003A7070D1345F5FF45BFB717004083A6B3
:1028E000470D1347F5FF758F23AAE70C03A7070CC5
:1028F000598D4DB7B717004003A7470D498FEDB766
:10290000B71700408847420541819377050491EB52
:102910009377F5013755E801130505803345F50236
:1029200082809377050C130700046397E700937781
:10293000F50137459C1CCDB72165130505D0828074
:1029400037E700E01C435443A183E206D58F1CC146
:10295000FD572320F7182322F718828013178500CC
:10296000B7E700E023A0E710618123A2A7108280CF
:10297000B7F700E08847CC4782808147373700406F
:10298000A14663C4C700328582800345B740E38E09
:10299000A6FE3385F5000345050085072304A740FF
:1029A000CDB797070020938767479C4317270020E0
:1029B0001307473B3E95636EE5001747002013075A
:1029C00067C46368A700170700202329A7443E8532
:1029D0008280FD57EDBF411122C406C62A840D37FF
:1029E0002947B307E502B2408D83B3D7870222445B
:1029F0009507B3D7E70237370040C207C1832316D4
:102A0000F70041018280716541111305052006C65A
:102A1000D937B7370040130770F82381E7000D4717
:102A2000A381E70013070004A380E700054723877D
:102A3000E700B240410182803737004083472700DA
:102A40001A0593F7F703C98F93F7F70F2301F700E0
:102A50008280B737004003C7170019C9D98DA380FA
:102A6000B70003C70700136787002380E700828051
:102A700093C5F5FFF98DA380B7008280AE872A87C2
:102A8000B736004021463738004099E36F10A05D0B
:102A900083C8B600E30B16FF05078348F7FFFD1751
:102AA000C20723041801C183CDB7411122C406C651
:102AB0002A84B9352947B307E502B2408D83B3D7DD
:102AC000870222449507B3D7E70237370040C20791
:102AD000C1832316F74041018280716541111305BE
:102AE000052006C6D937B7370040130770F8238191
:102AF000E7400D47A381E74013070004A380E740A8
:102B000005472387E740B24041018280CC41411113
:102B100006C6328503C6150083C5050022064D8E04
:102B200042068D654186138875A2630C0611634BBE
:102B3000C804138845A26300060D634AC800938544
:102B400035A26301B6082390060029464DA01388DC
:102B500055A26305060D938565A2E316B6FE8D4565
:102B60001D4663E6E5081146198E63F3C7003E86ED
:102B7000B7E704002390C600FC47976500009385E3
:102B8000E5879DA0138895A263030611634E060D89
:102B90001388A5A263000613938505A5E315B6FA6D
:102BA00099451D4663E5E504198E63F3C7003E862B
:102BB000B7E704002390C600FC47970500209385E3
:102BC00065261DA09D451D4663E3E5022146198E3D
:102BD00063F3C7003E86B7E70400FC472390C600B6
:102BE0009705002093858526BA9582970146B240C5
:102BF000328541018280AD451D46E3EAE5FE31465E
:102C0000198E63F3C7003E86B7E704002390C60021
:102C1000FC4797550000938565ECF9B7B1451D4613
:102C2000E3E7E5FC3546198E63F3C7003E86B7E758
:102C300004002390C600FC4797550000938505EBE0
:102C400065B78D451D46E3E4E5FA1146198E63F339
:102C5000C7003E86B7E704002390C600FC4797559F
:102C600000009385657A49B78D451D46E3E1E5F897
:102C70001146198E63F3C7003E86B7E70400239020
:102C8000C600FC47975500009385C579B1BFA5459F
:102C90001D46E3EEE5F42946198E63F3C7003E8630
:102CA000B7E704002390C600FC47975500009385C2
:102CB00025E21DBFB5451D46E3EBE5F23946198E09
:102CC00063F3C7003E86B7E704002390C600FC47C5
:102CD000975500009385C5DE01BFB7E7040003A345
:102CE000071397060020938666F04146A545170511
:102CF00000201305A5E602832D4559EF03C5050005
:102D000009476317E50803A84500411106C60347B4
:102D1000180032850346080022074168518F930846
:102D200028FE6308170363E9E80005186303070535
:102D30002390060029451DA8130648FE630BC70211
:102D40001518E31707FF15463E87637BF602154704
:102D500005A83E8691C30546B7E70400FC472390CB
:102D6000C6004206CC45418282970145B2404101EE
:102D700082801306700F3E876374F6001307700F8E
:102D8000B7E704002390E600FC4713160701D9BFFC
:102D9000239006000545828082804167791763048D
:102DA000E504411122C406C685472A84639FF500C5
:102DB000B7E7040022852244B24003A38713970596
:102DC0000020938565094101028389476399F500D5
:102DD000B7E7040083A7070B8545829771D9B240F6
:102DE0002244410182808280797122D452CC2E8487
:102DF0002A8A975500009385A5D117550000130521
:102E0000E5D206D63AC626D24AD0B68432894ECE0C
:102E1000EF308048A68517550000130525D2EF3006
:102E2000A0472945EF30804B8347840093F7070282
:102E3000E1E7834904008947054532476396F9086D
:102E4000544083C7160083C60600A207D58FC1660B
:102E5000138616FE638CC7028D16638FD7068D66A8
:102E60009386269029456391D706B7E70400A2858B
:102E7000225403A34714B250F249A6864A869254BC
:102E800002595285624A8547456102832D450DEFFF
:102E90009307700F354563E99702B7E70400FC47D5
:102EA00048441306700FCA8582978149970700200E
:102EB000938747FB9C43014581CB9C4391C74E853B
:102EC0002686CA8582970145B250225492540259EF
:102ED000F249624A456182802D457DF79307700F64
:102EE0003545E3E397FEB7E70400FC474844130683
:102EF000700FCA8582975DBF2145F9B7411122C481
:102F000037E404008327841326C2AA84416506C6D9
:102F100097050020938545F47D1582978327C40A81
:102F2000170500001305A5E78588829795C0032340
:102F300004132244B2409244970600209386C6DCD4
:102F40004146C54517050020130505CB4101028305
:102F5000B2402244924401454101828019C597073D
:102F6000002023A1A7F001458280454582801147BA
:102F7000636AA70A97560000938646B80A053695F5
:102F80001841411106C63697AE87B28502871307EE
:102F9000700F6145639DE700B7E70400FC47130627
:102FA000700F170500201305A5F382970145B24065
:102FB0004101828005476145E39BE7FEB7E70400D6
:102FC000FC470546170500201305C5E8F9BF1307A0
:102FD000700F6145E39DE7FCB7E70400FC4713066B
:102FE000700F17050020130525FFC1B71307700FD9
:102FF0006145E39EE7FAB7E70400FC471306700F4C
:10300000170500201305C50C4DB715476145E39022
:10301000E7FAB7E70400FC4715461705002013053B
:10302000E5E361B709458280411126C2B7E4040097
:1030300083A7C41322C44AC006C62E849705002065
:10304000938585E12A898297058905C59707002020
:10305000938787BA83D7A70BA28503A3440D2310B8
:10306000F4002244B24092444A850249014641019B
:103070000283B24022449244024949454101828080
:1030800097070020238207DE9707002023A007DE92
:10309000B717004003A7070CB706C0FFFD16758FD2
:1030A00023A0E70C03A7070DB7064000558F23A800
:1030B000E70C03A7070C3D9B23A0E70C03A7070D14
:1030C0001367070123A8E70C8280B717004003A508
:1030D000470C83A7470C598113451500C18B0589FF
:1030E00099E3136525009707002083C7E7D763801E
:1030F000A702970700202389A7D611C997070020A8
:103100009387C7D603A3070063030300028382806B
:1031100011456FE07FE0411193962500AA852D456A
:1031200006C697F0FF1FE7800064B24001454101E9
:103130008280011122CC06CE3714004026CA4AC82C
:103140004EC652C483447405034AB40583498405BA
:1031500003499405EFE03FB78347A40593F4F40FC8
:10316000137AFA0F93E71700230DF40493F9F90F7C
:103170001379F90FB717004003C7A705058B6DFF3B
:1031800003D5C705A38D4705238C3705A38C2705D9
:10319000A38B9704F2406244D2444249B249224A86
:1031A0000561828041119397050122C406C626C29B
:1031B000C1872E8463DC0700B7E40400FC548297C7
:1031C00019C1BC5482972165218D3DA093F715004C
:1031D00013C5150095E393F7250085C7FD35B7E7BF
:1031E0000400BC4F1306000A89451705002003455B
:1031F00065C8829713452400B2402244924441019D
:1032000082809397250163D50702B7E4040083A762
:10321000C41E8297F53DBC4C37F60200130606E04B
:103220008965170500200345E5C48297096569BFD4
:10323000939715010145E3D107FC175500001305CD
:10324000A596EF30201AB7E70400BC4F13060064C0
:103250009165170500200345E5C182971165ADB75B
:103260002D71232A9110FD74E98C232C81102328C1
:103270002111232631112A84AE8932899306001048
:103280000A86A6852D45232E111097F0FF1FE78093
:10329000804D13154401B7E70400FC4751810A052E
:1032A00013962900CA850A958297A68585660146E8
:1032B000254597F0FF1FE780004B0A86A6859306F9
:1032C0000010294597F0FF1FE780E0498320C111D6
:1032D0000324811183244111032901118329C11081
:1032E00015618280B7F7070003C70701411106C6C1
:1032F00022C426C24AC0A547631AF7009537B240D8
:1033000022449244024901454101828013942500E0
:10331000AA843289A286AA850146254597F0FF1F17
:10332000E7806044A2864A86A685294597F0FF1F5C
:10333000E7806043E9B71D71A2CC37E404005C5C10
:10334000485886CE494697550000938565818297F7
:1033500001E9175500001305E581EF30A00801A031
:10336000B7F600E0795798CAFD57DCCA0567B7E79A
:1033700000E023A0E7101306F00290C223A0E71894
:10338000010001003707002018471306000481459B
:103390009706002023AEE6AC4157A38AE7403C44A1
:1033A00008088297970700209387C7F33EC8856770
:1033B00013870760231AE1001D673ACC3707010520
:1033C000130707103ACE9387B7D31307B00F231014
:1033D000E1022312F102054797F7FFFF9387875910
:1033E0002301E1023ED817070000130707D3970710
:1033F0000000938747D4B7F50700BAC23EDC170731
:103400000000130767EE970700009387A7D0814657
:103410003000E1051945BAC43EDE97F0FF1FE78092
:10342000803418088147994630003E9603460600CE
:1034300085070507A30BC700E398D7FEC24791C7CE
:103440000357410185676373F70001A0B7E70400E4
:1034500083A7470A08088297AA8501C91745000073
:1034600013058572EF20506301A0F6406644256184
:103470008280411126C2B7E4040083A7040806C66F
:1034800022C417050000130525D2829717040020D7
:103490001304449E2300A4003128DD3603450400B4
:1034A000224403A38405B240924413060032896586
:1034B00041010283797106D622D413078008F337BD
:1034C000078093F787083EC201000100B71700404C
:1034D000930570052380B704130680FA2380C70480
:1034E0000100010083C6F70293F6A60FA387D70257
:1034F000238007049246F3A606800100010073377B
:103500000780137787083AC4010001002380B704BD
:103510002380C7040100010003C7F70213672700D7
:10352000A387E70223800704A247F3A707800100CF
:1035300001000545EFE06FFCE13E01478146814710
:10354000054685451305407EEFE01F8037E4040003
:103550003C446800514681458297B707C0A83EC8E1
:10356000B787E803938707D03ECA97F7FF1F938773
:1035700007E43EC67C5868008297B25022544561E9
:103580008280011122CC37E404008327041A06CE7E
:103590008297EF20E05A8547A307F100832744175D
:1035A0001306F1008545130550308297174500003A
:1035B0001305C55FEF201063F2406244056182800D
:1035C0008280411122C491462A84170600201306E6
:1035D00066D09D652D4506C697F0FF1FE780A018B1
:1035E000B7F7070003C70701A5476313F70001A05A
:1035F0009306001001469D65254597F0FF1FE78063
:10360000801697070020238787CC2244B24091463A
:1036100017060020130606CC9D652945410117F3C6
:10362000FF1F670043145171CAD137E90400832793
:10363000C904A2D52E8686D7A6D32E84AA851705BF
:103640000020130565B982979707002083C7C7B884
:103650001307700A638BE70E636CF7001307600AA9
:103660006382E704BE502E549E540E596D618280D1
:103670001307800A638AE7141307900AE394E7FEAE
:103680008D476309F41A974500009385E55D17455A
:1036900000001305A549EF20304017450000130531
:1036A000E55915A08D476306F40297450000938500
:1036B000A55B1745000013056547EF20F03D174552
:1036C00000001305E550EF20303D2945EF20104163
:1036D00051BF8547174500001305455117F7FF1FD8
:1036E000230EF778EF201050B7750200B76602007E
:1036F0000146054597F0FF1FE780E006930760F855
:1037000017070020230AF7AC97070020A38707AC10
:1037100093070026170700202322F7ACE57793874D
:10372000072117070020231DF7AAB145970700209E
:10373000238907AA97070020A385A7AA17050020B9
:10374000130585A9EF20006331BF914763E187022C
:103750009745000093854551174500001305053D29
:10376000EF209033174500001305454AA9BF970481
:10377000002083C4A4A69707002083C717A6A2042D
:10378000DD8C8327C9046D1422869705002093855C
:10379000F5A4280082978E0493160401B7750200E1
:1037A000C1823000A695094597F0FF1FE780A0FB76
:1037B000930770F8170700202300F7A29945970791
:1037C0000020A38DA7A09DBF914763E18702974585
:1037D0000000938565491745000013052535EF2046
:1037E000B02B174500001305E543F1BD97040020F9
:1037F00083C4C49E9707002083C7379EA204DD8C34
:103800008327C9046D142286970500209385159D92
:10381000280082978E0493160401B7750200C182B6
:103820003000A6950D4597F0FF1FE780C0F3930782
:1038300080F849B71745000013058541EF20903AFD
:103840001305C01297F0FF1FE780E0AE0145EFF0CF
:103850002F8F0D45BD33294597F0FF1FE780A0ADA1
:1038600097F0FF1FE780C09EF5BB41114AC097F655
:10387000FF1F83D60661328917F6FF1F0356665B6A
:1038800022C426C206C6AA842E84F52E6306090227
:1038900097F7FF1F83C7975E85C319CC97F7FF1F64
:1038A00083C7C75D91EBA2852244B24002492685B9
:1038B000924441016F20004CB2402244924402499C
:1038C000410182808347550083454500174500002C
:1038D0001305453CA207DD8D6F20101C1745000025
:1038E0001305453A6F2010308D4763F2B70A011176
:1038F00026CA06CE22CC0344350097F4FF1F83C4AA
:103900000458974500009385253AB337800017F790
:10391000FF1F2306F75609C4974500009385853994
:103920001745000013058539EF20101797F7FF1F83
:1039300083C7E75463839700812497F7FF1F83C7EA
:1039400007549DC385472306F100B7E7040083A70A
:1039500047177000854513055030829717450000C2
:103960001305C536EF2010289967938757EE231665
:10397000F100680085479145A30781002307F10006
:10398000EF20403FF2406244D24405618280828051
:10399000894763F2B708011122CC06CE26CA8344B8
:1039A000250085472A846398F404914763F0B7049F
:1039B000034545008347340022055D8D97F7FF1FBF
:1039C0002399A746A9269967938767EE2314F100E8
:1039D0008347340023059100A305F1008347440089
:1039E000954528002306F100EF20C038F2406244DC
:1039F000D24405618280FDF89967938767EE2314AE
:103A0000F10097F7FF1F83D7C742A305F1002305F5
:103A10000100A183F1B782800111996722CCD517EB
:103A200017F4FF1F1304B4452314F1008347040067
:103A300026CA97F4FF1F9384C4442305F10083D75B
:103A4000040028009545A305F100A18306CE2306B6
:103A5000F100EF20203203D604008345040017450F
:103A6000000013052528EF203003F2406244D244C1
:103A7000056182809D677971D9172316F10097F748
:103A8000FF1F83C7D73F06D62307F1008DCFB7E7C7
:103A90000400FC47414697F5FF1F9385E572130527
:103AA000F10082976800CD45EF20C02C97F5FF1FED
:103AB00083C5F53C174500001305C525EF20C07DE3
:103AC000B25045618280B7E70400BC47414681455A
:103AD0001305F1008297F9B7B767020369719387FD
:103AE00057AA3EC48567938727602316F10097F78E
:103AF000FF1F9387D73883C7070023248112A307AA
:103B000001002307F10097F7FF1F9387873783D7BB
:103B1000070037E40400232611122318F10097F759
:103B2000FF1F9387073183D70700414648082319B1
:103B3000F1007C4497F5FF1F938505698297F14555
:103B4000280011222312A1027C442C00281079465F
:103B500082973C44130561041306900D81458297BA
:103B600030109305700F0145EFF06FC08320C11234
:103B70000324811255618280B7C7A55A011193872A
:103B8000C7333EC497F7FF1F83C7672F3EC6B7F7FB
:103B9000070003C7070106CE22CCA5476313F70031
:103BA00001A01164930504F0930600100146254519
:103BB00097F0FF1FE78020BB3000930504F0A1467B
:103BC000294597F0FF1FE78000BA97F5FF1F83C5CF
:103BD000052B174500001305651EEF20E06BF24032
:103BE00062440561828001119165A1463000938590
:103BF00005F02D4506CE97F0FF1FE780C0B622479F
:103C0000B7C7A55A9387C7336312F702B245174562
:103C1000000013056512B335B00097F7FF1F23802E
:103C2000B726EF206067F240056182808145174525
:103C300000001305A51297F7FF1F23820724EF202A
:103C4000A0651D3FCDB7C16769768146FD170506A2
:103C50001397060141836364B7003E858280330772
:103C6000D50003470700B98F214713F81700858354
:103C700063050800B18FC207C1837D171377F70F63
:103C80006DF78506F1B749C1A547054763FFB7063C
:103C900083471500034705003168A207D98F1397A2
:103CA0008700A183D98FC207C1831308C855054770
:103CB000639D0705411106C622C426C203442500A0
:103CC000914763FD8702930754006399F502A301AE
:103CD000C50021822302C5009304340091C6A302CB
:103CE000D500A1822303D5002A84A685A93F269466
:103CF0002300A4002181A300A4000147B240224474
:103D000092443A854101828005473A858280B7C74F
:103D1000A55A01119387E7343EC42AC6B7F70700B6
:103D200003C7070106CE22CC26CAA5476313F700B6
:103D300001A091642A84938504EE93060010014645
:103D4000254597F0FF1FE78000A23000A14693852C
:103D500004EE294597F0FF1FE780E0A0A2851745F4
:103D600000001305A507EF202053BD33F240624445
:103D7000D2440561828001119165A146300093858E
:103D800005EE2D4506CE97F0FF1FE780C09D224728
:103D9000B7C7A55A9387E7346313F702B2451745AF
:103DA00000001305A5FD97F7FF1F2394B708C20570
:103DB000C181EF20604E0D33F24005618280D14712
:103DC000D14517450000130565FD17F7FF1F2312A6
:103DD000F706EF20604C17F5FF1F03558505053FDB
:103DE000E1BF411126C206C622C493F71500AE8476
:103DF0008DCBAD67371700409387A7AA1CC3B7E7E1
:103E00000400BC4F13060019854517F5FF1F034535
:103E10003502829713C51400B240224492444101F6
:103E2000828093F72500F1C797F5FF1F83C54505ED
:103E3000854793C4240063E7B70289CD97F7FF1F36
:103E400083C7D70381CB854517150020130585A9A6
:103E5000EF1050721395040197F7FF1F238207029A
:103E600041815DBF171400200344C4A797170020A9
:103E700083C757A722045D8CAD679387B755630E40
:103E8000F40463ED8700A9679387A755630DF404D5
:103E900097F7FF1F83C797FE8DCB19A8B16793874C
:103EA000C755630EF400B5679387D755E312F4FE48
:103EB00017150020130505A3EF10D06B39A0054698
:103EC00017150020130505A24D32A28517450000E5
:103ED000130585F2EF20403CB5BF171500201305F0
:103EE00065A0CD32DDB7171500201305A59FFD3263
:103EF000E9BF93F74500014585D317450000130539
:103F0000E5F0EF20204EEF10906D13C5440029B767
:103F10001567B71700401307575598C3D8439D66D8
:103F2000558FD8C3D843FD76758FD8C3D843136750
:103F3000F70FD8C335671307C7CC98C382804111E8
:103F40001305800406C622C426C23714004097E039
:103F5000FF1FE780C0158327840A8D4513050020C5
:103F600093E707202324F40AEFE0DF84B7E404009A
:103F7000EFE0BFB6C858EF20E0468327840C8545A4
:103F8000414593E707082324F40CEFE01F8D8D458E
:103F900013050008EFE07F8CEFE0FFA60145EFE09E
:103FA000BFA985450545894717F7FF1F230CF7EC87
:103FB000EFE03FAA37070004B7E700E023A0E710CF
:103FC000EFF06FB7EFF0EFCA39397533EFF06FDB11
:103FD0008D28352083A70408170500001305A5E0E8
:103FE000829797F7FF1FA385A7E4BC4C13060064D4
:103FF00085458297313F97E0FF1FE780603E411182
:104000000D658D4506C6EFE05F85B71700408D66EC
:1040100023A6D70C171500201305C59C1387C70CC2
:104020009387870C1CC15CC5856689675CC958C1CC
:1040300014C518C9B7E70400B24003A3871E4101A5
:10404000028397F7FF1F83C7F7E389EF411106C685
:10405000EF10404FB240854717F7FF1FA304F7E268
:1040600041018280828097F6FF1F83C6B6E189C630
:1040700001C599C16F10004E8280171600201306EB
:10408000E6978147B2861303F00FA9483308F6007C
:104090000348080013F7F70F6303A80C63066800D2
:1040A0008507E39517FF2947B387E6002380A7001C
:1040B00097170020938747957DA0411113D765007E
:1040C0001347170006C693F63500058B954791CA2E
:1040D000054699476387C60009469D476383C60026
:1040E000A14713F645003336C00093F68503050655
:1040F00085C2A1456389B604E1456388B60493058A
:1041000080026386B604930580036393B6009146EC
:1041100097F5FF1F2387F5D897F5FF1F2382C5D892
:1041200097F5FF1FA38ED5D6BE8517450000130552
:1041300065D1EF206016B240854717F7FF1FA30235
:10414000F7D6410182808546E1B78946D1B78D46D1
:10415000C1B717450000130565D16F20E01317178D
:1041600000201307678ABA972380B700E147E30668
:10417000F5F493077002E30EF5FC82802A87238012
:104180000500814717150020130545871308F00F18
:104190002946B306F50083C606006396E602971625
:1041A000002093866686B69783C70700054523805F
:1041B000F5009947636EF7029D4763FDE700E1470D
:1041C000630DF7008280638506018507E393C7FCD2
:1041D0000145C5B7238005008280B737004003C77B
:1041E000370083C7050093F70704D98F2380F500B4
:1041F0008280797126D24AD097F4FF1F83C444CCC1
:1042000017F9FF1F130909CB06D622D44ECE52CC84
:1042100056CA5AC8B307990083C7070093F7F70F28
:10422000A5C79387140093F7F70F0D476361F70C49
:1042300017F7FF1F2306F7C897F7FF1F938707C8D5
:10424000A69783C707001307100293F7F70363834A
:10425000E7286363F70A0544638A871EE3810766DC
:1042600009476389E71413070002E388E750B7E7BB
:1042700000E03707400023A0E71801000100CA94BE
:104280002380040023A0E710B787004003C767001E
:10429000058BE305077097F6FF1F83C686C20547A7
:1042A000E390E66E29472381E70209472383E7026B
:1042B0002385E70297F7FF1FA38607BE97F7FF1F27
:1042C000A38107C0B7870040A381070017F7FF1F2E
:1042D000A30C07BC05472383E700B2502254925435
:1042E0000259F249624AD24A424B4561828097F7AD
:1042F000FF1F238707BC89B7130730026386E70ACD
:1043000063E0E71413074002638AE708130700031A
:10431000E39FE7F497F7FF1F938707BAA69703C7B2
:104320000700A1471377F70FE316F716170A0020C7
:10433000130A4A6E83476A0097F6FF1F238BF6B471
:104340009707002083C7776D91C7FD5797F6FF1F2A
:104350002381F6B49705002083C5D56B97F7FF1F1F
:10436000A389B7B29707002083C7C76A93F90708E4
:104370009306000493F707066399D74E9307A009A5
:104380006381F51A63EEB7149307F0056380F54C6B
:10439000930750096384F52C01449DA3FD5717F73B
:1043A000FF1F2307F7AEE1B5FD5717F7FF1F2300E7
:1043B000F7AE75BD17450000130585BBEF208002E1
:1043C00097F7FF1F938747AFA69703C4070081495C
:1043D000170A0020130A0A7C1374F40F974A00008E
:1043E000938A8AB963C589042945EF10306F8547E0
:1043F00017F7FF1F230CF7A817F7FF1FA30887A8BD
:1044000017F7FF1F2300F7AA37E700E0B7064000C1
:104410002320D71801000100378600408347A602F9
:1044200093F7370F2305F6022320D71089B5B3077A
:104430003A0183C5070056858509EF10F0655DB721
:10444000854717F7FF1FA302F7A415B5174500000E
:10445000130505B2EF10107997F7FF1F9387C7A5D3
:10446000A69703C407008149170A0020130A8A6629
:104470001374F40F974A0000938A0AB063C3890447
:104480002945EF10B065854717F7FF1FA30EF79E6C
:1044900017F7FF1F230B879E17F7FF1F2304F7A0B3
:1044A00037E700E0B70640002320D71801000100DD
:1044B000378600408347660293F7370F2303F602DF
:1044C000A5B7B3073A0183C5070056858509EF10E4
:1044D000B05C6DB7854717F7FF1F2307F79A41BBFD
:1044E0009307400A638FF5329307200B638AF534F4
:1044F0009307100AE392F5EA83072A00014463D187
:1045000007409707002083C7175193F63700638051
:10451000061A05466380C6220946639BC6181D47D6
:1045200041AA170500200345054FC947170A002077
:10453000034A7A4E9705002083C5054E17040020D4
:104540000344944D6317F510CD476314FA10930795
:104550007008639AF5021307300FB7170E0063084F
:10456000E4001307900DB7B704006312E40817F7CF
:10457000FF1F2325F792BE8517450000130545A0B0
:10458000EF10905111BD93078008639DF50033042F
:104590008040B77746001374F40F938787CDB3D765
:1045A0008702F1B793079008639AF50033048040BF
:1045B00091671374F40F9387C766D5B79307A00864
:1045C000639BF50033048040B7173D001374F40F6C
:1045D00093870790E9B79307B008639AF50033040F
:1045E000804091671374F40F938797D04DBF93F574
:1045F000F5078D47639BF50033048040B7975B0058
:104600001374F40F938707D859BF8947639BF5004C
:1046100033048040B7770B001374F40F9387071BA4
:10462000BDBF8547639AF50033048040DD6713748E
:10463000F40F938767E3A5B789E9330480408D675A
:104640001374F40F938777DC99BFF1679387072082
:1046500039BF2534A28552850D343DBB93056100D9
:10466000170500200345253B170400200344B43AF6
:10467000313693057100228511363C0017F7FF1F74
:104680002328F782834761002304F10083477100E8
:10469000A304F100894717E7FF1F230CF77E835718
:1046A0008100170700202317F736094491AC1547FE
:1046B00093F64700B336D00093F78703850685C38A
:1046C0002146638BC7066146638AC70613068002CC
:1046D0006388C706130680036393C700914717E6F4
:1046E000FF1F230FD67A97E6FF1FA38BF67A97E773
:1046F000FF1F2388E77A170700200347E7319376E7
:1047000007049707002083C737318DEE1377770CA6
:1047100093067008630CD7021377F7078D46631E64
:10472000D70AB307F040B7955B0093F7F70F93856F
:1047300005D881A81947ADBF854755B7894745B703
:104740008D4771BF930670086311D7021307300FAE
:10475000B7150E006389E7021307900DB7B5040083
:104760006383E7021307700845BF9306800C63114B
:10477000D702B307F040B775460093F7F70F93855C
:1047800085CDB3D5F50297E7FF1F23A9B770EDB329
:104790009306900C631AD700B307F040916593F726
:1047A000F70F9385C566F1BF9306A00C631BD70076
:1047B000B307F040B7153D0093F7F70F93850590C9
:1047C000C9B79306B00CE319D7F4B307F04091656D
:1047D00093F7F70F938595D06DB78946631BD70084
:1047E000B307F040B7750B0093F7F70F9385051BE0
:1047F00049BF8546631AD700B307F040DD6593F7DC
:10480000F70F938565E3B5BF09EBB307F0408D65FE
:1048100093F7F70F938575DCADB7F16593850520A8
:104820009DB783472A00C18B99C7854717E7FF1FAC
:104830002304F76695B697E7FF1F238F0764A9BE89
:10484000854717E7FF1FA30EF764B9B63C0017E7CB
:10485000FF1F232FF7640947930700032314F10078
:1048600097E6FF1F2387E6622DBD639C0754A94787
:1048700063E2B742173700001307075A8A05BA9553
:104880009C41BA978287170400200344D418094A30
:104890006308440F636A8A0885476307F40A93072D
:1048A000F00F17E7FF1F0347C75E63F6E70017E740
:1048B000FF1F2300F75E17EAFF1F034A8A5D930775
:1048C00000041374FA0F63F447011304000497E71C
:1048D000FF1F9387E75D83AA070022861705002044
:1048E00013054513D685330A8A40A29AEF10700F3C
:1048F00097E7FF1F238F475997E7FF1F23AA575BAF
:1049000097E7FF1F83C7F75815476390E75EB7E740
:1049100000E03707400023A0E71801000100B78638
:1049200000402380860239A58D476306F40A994723
:10493000E317F4F6973700009387875417E7FF1FB4
:104940002328F756A947B1BF17E7FF1F034767574B
:1049500097070020938707304946973500009385D5
:10496000E55A6306870097350000938565563E85B6
:10497000EF10300717E7FF1F232CA752C94715B7C1
:1049800097E6FF1F83C6E6530547970700209387E6
:10499000672C6392E6023E8513067002973500008D
:1049A00093854554EF10F00317E7FF1F2322A7500C
:1049B00093077002FDB53E8513063004973500005D
:1049C0009385C54CEF10F00117E7FF1F2322A74E78
:1049D00093073004F9B59705002083C5C503173543
:1049E00000001305255BEF10300B854A17EBFF1F06
:1049F000034B2B4D9705002083C5E50117350000BB
:104A00001305455963145B0BEF101009970700203D
:104A100083C76700A5CBE364F4E8174400001304E0
:104A2000E4A3638C6701173400001304E451638628
:104A30004701173400001304A4522285EF10B0225E
:104A40001375F50F9307150086071707002023033A
:104A5000F7208D4717070020A30EF71E97070020A9
:104A60009387471F0147BE861376F70F8907636553
:104A7000A60297E7FF1F23ADD7429707002083C701
:104A8000671D05B5974700009387879C17E7FF1FB1
:104A90002320F742914731B53306E4000346060070
:104AA000A380070005072380C7007DBFEF10C07EED
:104AB0009707002083C727F6F1D7E362F4DE174497
:104AC000000013042499638C570117340000130469
:104AD000244563864701173400001304E44522850A
:104AE000EF1070181375F50F930715008607170759
:104AF00000202301F7168D4717070020A30CF71499
:104B000097070020938707150147BE861376F70F96
:104B10008907E370A6F63306E40003460600A38087
:104B2000070005072380C700D5B79705002083C578
:104B300085EE173500001305A546EF10E07597E7E1
:104B4000FF1F83C7B73693E7470017E7FF1FA30F81
:104B5000F73483472A0017E7FF1FA307F7346FF0E6
:104B6000BF83173500001305E544EF10B00797E742
:104B7000FF1F9387673383C7070017070020230BA6
:104B8000F7E817E4FF1F0344C430333480008DBBC3
:104B90001735000013054543EF10D00497E7FF1FBA
:104BA00083C7D73093E7070117E7FF1FA300F7304C
:104BB00083472A0017E7FF1F2308F72E6FF0CFFD6A
:104BC0001735000013058541EF10D00103470A0097
:104BD0007D8B51EFB787004003C767021377C70B80
:104BE000136727002383E70203C7A7021377C70BC6
:104BF000136727002385E70203C7E7021377C70B74
:104C0000136727002387E70203C727031377C70B20
:104C1000136727002389E702854717E7FF1F23054E
:104C2000F72617E7FF1FA302F72617E7FF1F23004A
:104C3000F72617E7FF1F230DF72497E7FF1FA3852C
:104C4000072497E7FF1F2383072497E7FF1FA3800D
:104C5000072497E7FF1FA38D072297E7FF1FA38372
:104C6000072497E7FF1FA38E07246FF0EFF2894711
:104C70006312F7029707002083C707DA9146638C17
:104C8000D70863E0F604638EE70C6369F70A05470B
:104C90006380E70EFD5717E7FF1FA30CF71E3707CA
:104CA0004000B7E700E023A0E71801000100B78645
:104CB00000401306F0FC2381C60223A0E7106FF02A
:104CC0000FDB130720086382E7086362F70213070C
:104CD0001008E391E7FC378700408347670293F7AA
:104CE000C70B93E727002303F7026FF0EFEA1307E0
:104CF00030086389E70213074008E39DE7F8378728
:104D000000408347270393F7C70B93E72700230946
:104D1000F7026FF06FE8378700408347270393F768
:104D20003707F5B7378700408347E70293F7C70B8C
:104D300093E727002307F7026FF00FE6378700405D
:104D40008347E70293F73707F5B737870040834774
:104D5000A70293F7C70B93E727002305F7026FF02D
:104D6000AFE3378700408347A70293F73707F5B7CC
:104D7000378700408347670293F73707ADB717358A
:104D800000001305A526EF10E06597070020238398
:104D900007C8C5BB1735000013054526EF10806412
:104DA00097070020239807C697E7FF1F9387670E92
:104DB00003C40700894763F3870009441374F40FA1
:104DC00081B613070002E397E7EC639F0908638D40
:104DD000F500930720026389F506173500001305D7
:104DE0006525EF10604B7DB5173500001305C52113
:104DF000EF10405F0144173B0000130B2B22A14A28
:104E0000B3078A0083C507005A850504EF10C04820
:104E1000E31854FF17350000130505DFEF10805C21
:104E200017040020034444BF11E497E7FF1FA38C3D
:104E30000704F9B48947E31FF4E4854717E7FF1F28
:104E4000A303F7046FF04FD5170600200346B6BC46
:104E50009705002083C525BC173500001305851C68
:104E6000EF1080436FF04FD3638DF504930710026A
:104E7000E395F5F69705002083C505BA17350000C0
:104E80001305451CEF10404197E7FF1F23A247037E
:104E900097E7FF1F93878700944383D7470017E75F
:104EA000FF1F03470700170600202325D6B61D4421
:104EB000970600202392F6B697070020238FE7B4C9
:104EC00081B49705002083C525B51735000013056B
:104ED000E518EF10603C97E7FF1FA38607FA9707D6
:104EE0000020239907B26FF04FFC2547E381E7A22A
:104EF00019476391E702B786004023808602B7E72F
:104F000000E03707400023A0E71801000100130666
:104F100000FC55B31307100A6391E702B7860040FF
:104F200023808602B7E700E03707400023A0E71898
:104F300001000100130680FCBDBB1307A009E38F2D
:104F4000E7FC1307400AE38BE7FC13072002E3802A
:104F5000E79C0547E38DE79AB7E700E03707400095
:104F600023A0E718E39B099A01000100B7860040DF
:104F700023808602130620FC3DBB17E7FF1F034773
:104F800057F16304F71E63E7E7029547630CF70EDA
:104F900099476308F704B786004023800602B7E705
:104FA00000E03707400023A0E718010001001306C6
:104FB000A0FC11B39307F005630AF70093075009AB
:104FC0006306F70093071002E317F7FCB7E700E06A
:104FD0003707400023A0E71801000100B786004012
:104FE00051BF97E9FF1F83C9C9EA93070004CE8A1E
:104FF00063F43701930A000497E7FF1F938747EB99
:1050000003AA070013F4FA0F2286D28517050020A1
:10501000130545A0EF10E01CB3878940529417E7B1
:10502000FF1F2308F7E697E7FF1F23A387E8638E98
:105030000902B787004023805703B7E600E0370630
:10504000400023A0C6180100010003C72702134730
:1050500007042381E70203C727021377C70F2381C1
:10506000E70223A0C6106FF08FA0B7860040238010
:105070000602B7E700E03707400023A0E718010069
:105080000100CDBD378700408347370097E6FF1FFB
:1050900083C696E193F70708D58FA301F700B706FB
:1050A0004000B7E700E023A0D71801000100130675
:1050B000A0FC2301C70223A0D7106FF04F9B97E7F6
:1050C000FF1F938767DFA69783C7070093F7F70F44
:1050D000C9CF97E7FF1F83C7C7DEC1EB17E7FF1FE5
:1050E000034737DB930700026311F7089707002097
:1050F0009387479203AB0700970A002083CACA919F
:10510000170A0020034A5A919709002083C9E990A1
:10511000D2875687CE865A8697E5FF1F83C5B5D6B8
:1051200017350000130505F5EF10001797E7FF1F6F
:1051300023A667D797E7FF1F238457D797E7FF1F5B
:10514000A38047D797E7FF1F238D37D597E7FF1F2A
:10515000238B87D2B7E700E03707400023A0E7188A
:1051600001000100B7860040F1B3B7E700E0370760
:10517000400023A0E71801000100B786004005BDEC
:1051800029472381E70209472383E7022385E702B2
:105190002387E7022389E7026FF0CF9103C76700F7
:1051A000118B630C079283C75700918BB5CF17E71C
:1051B000FF1F034707D185476313F70697E7FF1FD4
:1051C000A381E7CE97E7FF1F238007CC97E7FF1F58
:1051D000A38D07CA97E7FF1F238B07CA97E7FF1F17
:1051E000238807CA97E7FF1FA38007CA97E7FF1F17
:1051F000238E07C897E7FF1FA38B07C897E7FF1FFA
:10520000A38807C897E7FF1FA38E07C897E7FF1F6C
:10521000A38907CAB787004011476FF0CF8B17E704
:10522000FF1F2302F7C679BF854717E7FF1F230D2E
:10523000F7C417E7FF1FA30AF7C417E7FF1F2308E8
:10524000F7C417E7FF1F2305F7C469BF854717E7B2
:10525000FF1F230BF7C217E7FF1FA308F7C217E7CB
:10526000FF1F2306F7C217E7FF1F2303F7C217E745
:10527000FF1FA30B07C017E7FF1F230907C017E78E
:10528000FF1FA30607C097E7FF1FA38307C0828005
:10529000411106C6653FB78700402380070013070A
:1052A00040FC2386E7001307C004A386E70017F736
:1052B000FF1F130727762398E70017F7FF1F130731
:1052C0006779239AE700170700201307A784239C18
:1052D000E700170700201307E78F239EE700294701
:1052E0002381E70209472383E7022385E702238717
:1052F000E7022389E702A3810700930600F8A38051
:10530000D700930690022380D700FD562383D70051
:105310002381E700B706400037E700E02320D710DD
:1053200003C7170013671700A380E700B24097E791
:10533000FF1F239B07B641018280411106C6393702
:10534000B787004023800700130700FC2386E7008F
:105350003147A386E70017F7FF1F1307A76B2398B2
:10536000E70017F7FF1F1307E76E239AE70017F709
:10537000FF1F1307277A239CE70029472381E702B1
:1053800009472383E7022385E702A38107009306E9
:1053900000F8A380D700930690022380D700FD5623
:1053A0002383D7002381E700B706400037E700E0FA
:1053B0002320D71003C7170013671700A380E70047
:1053C000B24097E7FF1F239107AE41018280F1674A
:1053D0009387072017E7FF1F2322F7AC854717E7BE
:1053E000FF1F231FF7AAA14717E7FF1F230BF7AAE9
:1053F00097E7FF1FA38707AA97E7FF1F238407AA42
:1054000097E7FF1FA38107A897E7FF1F238D07A634
:10541000814717F5FF1F1305655EFD5517F6FF1F42
:105420001306865E2947B306F5002380B600B3064F
:10543000F600238006008507E397E7FE97E7FF1F46
:10544000238A07A697E7FF1FA38607A697E7FF1FF4
:10545000238307A697E7FF1FA38E07A297E7FF1FE7
:10546000A38C07A297E7FF1F238707A297E7FF1FD9
:10547000238207A297E7FF1F238107A297E7FF1F59
:10548000A38B07A097E7FF1F238807A097E7FF1FBD
:10549000A38307A2828017E7FF1F034787A28547E0
:1054A0006313F70059BDEDB3411122C406C617E7D7
:1054B000FF1F034707A185472E8613F4F50FAA8522
:1054C0006315F70417F5FF1F1305C568EF0070514A
:1054D00097E7FF1FA38B079AB787004023848702B3
:1054E000B7E600E03706400023A0C618010001001F
:1054F00003C7A7021377C70F2385E702B2402244F0
:1055000023A0C61001454101828017F5FF1F130536
:105510006558EF00104D97E7FF1F23870796B78761
:10552000004023828702B7E600E03706400023A050
:10553000C6180100010003C767021377C70F238352
:10554000E7026DBF411106C65935B2404101A1B70E
:105550006FE03FCA59C1D1C197E7FF1F83C7C79406
:10556000ADCF011122CC4AC84EC656C25AC006CE93
:1055700026CA52C42E89AA890144930A0004371B03
:10558000030063772403B3078940C207C183BE8445
:1055900063F4FA0093040004C204C180130A1BD40C
:1055A00097E7FF1F83C7478E8DE37D1A631C0A00B0
:1055B000F2406244D2444249B249224A924A024BE2
:1055C00005618280EFE0FFC2E1BF33858900269448
:1055D000A6854204D13D41806DB7828001119307B9
:1055E000700F2316F10006CE97E7FF1F83C7178EB3
:1055F0008DE7B7E7040083A7870D17E6FF1F034673
:10560000A6836C0017E5FF1F0355858C8297333501
:10561000A00097E7FF1FA38BA78AF2400561828055
:1056200041119397050122C406C626C2C1872E8464
:1056300063D40702B7E40400FC5417D5FF1F0345E9
:10564000A57F829719C1BC5482972165218DB240F4
:10565000224492444101828093F715008DC7B7E739
:10566000040083A7471A17D6FF1F1306E67097F5A5
:10567000FF1F9385256E17D5FF1F0345E57B829796
:1056800013451400E9B793F7250099CFB7E7040055
:10569000BC4F13060064894517D5FF1F0345C57924
:1056A00082971345240065B793F785009DC7B7E738
:1056B000040003A8871A1307401F97D7FF1F83C74B
:1056C000A777814613064006994517E5FF1F035546
:1056D00025800298134584009DBF93F7450001453E
:1056E000BDD7B7E4040083A7041817D5FF1F0355DF
:1056F000257E8297BC4C13060064914517D5FF1F89
:105700000345857382971345440091B797D7FF1FD0
:1057100083D7077C6396A70217D7FF1F231BB77A8F
:1057200017D7FF1F2318C77A17D7FF1F2315D77A5C
:105730002E8617350000130525A2BE856F00D035D3
:10574000173500001305C5A26F00D0490357450067
:10575000011106CE22CC97D7FF1F83D76777173565
:1057600000001305E5A06310F706C167F91717D706
:10577000FF1F232FF77437E4040097D7FF1F23ABD5
:1057800007747C4C894517D5FF1F0345E56A82974E
:105790007C4C914517D5FF1F0345056A829797D723
:1057A000FF1F83C7C76D95C78547A307F1008327F0
:1057B00044171306F10085451305503082971735BD
:1057C000000013056590EF00F041F240624405616E
:1057D000828097D7FF1F83C7976A1735000013058C
:1057E0006593F5F38547A307F10083274417130654
:1057F000F1008545130550308297173500001305D9
:10580000E58ED1B77D15954763EEA71817370000D1
:10581000130747880A053A951C41011122CC06CE90
:1058200026CABA972E848287173500001305C594BF
:10583000EF00503B05A203C725009947631CF70002
:105840002E85293783456400173500001305C5935D
:10585000EF00902497D7FF1FA3820762173500003F
:1058600013054594F1B703C7250095476317F70261
:10587000C16717D7FF1F0357A765F91703D5A50001
:105880006307F702B7E7040083A7C71782971735A6
:10589000000013052592EF00F034854717D7FF1F4E
:1058A000A30EF75C173500001305459351B797D742
:1058B000FF1F239FA76083D7E500B7E404000966B4
:1058C00017D7FF1F2317F76083D70501130606902C
:1058D00017D5FF1F0345455617D7FF1F231CF75E3B
:1058E00083D72501A14517D7FF1F2316F75EBC4CB0
:1058F0008297BC4C13060064914517D5FF1F0345E2
:10590000A55382970356E4008355A4001735000081
:105910001305858BEF00501849B7173500001305A4
:10592000A58C39B783C525009147639AF502854751
:10593000173500001305C58CA307F100EF00902A6E
:10594000B7E7040083A747171306F1008545130541
:1059500050308297F2406244D24405618280994778
:10596000639DF5002285DD33834564001735000013
:1059700013058581EF005012F1BF9547639FF50035
:10598000834714001735000013058587E39207EA63
:10599000173500001305858861BD17350000130514
:1059A0006588C9BF82806D71232481102326111060
:1059B00023229110328401CD89476306F5028320AA
:1059C000C110032481108324411051618280173556
:1059D00000001305E585AE84EF00D020A285268562
:1059E000EFD01FBEE9BFB7E70400FC47280082974D
:1059F0001735000013058584EF00D01E8347810012
:105A000039C01307000B638EE7001387A7051377D0
:105A1000F70F8D4663E9E602A2852800EFD0BFC0EC
:105A200079BF8547E3FD87F883459100173500006E
:105A300013058581B335B00097D7FF1F2380B74486
:105A4000EF009005ADBF03479100A207D98F3567DE
:105A50001307D755638DE7066366F7022D671307B3
:105A6000B7556381E70631671307C7556386E704B7
:105A700029671307A7556392E702A2852800EFD094
:105A8000FFE535BF39679306E7656383D70663E9AA
:105A9000F6001307E7556388E704A285280089B755
:105AA0003D679306F755638AD7041307F766E396B5
:105AB000E7FEEFD03FFC21B70146A2852800EFD0DA
:105AC000DFDAF5BDA2852800EFD0DFDFCDBD894745
:105AD000E3F787EE9305E4FFC205C1811305A1003A
:105AE000EFC0DFF9E9BDA2852800EFD0FFDFC1BD1F
:105AF000A2852800EFD0DFE9D9B5EFD0FFF1C1B51D
:105B0000411122C417D4FF1F1304C428AA861726E4
:105B100000001306A6592285C14506C6EF00700D88
:105B20000357440097D7FF1F9387C7272393E700A6
:105B3000035764002394E700B2402244410182806D
:105B4000130101DE232C812037E40400832704089D
:105B5000232E1120232A912023282121232631219D
:105B600017050000130505AC829717D9FF1F13090D
:105B7000A92C994785442300A9002318F1009725F3
:105B800000009385A55B93074006172500001305C9
:105B9000E5F92314F1102304910097D9FF1F93898D
:105BA000492EDD2D83D50900172500001305C550AA
:105BB000E5252945252703D50900856991378327E0
:105BC00044173000854513055030829783274417CA
:105BD00017D6FF1F1306061DCD451305703082979B
:105BE0008327441717D6FF1F1306C619B54513059B
:105BF00060308297832744171008894513051031B8
:105C000082978327441730028945130520318297F4
:105C100083274415938509C80D458297832744152A
:105C2000938509C811458297A30191002302910031
:105C300023049100232401102308010083278416E4
:105C4000300291451305704082978327841613060E
:105C50003100854513050040829783278416500044
:105C600085451305104082978327841610088545C3
:105C7000130520408297832784163000854513053D
:105C800050408297832704157D55829783274413BC
:105C90007D5582977D55EFD06FA68327440C829760
:105CA000EFD0AF838327841417D6FF1F1306860E09
:105CB000D5450145829789471306700F814508082D
:105CC0002302F100EFB0BFF58D471306700F814539
:105CD00028022308F100EFB09FF491472304F1104C
:105CE00097D7FF1F93870716984383C747003AC487
:105CF0002306F100EFD05FDE500085450545EFD06B
:105D00000FA710089305700F0945EFD04FA630027A
:105D10009305700F0D45EFD08FA5300095451145C7
:105D2000EFD0EFA4C16717D7FF1F1307671AF91742
:105D30001CC32322070017D5FF1F1305A50FEFD0A3
:105D4000EFA18327C41D17D5FF1F1305A517829741
:105D50003C4803450900854582978320C1210324DF
:105D6000812183244121032901218329C120130199
:105D7000012282800111C16726CA06CEAA8422CCE4
:105D800017D5FF1F0355C514F9176305F50437E44C
:105D90000400832784122E862315B1000147814613
:105DA000ED4582977C440356A1002AC6A6858297BA
:105DB0002C0017D5FF1F0355A511EFD0EFA619C969
:105DC0001725000013058538312D8327C412ED45B2
:105DD00028008297F2406244D2440561828001111A
:105DE0008547A307010017D7FF1F2301F70EB7E769
:105DF000040083A7471706CE1306F1008545130557
:105E000050308297F24005618280014863C6050EDA
:105E100063DB06003306C040B337C000B306D04092
:105E20001348F8FF9D8EB6873283AA8EAE886391A1
:105E3000061863FCC50C41676361E61EB7070001E5
:105E40006365F63693568601E1471727000013076E
:105E50002741369703470700BA97130700021D8FA3
:105E600019CBB395E500B357F5003313E600B3E85B
:105E7000B700B31EE50013560301B3D7C80293164B
:105E80000301C18213D70E01B3F5C8023385F602B0
:105E9000C205B3E8E50063FAA8009A981387F7FFF4
:105EA00063E4680063E9A832BA87B388A840B3D531
:105EB000C802C20E93DE0E01B3F8C802B386B60262
:105EC000C208B3E8D80163FBD8009A981387F5FF9E
:105ED00063E56800F91563E3D800BA8513950701F7
:105EE0004D8D8145630908003305A040B337A000FC
:105EF000B305B0409D8D82803305A040B337A0002C
:105F0000B305B0409D8D7D5821B701E6054333535D
:105F1000D3024167636AE30EB7070001636BF3289E
:105F200093568301E147172700001307673336971D
:105F300003470700BA97130700021D8F65EB9318FC
:105F40000301B3866540135F030193D808018545BB
:105F500013D70E01B3D7E603B3F6E6033386170370
:105F6000C206558F637AC7001A979386F7FF63645A
:105F700067006365C726B687118FB356E703C20E65
:105F800093DE0E013377E703B388160342073367C6
:105F9000D701637B17011A971386F6FF63656700C5
:105FA000F91663631701B28613950701558D1DBF5E
:105FB00063E1D504C16763E1F604B707000163E25A
:105FC000F61E93D8860161479727000093874729DB
:105FD000C69703C30700930700023A93B38767404D
:105FE000E9EB63ECB61C3335C5001345150081455C
:105FF000D5BD81450145FDB59307F00F63F2D71C70
:1060000093D886002147C9B71307F00F9A86E37C1F
:1060100067F093568300A14739B71307F00FB28694
:10602000E375C7E293568600A14705B53313E30035
:1060300033D6F500135F0301335EE603B396E50044
:10604000B357F500DD8E9318030193D80801B31EF2
:10605000E50093D50601B377E6033387C803C2078B
:10606000CD8F63FBE7009A971306FEFF63E3671685
:1060700063F1E716791E9A97998F33D6E703139742
:1060800006014183B3F7E7033385C80293960701FE
:10609000D98E63FBA6009A969307F6FF63E7661214
:1060A00063F5A61279169A9693150E01898ED18DF5
:1060B00045B533576600B396F600D98EB3D8650060
:1060C00013DF0601B3DEE803139E060133536500B8
:1060D000135E0E01B395F500B365B30013D7050148
:1060E0003316F600B3F8E8033303DE03C20833E7E0
:1060F000E800637B670036979388FEFF6369D70CDF
:106100006377670CF91E3697330767403353E7030D
:10611000C205C1813377E703B3086E024207D98D08
:1061200063FB1501B6951307F3FF63EED50863FC17
:1061300015097913B695C20E416FB3EE6E001307C1
:10614000FFFFB3F6EE0013D30E01718F4182338E41
:10615000E602B3851541B386C60293580E01330794
:10616000E302BA96C6963306C30263F3E6007A9654
:1061700013D306011A9663E2C5026385C5007685CE
:1061800081458DB341677D17F98EC206337EEE00DF
:10619000B317F500F296E3F4D7FE1385FEFF8145B1
:1061A00091B393D80601414705B593560601C147FF
:1061B00069B993560301C147BDB3814505451DB378
:1061C000B688014711B53A83BDB73E86F1BDC68E8C
:1061D00025BF328E55B5F9179A98C1B9F9171A9794
:1061E00061BBB3C7A5008D8B3307C50081E78D4721
:1061F00063EEC700AA876370E50A83C605008507BA
:106200008505A38FD7FEE3EAE7FE8280937635000B
:10621000AA8791CA83C6050085078505A38FD7FE87
:1062200093F63700FDB79376C7FF138606FE63F03B
:10623000C70683A3050083A2450083AF850003AF93
:10624000C50083AE050103AE450103A3850183A804
:10625000C5019385450223A0770003A8C5FF23A2AB
:10626000570023A4F70123A6E70123A8D70123AAF7
:10627000C70123AC670023AE17019387470223AE03
:1062800007FF75B790419107910523AEC7FEE3EB79
:10629000D7FEE3E4E7F6828039713EDA2ED232D4BB
:1062A00036D63AD842DC46DE97D7FF1F938707B928
:1062B00022CC804326CA06CEAA8409C41C4C99E38A
:1062C0002285C5230C4454102686228536C6EF004D
:1062D000F05AF2406244D24421618280011197D782
:1062E000FF1F9387A7B522CC804306CEAA8519C489
:1062F0001C4C89E72AC622856D23B24510442285AD
:106300006244F24005616F10603C011126CA4AC820
:1063100006CE22CC4EC652C4AA842E8901C51C4D7D
:1063200091E341239C4C804499E326859D2B97273C
:1063300000009387E704631CF402C0408357C40045
:10634000A18BB1C71C48A1C7FD59294A1C448345EC
:106350000900FD17B1E91CC463DE07062286A945C2
:106360002685192AFD576308F502294535A0972788
:1063700000009387E7026314F4008044C1B79727B5
:1063800000009387E7FDE31BF4FAC04445BFA285F4
:1063900026855D2255D97D55F2406244D24442495A
:1063A000B249224A056182801CC4050963D70700EF
:1063B000184C63CBE700638945011C401387170025
:1063C00018C02380B70059B7228626857520E31FA1
:1063D00035F7D1B71C401387170018C02947238011
:1063E000E70061B797D7FF1F938747A5AA85884322
:1063F00029BF35713ECBA6DA36C73AC942CD46CF62
:1064000097D7FF1F938787A386DEA2DC844363DBD5
:1064100005009307B0089CC07D55F6506654D654CD
:106420000D61828093078020231AF1002AC42ACCB0
:10643000814799C19387F5FF3EC83ECE7401FD5751
:106440002E8426852C00231BF10036C2EF00901409
:10645000FD576355F5009307B0089CC05DDCA2476B
:10646000238007005DBFAA87850703C7F7FF6DFF7D
:106470003385A7407D158280011122CC26CA4AC8E7
:1064800006CE4EC6AA842E89328401C51C4D91E3E6
:106490000929972700009387A7EE6319F406C040E7
:1064A0001C4C1CC48357C400A18BC9C31C48BDCF5E
:1064B0001C4808409379F90F1379F90F1D8D5C483A
:1064C0006346F500A2852685752C2DE51C4405053F
:1064D000FD171CC41C401387170018C02380370108
:1064E0005C486389A7008357C400858B81CBA9478B
:1064F0006316F900A285268571240DEDF2406244F1
:106500004A85D2444249B2490561828097270000FA
:10651000938707E96314F400804459B79727000074
:10652000938707E4E31EF4F6C0449DBFA285268549
:1065300021203DDD7D59D9B7411197D7FF1F9387A2
:10654000E78F26C2844322C44AC006C62A892E8405
:1065500089C49C4C99E32685A92697270000938738
:1065600027E2631CF402C0400317C400931707011D
:10657000C18393F68700B5EE93F607019DEEA5471C
:106580002320F900136707042316E4007D55B24069
:106590002244924402494101828097270000938758
:1065A00027E06314F4008044C1B797270000938765
:1065B00027DBE31BF4FAC04445BF918B8DC74C58D1
:1065C00089C9930744046384F5004A859123232AEB
:1065D00004028357C4002322040093F7B7FD231657
:1065E000F4001C481CC08357C40093E7870023169F
:1065F000F4001C4881EF8357C4001307002093F771
:1066000007286385E700A2854A85A5218357C40032
:1066100013F7170005C75C4823240400B307F040B4
:106620001CCC1C480145A5F78317C40013F70708C5
:1066300039DF93E707042316F40089BF898B0147EC
:1066400091E3584818C4F1BF83D7C500011122CC8B
:1066500026CA06CE4AC84EC613F78700AA842E84DF
:1066600071EFD841634DE000B841634AE000014555
:10667000F2406244D2444249B24905618280585492
:106680007DD703A904009396370123A0040063DD9E
:10669000060670488357C400918B99C75C401D8ED5
:1066A0005C5899C33C401D8E5C540C508146268535
:1066B0008297FD570357C400631DF5009440F547CA
:1066C00063E8D706B70740208507B3D7D700858B87
:1066D000A5C31C48232204001CC09317370163D8AC
:1066E0000700FD576314F5009C4091E368C84C58BF
:1066F00023A02401ADDD930744046384F5002685BF
:106700000129232A0402A5B70C5001468546268597
:106710000297FD572A86E31FF5F69C40A5DF7547D3
:106720006385E70059476394E70423A0240181B7F8
:10673000136707042316E4007D551DBF83A90501D7
:10674000E38709F203A905008D8B23A035013309E6
:106750003941014791E3D84918C4E35A20F11C5448
:106760000C50CA864E86268582976349A0008357BF
:10677000C40093E707042316F4007DBFAA993309E8
:10678000A940E1BF9C49B9CF011122CC06CE2A8491
:1067900011C51C4D81E72EC62922B245972700005E
:1067A000938707BE639BF5004C408397C50095C750
:1067B00022856244F240056141BD9727000093871E
:1067C00027BE6394F5000C44CDB79727000093874C
:1067D00027B9E39CF5FC4C44C9BFF2406244014533
:1067E0000561828001458280411122C406C62A8447
:1067F0002316B5002317C50023200500232205001A
:10680000232405002322050623280500232A05004A
:10681000232C0500214681451305C505EFB02FC087
:1068200097170000938747F65CD09717000093876F
:10683000A7F81CD4971700009387E7FC5CD4971740
:1068400000009387A7FF00D01CD8B240224441012A
:10685000828097050000938525F389AA411126C2FD
:10686000130680069384F5FFB384C4024AC02E89C0
:1068700022C406C693854407A1262A8401CD23207D
:10688000050023222501310508C4138684068145AD
:10689000EFB0EFB82285B240224492440249410150
:1068A00082801C4DBDE3411106C622C4970700003B
:1068B000938767FA1CD5972700009387A7BA9C4354
:1068C0002324050423260504232805046314F50066
:1068D00085471CCD2A841D2848C02285052808C468
:1068E00022852D2048C4484001469145F53D084485
:1068F0000546A545D53D48440946C945F535854772
:106900001CCCB240224441018280828041119727F1
:106910000000938727B526C284434AC006C69C4C14
:1069200022C42A8999E32685AD3F93848404804458
:10693000DC40FD1763D607009C40B9CF8440C5BF3B
:106940000317C40039E7C1778507232204062320F3
:10695000040023220400232404005CC42328040030
:10696000232A0400232C0400214681451305C40575
:10697000EFB0EFAA232A0402232C040223240404E8
:10698000232604042285B240224492440249410154
:1069900082801304840671BF91454A85C13588C041
:1069A00051FDB1472320F9000144E9BF797122D498
:1069B0004AD052CC56CA5AC85EC606D626D24ECE49
:1069C0002A8AAE8A130485040149054BFD5B09EC54
:1069D000B25022544A8592540259F249624AD24A2C
:1069E000424BB24B45618280044483294400FD1927
:1069F00063D409000040E1BF83D7C400637BFB0080
:106A00008397E40063877701A6855285829A33696C
:106A1000A90093848406E1BF1971A6DAAE84839538
:106A2000E500A2DC86DE328463DC050083D7C40087
:106A300023A0060093F7070885E7930700401DA0F1
:106A4000300836C6EF001066B246E34105FE7247D5
:106A5000BD67F98F7977BA9793B717009CC2F1BFDA
:106A6000930700041CC0F6506654D65401450961D2
:106A7000828083D7C500011122CC06CE26CA4AC81F
:106A8000898B2E8489CF930774041CC01CC885474A
:106A90005CC8F2406244D24442490561828074007D
:106AA0003000AA84953FA2452A892685112A01ED46
:106AB0008317C40013F7072069FFF19B93E72700B2
:106AC0002316F400C9B7970700009387C7D89CD452
:106AD0008357C40008C008C893E707082316F400CA
:106AE000A2475CC8B24791CF8315E4002685EF002A
:106AF000905E01C98357C400F19B93E717002316EA
:106B0000F4008357C4003369F9002316240151B7F8
:106B1000DDC583A7C5FF411122C406C626C2138462
:106B2000C5FF63D307003E94AA84EF00506797C760
:106B3000FF1F9387673A9C4391EF2322040097C776
:106B4000FF1F23AB87382244B2402685924441017F
:106B50006F001065637EF40014403307D400639621
:106B6000E7009843DC43369718C05CC0C9BFBA87BA
:106B7000D84319C3E37DE4FE94433386D700631FF3
:106B800086001040B29694C33386D700E31DC7FA3F
:106B900010435843B29694C3D8C375B76375C40005
:106BA000B1479CC04DB71040B306C4006316D70070
:106BB00014435843B29614C058C0C0C369B782800A
:106BC000011126CA93843500F19806CE22CC4AC81A
:106BD0004EC6A104B14763FBF404B14463EAB404B4
:106BE0002A89EF00D05B97C7FF1F9387E72E984352
:106BF0003A8429E897C7FF1F9387472E9C4389EB68
:106C000081454A85EF00F03497C7FF1F23A8A72CC2
:106C1000A6854A85EF00F033FD59631B3507B14760
:106C20002320F9004A85EF00B05729A0E3D804FAE1
:106C3000B1471CC10145F2406244D2444249B249C5
:106C4000056182801C40858F63C10704AD4663F6F1
:106C5000F6001CC03E9404C001A85C406315870286
:106C600017C7FF1F232AF7264A85EF007053130525
:106C7000B4009307440061993307F5404DDF3A941F
:106C8000898F1CC04DBF5CC3C5B72287404095B7F4
:106C9000130435007198E30085FCB305A4404A85D0
:106CA000EF00302BE31935FB9DBF01114AC803A942
:106CB000850022CC52C45AC006CE26CA4EC656C241
:106CC0002E84328B368A63ED260983D7C50013F7ED
:106CD000074849C704408C495848AA8AB389B44038
:106CE0008D44B384E4020947B3C4E4021387160059
:106CF0004E9763F3E400BA8493F70740D1C3A685A7
:106D000056857D3D2A890DE5B14723A0FA008357BA
:106D1000C4007D5593E707042316F400F240624453
:106D2000D2444249B249224A924A024B05618280CA
:106D30000C484E86EFF0EFCA8357C40093F7F7B7BD
:106D400093E707082316F4002328240144C84E992A
:106D5000B38434412320240104C4528963732A017B
:106D6000528908404A86DA85EF00D03E1C4401452E
:106D7000B38727411CC41C403E992320240179BFBE
:106D800026865685EF00F0412A895DFD0C48568520
:106D900041339DBF83D7C500717126D34AD14ECFF1
:106DA00006D722D552CD56CB5AC95EC762C566C337
:106DB00093F70708AA892E89B284B1C39C49A1E33D
:106DC0009305000436C6ED3B2320A9002328A90023
:106DD000B24615E1B14723A0F9007D55BA502A54B7
:106DE0009A540A59FA496A4ADA4A4A4BBA4B2A4C27
:106DF0009A4C4D61828093070004232AF90093077F
:106E00000002A30CF1029307000302DA230DF10242
:106E100036CE930B5002971A0000938A6A5A054C9B
:106E2000294B26848347040099C3639C7709B30CDC
:106E30009440638D0C00E6862686CA854E85B5355E
:106E4000FD576304F51AD256E69636DA83470400F6
:106E5000638D0718FD579304140002D002D63ED26A
:106E600002D4A301010682DC83C5040015465685C1
:106E7000EF00B02C13841400825731E513F707019B
:106E800009C713070002A301E10613F7870009C72A
:106E90001307B002A301E10683C604001307A00292
:106EA000638BE602B25726848146254603470400D9
:106EB00093051400130707FD6374E6068DC63ED6DE
:106EC0001DA0050485B7330555413315AC00C98FA6
:106ED0003ED0A28451BF724793064700184336CE76
:106EE000634907023AD6034704009307E002631F91
:106EF000F704034714009307A002631BF702F2474D
:106F00000904138747009C433ACE63C107023ED26F
:106F100035A83307E04093E727003AD63ED0E1B7E3
:106F2000B387670385462E84BA9749B7FD57C5B71F
:106F3000050402D281468147254603470400930594
:106F40001400130707FD6378E606F1F28345040099
:106F50000D461715000013052547EF00101E11CD33
:106F600097170000938747461D8D93070004B3973A
:106F7000A700025505045D8D2AD0834504001946FB
:106F8000171500001305854493041400230CB10267
:106F9000EF00B01A25C59797FFFF9387A70695E7DF
:106FA0000257F2471377071009CF91073ECED25709
:106FB000D2973EDABDB5B387670385462E84BA976C
:106FC000ADBF9D07E19BA107D5B7780897060000E4
:106FD0009386E6CD4A860C104E8597000000E700A8
:106FE0000000FD572A8AE314F5FC8357C9007D553C
:106FF00093F70704E39407DE5255CDB3780897065C
:1070000000009386C6CA4A860C104E852129D1BF3E
:107010001C46FD171CC663DA0700184E63C5E7005F
:10702000A9476394F5006FF02FC51C422E85138786
:10703000170018C22380B7008280011122CC26CA13
:107040004AC84EC652C406CE2A89AE893284B304D9
:10705000D6007D5A63149400014509A883450400B5
:107060004E864A8575370504E31645FFF2406244B3
:10707000D2444249B249224A05618280357122CD0B
:1070800026CB4AC94EC706CF52C556C35AC1DEDE0B
:10709000E2DCE6DAAA89AE843289368409C51C4D61
:1070A00099E3EFF01F80971700009387672D639C8B
:1070B000F40C83A4490083D7C400A18BFDC79C486E
:1070C000EDC793070002A304F1029307000302D265
:1070D0002305F10222C6930B5002971A0000938AEF
:1070E0002A2E054C294B4A848347040099C3639197
:1070F000770FB30C2441638D0C00E6864A86A68583
:107100004E85253FFD576307F51E9256E69636D20B
:10711000834704006380071EFD571309140002C84B
:1071200002CE3ECA02CCA309010482D483450900E1
:1071300015465685EF00700013041900C24759E93F
:1071400013F7070109C713070002A309E10413F7A6
:10715000870009C71307B002A309E10483460900A9
:107160001307A0026380E608F2474A848146254659
:107170000347040093051400130707FD6379E60A2B
:10718000B5CA3ECE85A897170000938767216395FF
:10719000F40083A4890005B7971700009387471C64
:1071A000E39BF4F083A4C90039B7A6854E85EFF0C0
:1071B000AFB801D97D55FA406A44DA444A49BA4920
:1071C0002A4A9A4A0A4BF65B665CD65C0D6182805D
:1071D000050419BF330555413315AC00C98F3EC8AE
:1071E0002289A9B7324793064700184336C6634938
:1071F00007023ACE034704009307E002631FF70437
:10720000034714009307A002631BF702B247090467
:10721000138747009C433AC663C107023ECA35A89C
:107220003307E04093E727003ACE3EC8E1B7B38783
:10723000670385462E84BA9725BFFD57C5B7050459
:1072400002CA81468147254603470400930514007E
:10725000130707FD6376E606F1F2834504000D4649
:107260001715000013054516C92D11CD97170000FD
:10727000938787151D8D93070004B397A700424598
:1072800005045D8D2AC883450400194617150000C2
:107290001305C513130914002304B102792D3DC150
:1072A0009797FFFF938707D695E74247B247137733
:1072B000071009CF91073EC69257D2973ED225B507
:1072C000B387670385462E84BA97BDBF9D07E19BB0
:1072D000A107D5B7780097060000938646D6268684
:1072E0000C084E8597000000E7000000FD572A8A31
:1072F000E314F5FC83D7C40093F70704E39C07EA83
:10730000125555BD780097060000938646D3268611
:107310000C084E85012AD9BF797156CA9C49BA8A90
:10732000984522D426D24ECE52CC06D64AD05AC840
:107330005EC6AA892E84B284368A63D3E700BA87F0
:107340009CC00347340419C385079CC01C4093F7B5
:10735000070281C79C4089079CC003290400137958
:107360006900631A0900130B9401FD5B5C449840AB
:10737000998F634CF9041C408346340493F7070249
:10738000B336D000A5EB13063404D2854E85829A1D
:10739000FD576303F5041C4011469840998B5444F3
:1073A00081446397C700B384E64063D304008144FB
:1073B0001C4418486354F700998FBE94014969042E
:1073C0007D5B63982405014509A885465A86D285C8
:1073D0004E85829A631E75017D55B2502254925497
:1073E0000259F249624AD24A424BB24B456182800D
:1073F0000509ADBF3307D40013060003A301C7047A
:107400000347540493871600A2978906A381E704D3
:107410009DBF85462286D2854E85829AE30E65FB06
:10742000050945B7797122D426D24AD04ECE06D668
:1074300052CC56CA5AC8B68983C6850193079006AE
:107440003289AA842E8413863504638DF60263E2A2
:10745000D706930780056387F61863EDD70063802E
:10746000062293073004638EF60A930A240423014C
:10747000D404C9A0930730066385F60A9307400633
:10748000E395F6FE1C40084393F607089305450074
:10749000C5C61C410CC363D807001307D002B3074D
:1074A000F040A301E404971600009386A6F2294752
:1074B0006DA8930700076383F61663E5D702930769
:1074C000E006638AF6189307F006E390F6FA0C409C
:1074D0001C4313F80508138547006307080608C313
:1074E0009C438DA893075007E383F6FE930780071C
:1074F000638AF61293073007E399F6F61C43D041EE
:1075000081459386470014C383AA07005685352119
:1075100001C53305554148C05C401CC8A3010404A3
:1075200071A81C43930A2404938647009C4314C308
:107530002301F4048547D5B793F607041C410CC317
:10754000B9DAC207C18781BF93F5050408C3C9D959
:1075500083D707001307F0066387E60E971600002F
:10756000938646E72947A30104044C400CC463C535
:10757000050008406D9908C099E3B28A91CDB28A9E
:10758000B3F5E702FD1AB69583C505002380BA005E
:10759000B3D5E70263FFE70AA147631EF7001C406B
:1075A000858B91CB58401C4863C7E70093070003C5
:1075B000A38FFAFEFD1A3306564110C84E87CA86BD
:1075C0007000A2852685893B7D5A631E450B7D553B
:1075D000B250225492540259F249624AD24A424B62
:1075E00045618280A382D50497160000938686DECB
:1075F0000C40084313F805081C411105630D0802EF
:1076000008C313F7150001C793E505020CC04147F5
:10761000B9FB0C4093F5F5FD0CC0B1B79C4193E765
:1076200007029CC193078007A302F4049716000089
:10763000938686DB75BF13F8050408C3E30308FCD3
:10764000C207C1837DBF971600009386A6D8214745
:1076500019BFAE8735B794411C43CC4913F80608CF
:10766000138547006306080008C39C438CC301A828
:1076700008C393F606049C43F5DA2390B700232849
:107680000400B28A25BF14485686CA852685829989
:10769000E30F45F31C40898B8DE7B2474844E3591B
:1076A000F5F23E8535B785465686CA852685829988
:1076B000E30F65F1050A5C443247998FE345FAFE12
:1076C000E9BF014A930A94017D5BF5B7011122CC11
:1076D00006CE2A8409C91C4D99E732C62EC4EFF0A4
:1076E0004F9C3246A24597170000938767C96316DF
:1076F000F60250401C46FD171CC663D00704184E06
:1077000063C7E70093F7F50F29476398E7022285DF
:107710006244F24005616FE03FD6971700009387FF
:1077200027C86314F6001044F1B797170000938739
:1077300027C3E311F6FC504475BF1C4213F5F50F47
:107740001387170018C22380B700F2406244056116
:107750008280411122C42A842E8597D7FF1F23A13E
:10776000076006C6EFB0EFA3FD576319F50097D782
:10777000FF1F9387E75E9C4391C31CC0B240224425
:1077800041018280411122C42E848395E50006C602
:10779000AD24634905007C48AA977CC8B2402244C6
:1077A000410182808357C4007D777D17F98F2316AE
:1077B000F400EDB783D7C500011122CC26CA4AC810
:1077C0004EC606CE93F70710AA842E843289B68956
:1077D00091C78395E5008946014635228357C40049
:1077E0007D777D17F98F2316F4008315E40062443A
:1077F000F240CE864A86B24942492685D244056186
:107800003DA8411122C42E848395E50006C6E528D3
:10781000FD570357C400631BF500FD77FD17F98F73
:107820002316F400B2402244410182808567D98F3B
:107830002316F40068C8FDB78395E50025A841111B
:1078400022C42A842E85B285368697D7FF1F23A9A6
:10785000075006C6EFB06F92FD576319F50097D732
:10786000FF1F9387E74F9C4391C31CC0B240224443
:1078700041018280411122C42A842E8597D7FF1F9F
:1078800023A0074E06C6752AFD576319F50097D742
:10789000FF1F9387E74C9C4391C31CC0B240224416
:1078A00041018280411122C42A842E85B28597D756
:1078B000FF1F23A7074A06C6692AFD576319F5006B
:1078C00097D7FF1F9387C7499C4391C31CC0B24001
:1078D000224441018280411122C42A842E8597D7F7
:1078E000FF1F23AF074606C6AD2AFD576319F500F3
:1078F00097D7FF1F9387C7469C4391C31CC0B240D4
:10790000224441018280411122C42A842E85B285FD
:10791000368697D7FF1F23A5074406C6992AFD5729
:107920006319F50097D7FF1F938787439C4391C343
:107930001CC0B24022444101828093F5F50F2A9683
:107940006314C5000145828083470500E38DB7FEBF
:107950000505FDB763F3A504B386C500637FD502B3
:107960009345F6FF8147FD176393F50082803387C7
:10797000F600034807003387C7002A972300070152
:10798000DDB73387F500834607003307F500850729
:107990002300D700E317F6FE82808147E5BF82808F
:1079A000828081E5B2856FF0AFA1011122CC06CEB5
:1079B00026CA4AC84EC6328401EEEFF06F950149DF
:1079C000F24062444A85D2444249B249056182800C
:1079D000AE84AA89A9282689E37485FEA2854E85EE
:1079E000EFF00F9E2A8969DDA6852286EFE06FFF02
:1079F000A6854E85EFF0CF91E1B7411122C42A84CC
:107A00002E85B285368697D7FF1F23AB073406C66F
:107A10008D28FD576319F50097D7FF1F93874734CB
:107A20009C4391C31CC0B24022444101828083A781
:107A3000C5FF1385C7FF63D50700AA959C413E95F6
:107A400082809307800517D7FF1F232BF7307D55C2
:107A500082809307800517D7FF1F2323F7307D55BA
:107A600082809307800517D7FF1F232BF72E014530
:107A700082809307800517D7FF1F2323F72E7D559C
:107A800082809307800517D7FF1F232BF72C7D5586
:107A90008280000038ADFFFF60ADFFFF88ADFFFFC3
:107AA000A0ADFFFFBAADFFFFCAADFFFFF2ADFFFF14
:107AB0001AAEFFFF32AEFFFF4CAEFFFFFE0065784F
:107AC000706572696D656E74616C0000626C6564EE
:107AD00065732E636F6D00004D6F64656C204E758D
:107AE0006D6265720000000053657269616C204E22
:107AF000756D62657200000096B4FFFFBCB4FFFFB5
:107B0000D6B4FFFFF4B4FFFF12B5FFFF73696D70C9
:107B10006C6550726F66696C655F57726974654118
:107B200074747243420000004150505F4442472049
:107B300025733E200000000073696D706C65507203
:107B40006F66696C655F57726974654174747243DE
:107B500042206C656E3A20256400000043483539A8
:107B6000785F424C455F4C49425F56312E330000EE
:107B7000686561642066696C65206572726F722E3B
:107B80002E2E00004C494220696E69742065727285
:107B90006F7220636F64653A202578202E2E2E0A9E
:107BA000000000002A2000004170705F496E697477
:107BB0003A20424C452D6F6E6C7920286E6F204D17
:107BC00065736820737461636B290D006C6F63616A
:107BD0006C20696D61676520696E666F206C656EEB
:107BE00020657272000000004F54413A2073757393
:107BF00070656E64204335354320424C45206E6FDE
:107C0000746966790D0000006C6F63616C2075709B
:107C100064617465206C656E2065727200000000FE
:107C20006C6F63616C20766572696679206C656E35
:107C300020657272000000006C6F63616C20656EDD
:107C400064206C656E206572720000004941505FCF
:107C5000454E442028424C45206C6F63616C290DD1
:107C6000000000004170705F426C655F4C6F6361A3
:107C70006C5F4F74615F48616E646C65000000006A
:107C8000436F6E66696720476174657761790D009F
:107C90007461726765745F64657620253034580DB1
:107CA0000A00000044495341424C45440000000092
:107CB000454E41424C4544004465627567206D6FF6
:107CC00064652025730D0A004164766572746973DA
:107CD000696E6720656E61626C65640D000000006E
:107CE0005175657279204D65736820416464722016
:107CF0002D2050726F766973696F6E65643A2564E2
:107D00002C20416464723A3078253034580D0A00D2
:107D10005175657279204D657368204B6579202D0A
:107D20002050726F766973696F6E65643A25640DD1
:107D30000A0000004465627567206D6F6465206C01
:107D40006F616465642066726F6D20666C61736834
:107D50003A2025640A0000004465627567206D6F53
:107D60006465207573696E672064656661756C74FF
:107D70003A2025640A0000004D65736820475720AB
:107D8000647374206C6F616465643A2030782530C8
:107D900034580D0A000000004D65736820475720D5
:107DA0006473742064656661756C743A203078255C
:107DB0003034580D0A0000004465627567206D6F0D
:107DC000646520736176656420746F20666C6173EE
:107DD000683A2025640A00004D65736820475720E3
:107DE0006473742073617665643A2030782530348A
:107DF000580D0A00434D445F484541443A307825C8
:107E00003034580D0A00000053746F705F4164767F
:107E10007200000080CFFFFFACCDFFFF80CEFFFFE0
:107E200080CEFFFF80CEFFFF16CDFFFF72CAFFFF9F
:107E300080CEFFFF4ECDFFFF7CCDFFFF6ACFFFFF5F
:107E400043483334312073657420706172613A2580
:107E50006420256420256420627265616B3A2530B8
:107E600032780D0A000000006D6F64656D20736547
:107E7000743A253032780D0A000000000A0600022C
:107E8000FF00FF40010000000902430002010080E2
:107E90003009040000010202010005240010010461
:107EA00024020205240600010524010100070584BF
:107EB0000308000109040100020A0000000705018F
:107EC000024000000705810240000000120110017D
:107ED00002000040861A40800030010203010000C9
:107EE0000902270001010080300904000003FF019E
:107EF00002000705820220000007050202200000A0
:107F0000070581030800010012011001FF00024073
:107F1000861A2375003101020301000055534232D5
:107F20002E3020546F2053657269616C20506F723F
:107F300074000000574348313231323132545331EA
:107F400000000000555342322E3020546F205365FC
:107F50007269616C20506F7274000000574348349E
:107F60003534353435545332000000007573625F88
:107F70007265630025303278202000004348333496
:107F80003120736574206270733A25640D0A000015
:107F90007374722025640D0A000000005345545F7D
:107FA000414444524553533A25640D0A00000000F1
:107FB0004745545F434F4E46494755524154494FF8
:107FC0004E0D00005345545F434F4E4649475552AE
:107FD0004154494F4E0D0000434C4541525F4645C8
:107FE00041545552450D00004745545F494E544594
:107FF00052464143450D00004745545F5354415498
:1080000055530D005345545F4C494E455F434F4413
:10801000494E470D00000000253032782000000056
:1080200063746C202530327820253032780D0A00B8
:1080300043444320526571436F646525780D0A00FF
:108040004745545F4C494E455F434F44494E473A7C
:1080500025640D0A000000004745545F534552490E
:10806000414C5F53544154453A25640D0A000000C9
:108070004C494E455F434F44494E472025642025D7
:10808000642025642025642025640D0A000000007A
:1080900098D7FFFFA6D7FFFF94D8FFFFD6D7FFFFE3
:1080A0008AD8FFFF00D9FFFF574D315F2530345884
:1080B000000000006D795F6E65745F616464723A00
:1080C0002564000052657374617274206164766582
:1080D00072746973696E6720284445425547206D64
:1080E0006F6465290000000052657374617274202A
:1080F0006164766572746973696E6720286E6F7447
:108100002070726F766973696F6E65642900000074
:1081100053746F70206164766572746973696E67F9
:108120002028616C72656164792070726F76697362
:10813000696F6E65642900005065726970686572C8
:10814000616C5F496E6974004E6F74696679204591
:1081500052522000557064617465202578202D20CE
:10816000496E74202578200A000000004552522EE6
:108170002E000000496E697469616C697A65642E2D
:108180002E000000446973636F6E6E6563746564EE
:108190002E2E20526561736F6E3A25780A0000001A
:1081A0004164766572746973696E672E2E000000F3
:1081B000436F6E6E656374696F6E206D61782E2EED
:1081C0002E000000436F6E6E202578202D20496E12
:1081D00074202578200A0000436F6E6E6563746515
:1081E000642E2E00436F6E6E656374656420416477
:1081F000766572746973696E672E2E0057616974B3
:10820000696E6720666F7220616476657274697347
:10821000696E672E2E0000004572726F722E2E005E
:108220004572726F722E2E25780A000052657620F4
:108230004348415231000000526576204348415284
:10824000332E2E004F544120433535432073757330
:1082500070656E642025750D0A00000000010202A1
:1082600003030303040404040404040405050505CE
:1082700005050505050505050505050506060606AA
:10828000060606060606060606060606060606068E
:10829000060606060606060606060606070707077A
:1082A000070707070707070707070707070707075E
:1082B000070707070707070707070707070707074E
:1082C000070707070707070707070707070707073E
:1082D000070707070707070707070707080808082A
:1082E000080808080808080808080808080808080E
:1082F00008080808080808080808080808080808FE
:1083000008080808080808080808080808080808ED
:1083100008080808080808080808080808080808DD
:1083200008080808080808080808080808080808CD
:1083300008080808080808080808080808080808BD
:1083400008080808080808080808080808080808AD
:1083500008080808080808080808080800000000BD
:10836000000000000000000000000000000000000D
:1083700000000000000000000000000000000000FD
:1083800000000000000000000000000000000000ED
:1083900000000000000000000000000000000000DD
:1083A00000000000000000000000000000000000CD
:1083B000000000000000000000000000232D302B12
:1083C00020000000686C4C00656667454647000069
:1083D00030313233343536373839414243444546FB
:1083E00000000000303132333435363738396162BD
:1083F000636465660000000076312E3000000000E6
:10840000262A000076312E3000000000272A0000C6
:10841000292A00000A18000002000000148400004D
:1084200076312E3000000000282A0000E0FF000016
:10843000020000002C840000E1FF0000E2FF0000C9
:10844000E3FF0000E4FF0000E5FF0000040309046F
:108450007763682E636E00007763682E636E00009A
:10846000B42D0020020000000CE004000100000018
:10847000188400000200000012E004000100000067
:108480001E2E0020020000001084000001000000E9
:10849000CC7A00000200000012E00400010000009D
:1084A0001C2E0020020000000084000001000000DB
:1084B000F88300000200000012E004000100000048
:1084C0001D2E0020020000000C84000001000000AE
:1084D000048400000200000012E00400010000001B
:1084E000272E002002000000288400000100000068
:1084F000208400000C2B00000000000000000000A1
:10850000020000000CE004000100000030840000C4
:108510000200000012E0040001000000282E0020EC
:10852000020000003884000003000000DC2E002060
:108530000200000016E0040001000000102D0020E1
:108540000200000012E0040001000000292E0020BB
:10855000020000003C84000001000000502E0020BA
:108560000200000016E0040001000000242D00209D
:108570000200000012E00400010000002A2E00208A
:10858000020000004084000002000000D42F002000
:108590000200000016E0040001000000382D002059
:1085A0000200000012E00400010000002B2E002059
:1085B000020000004484000000000000CC300020D5
:1085C0000200000018E0040003000000542E002008
:1085D0000200000016E00400010000004C2D002005
:1085E0000200000012E00400010000002C2E002018
:1085F000020000004884000004000000582E002003
:108600000200000016E0040001000000602D0020C0
:10861000F82C0000E82D00000000000043686172A3
:1086200061637465726973746963203100000000CE
:10863000436861726163746572697374696320323F
:10864000000000004368617261637465726973744D
:1086500069632033000000004368617261637465E0
:1086600072697374696320340000000043686172AA
:10867000616374657269737469632035000000007A
:1086800004580000DC5500000C57000002010603EE
:1086900002E0FF05FFD7070000000000574D315FE3
:1086A0003030303000000000000000000909574D54
:1086B000315F30303030051206006400020A0000DD
:1086C000000000007C8300009C8300005C830000AD
:1086D000000000000000000000000000000000009A
:1086E000000000000000000000000000000000008A
:1086F000000000000000000000000000000000007A
:108700000000000000000000000000000000000069
:108710000000000000000000000000000000000059
:1087200000000000604D00200202020001D7070097
:10873000001001020A02081002FF1400A6590000EE
:10874000FF000000B42D002000000000010203041F
:048750000500000020
:020000040004F6
:10D000006F00C076000000000000000090000020CB
:10D010008C020020A9BDF9F590000020000000005E
:10D0200000000000900000209000002000000000A0
:10D030000000000090000020000000009000002090
:10D0400000000000900000209000002090000020D0
:10D050009000002090000020900000209000002010
:10D0600000000000900000209000002090000020B0
:10D0700090000020900000209000002090000020F0
:10D0800090000020900000209000002090000020E0
:10D090009000002001A0011113078008F3370780DA
:10D0A00093F787083EC201000100B71700409305BF
:10D0B00070052380B704130680FA2380C70401009B
:10D0C000010083C6B70493F6F60DA385D704238029
:10D0D00007049246F3A6068001000100937605023C
:10D0E000D5CEF336078093F6860836C401000100DA
:10D0F0002380B7042380C70401000100B706140091
:10D100007D89558D88C70100010001000100238041
:10D110000704A246F3A606800100010073370780CA
:10D12000137787083AC6010001002380B7042380E3
:10D13000C7040100010001000100372700409306E9
:10D140001005A303D78023800704B247F3A7078005
:10D150000100010093078008F3B7078093F7870861
:10D160003ECE01000100B717004013077005238071
:10D17000E704130780FA2380E7040100010003C7D6
:10D18000B70413670708A385E70423800704F24761
:10D19000F3A70780010001000561828093760504F2
:10D1A000BDC6F336078093F6860836C80100010035
:10D1B0002380B7042380C70401000100B7061400D0
:10D1C000938606047D89558D88C701000100010002
:10D1D000010023800704C246F3A606800100010077
:10D1E00073370780137787083ACA0100010023804C
:10D1F000B7042380C70401000100372700409306CD
:10D200002005A303D78023800704D24781B7733753
:10D210000780137787083ACC010001002380B70408
:10D220002380C7040100010098471367070C98C7C3
:10D2300023800704E24719BF011181460146814559
:10D24000114506CE7D2A93078008F3B7078093F730
:10D2500087083EC601000100B7170040130770059C
:10D260002380E704130780FA2380E704010001000C
:10D2700003C76704136717002383E70423800704A9
:10D28000B247F3A7078001000100F24005618280E8
:10D2900041118146014681451145A52213078008A9
:10D2A000F337078093F787083EC401000100B717E2
:10D2B0000040130670052380C704930680FA23807C
:10D2C000D70401000100FD552396B702238007040F
:10D2D000A245F3A50580010001007337078013778D
:10D2E00087083AC6010001002380C7042380D704C1
:10D2F0000100010003C76704136717002383E704D5
:10D3000023800704B247F3A707800100010001A0B2
:10D31000BD473305F50201007D1575FD8280411181
:10D3200022C426C206C6AA84014463179400B240F0
:10D33000224492444101828005041305803E420448
:10D34000C13F4180DDB72303048015472303E480F8
:10D3500001002302A480828083076480E3CE07FE5D
:10D3600023030480828083076480E3CE07FE0345A5
:10D370004480828083076480E3CE07FE2302A4807A
:10D380008280411126C44AC24EC006C61377F50BEF
:10D39000AD47AA892E8995446306F700194565377C
:10D3A000653F8D444E854537FD59FD146398340122
:10D3B000B240A244124982494101828013550901B9
:10D3C0001375F50F453F2209CDB7011126CC06CEC6
:10D3D000B704080051371545BD37713769372AC67C
:10D3E000A53F32459377150089EB1365150013753A
:10D3F000F50FF240E24405618280FD14E9FC01452D
:10D40000CDBF397126DC4ADA4ED852D656D45AD21C
:10D410005ED006DE62CE66CCB7E700E07D5783AA19
:10D42000070022C603AA470023A0E71823A2E71893
:10D43000B7170040130770052380E704130780FA2D
:10D440002380E70483C74704930B75FFB684E20784
:10D4500093FBFB0F8546AA892E8B32893724004027
:10D46000E187015763FA76016308D50089461307FF
:10D4700000026313D5000157D98F93F7F70FB71C3C
:10D4800000402382FC0411472303E4801305F00FBE
:10D490005D3D094CD135636D7C11B7050700DA9508
:10D4A00037870700795563F2E504B3879500636E0B
:10D4B000F702370B0800A94733EB65016399F906BA
:10D4C00089E48144513D26850DA0DA850945553D05
:10D4D00005090345F9FFFD14050B693D81C49377E8
:10D4E000FB0FFDF7DD3569FD7D55B71700401307CC
:10D4F00070052380E704130780FA2380E70403C73D
:10D500004704418B2382E704F250B7E700E023A0F1
:10D51000571123A24711E25432445259C259325A88
:10D52000A25A125B825B724CE24C21618280A54759
:10D530006395F90685691309F00FB3069900B37472
:10D540002B01B6941349F9FFB3749900856B3379B5
:10D550006901416B9387F9FFB3F7270199E363FCF6
:10D56000340193D94900C147E3E637FF99BF056904
:10D57000C1697D19D9B71305800D63886901130549
:10D5800000026384790113051008CA85DD3B353D2F
:10D5900021DD4E99B3843441D9B7DA852D45D53391
:10D5A000CA94E30099F205097D3BA30FA9FED5BFFC
:10D5B0009387F9FF93F7F70F6361FC0C83C71C0493
:10D5C00013073008631FF70437070800636BEB0489
:10D5D000B3079B00B706100063F5D704334BEB008D
:10D5E00089476393F9068980D549E38C04ECDA8591
:10D5F0000945413B11090327C9FF91472320E480D6
:10D6000003076480E34E07FE23033481FD17EDFB1F
:10D61000FD14110B81C49377FB0FE9FF7D3371F586
:10D62000E1B5B717004003C75704B70708001377E1
:10D63000070219E3B78707007955E378FBEA330758
:10D640009B00E3FFE7F855B58547E382F9F2DA85F9
:10D650002D45053B9389F4FFE38504E6293393F7D1
:10D66000390091EB832604800327090093074900C2
:10D67000E39AE6E43E89CE84F1BFB5476396F900AC
:10D680001305900BC93135BDB1471305B00AE38BC3
:10D69000F9FE99476391F904B7050800B365BB002B
:10D6A0002D45C53181448D4BA1497539639674016F
:10D6B000832704802320F9008504E39834FF83271F
:10D6C000048013172B01635507002312F900D5BB03
:10D6D0002322F900FDB39D476399F90281451305A3
:10D6E000B0044531BD442320090023220900FD591F
:10D6F0009D3993F77400CA9703C70700FD14398D4D
:10D700002380A700E39634FF6DBBA1476392F90421
:10D710006D398144630D0B008D479304C00363088A
:10D72000FB009304000563048B019304400413750C
:10D73000C507E30895D819453931393905452131EF
:10D7400026850D3909453D314931E31C05D669BBB4
:10D7500091476399F90013056006F536F53E130508
:10D7600090090DB7E38F09D4F154A9BB9731FB1F82
:10D770009381C17F1791FB1F1301C188170500001A
:10D78000130585889735FB1F9385C5871736FB1FC3
:10D790001306C6FD63FAC5008322050023A05500C9
:10D7A00011059105E3EAC5FE170500001305857311
:10D7B0009735FB1F938585FB1386818063FAC5002F
:10D7C0008322050023A0550011059105E3EAC5FE5B
:10D7D00013858180938581816377B50023200500BF
:10D7E0001105E36DB5FEFD42739002BC8D4273904E
:10D7F0004280B72200009382828873900230973271
:10D80000FB1F9382228093E2320073905230970282
:10D8100000009382622B73901234730020300D0647
:10D82000719A81473307F5006393C70082801443E0
:10D830003387F500910714C3F5B7914763EEB7023C
:10D8400017070000130787628A05BA959C41BA97AB
:10D850008287B717004003A7470B1345F5FF698F71
:10D8600023AAE70A03A7070B698F23A8E70A03A7E0
:10D87000070A798D23A0A70A8280B717004083A6E4
:10D88000470B1347F5FFF98E23AAD70A83A6070B88
:10D89000558D23A8A70A83A6070A758F23A0E70A38
:10D8A0008280B717004003A7470B498F23AAE70AD6
:10D8B00003A7070B1345F5FF45BFB717004083A625
:10D8C000470B1347F5FF758F23AAE70A03A7070A3B
:10D8D000598D4DB7B717004003A7470B498FEDB7D8
:10D8E000B71700408847420541819377050491EBC3
:10D8F0009377F5013755E801130505803345F502A7
:10D9000082809377050C130700046397E7009377F1
:10D91000F50137459C1CCDB72165130505D08280E4
:10D92000411122C406C62A84653F2947B307E50290
:10D93000B2408D83B3D7870222449507B3D7E7025D
:10D9400037370040C207C1832316F7404101828068
:10D95000716541111305052006C6D937B737004058
:10D96000130770F82381E7400D47A381E7401307B1
:10D970000004A380E74005472387E740B240410108
:10D980008280411122C491462A84138681809D653C
:10D990002D4506C69730FB1FE780A0A6B7F7070006
:10D9A00003C70701A5476313F70001A09306001002
:10D9B00001469D6525459730FB1FE78080A42384A1
:10D9C00081802244B2409146138681809D6529451D
:10D9D00041011733FB1F6700C3A2130101BF2326B8
:10D9E00011402324814023229140232021411737D5
:10D9F000FB1F0347A7D78D476310F706B7660200E2
:10DA00000146856505459730FB1FE780809F377489
:10DA1000020037A9FDFFB7D4040022851306004099
:10DA20008A85F53BB3052401930600400A86094523
:10DA3000130404409730FB1FE780A09CE31F94FC75
:10DA400005458137B76602000146B77502000545F6
:10DA50009730FB1FE780E09A856782978320C1405B
:10DA600003248140832441400329014013010141E3
:10DA700082800111914670009D652D4506CE97303C
:10DA8000FB1FE78000980347C10089469307F7FF13
:10DA900093F7F70F63E2F6029737FB1F2388E7CC73
:10DAA0009735FB1F83C585CC170500001305453D41
:10DAB0008528F2400561828085471737FB1F2307C1
:10DAC000F7CAF9BF41111305800406C69720FB1F52
:10DAD000E780605C371700408327870A1305002022
:10DAE0008D4593E707202324F70A813B953551376D
:10DAF000ED35B24001454101828081473737004012
:10DB0000A14663C3B70082800346B740E38EC6FEDA
:10DB10003306F5000346060085072304C740D5B742
:10DB20003571CAD813094108A6DAD2D4DAD02EC387
:10DB300086DEA2DCCED6D6D2DECEE2CCE6CAEAC8FB
:10DB4000AA8432C536C73AC93ECB42CD46CF4AC475
:10DB50008145014A170B0000130B4B3683870400E5
:10DB600085E789C5C205C1815285413FF65066549B
:10DB7000D6544659B659265A965A065BF64B664C09
:10DB8000D64C464D0D618280130750026389E70031
:10DB900063140A00268A814585058504C1B791C5AD
:10DBA000C2055285C181913F014A81471307B002E6
:10DBB0009305D002130500031308000293083002F6
:10DBC0008386140013861400638EE6026341D70235
:10DBD000638D0603638E1603138706FD1377F70F15
:10DBE000A54563EDE5060147254529481DA863873E
:10DBF000B600E393A6FE93E7170019A093E7070189
:10DC0000B2847DBF93E74700E5BF93E78700CDBFB0
:10DC100093E70702F5B73307070305062E971307A7
:10DC200007FD83050600938605FD93F6F60FE37462
:10DC3000D5FE830506009306E002639AD50C8305A2
:10DC40001600254593041600938605FD93F6F60FFE
:10DC5000636FD50881462545294805A89305A0028C
:10DC60007D57E398B6FC03270900138624001109A9
:10DC7000E35107FC3307E04093E707015DBFB3863C
:10DC800006038504AE96938606FD838504001386FD
:10DC900005FD1376F60FE374C5FE038604009305B5
:10DCA00080066308B6001376F6FD9305C00463137F
:10DCB000B60085040386040093058005630CB60452
:10DCC00093058007630AB604930750026307F600C2
:10DCD000854548002302F1000D3583870400A9CF54
:10DCE000854548002302F100093D81457DB51305B6
:10DCF000A0028146E393A5FA832609009304260037
:10DD00001306490063D306008146328979B7B2848D
:10DD1000FD5661B793E7070413F607045A8809E62E
:10DD2000170800001308081793FA070163880A0010
:10DD3000F99B9305000201A8FD1445BF13F61700D7
:10DD4000930500037DD6A302B1002303010093FBDA
:10DD500007020326090063830B00791741E61306C7
:10DD600000032306C1008549368C63D336014E8CEF
:10DD7000C58B330487418DE7A28C130D00026341EC
:10DD800090099307F4FF228763530400014733840B
:10DD9000E7408307610089C7854513056100B13BF2
:10DDA00063820B0293070003854513057100A303EB
:10DDB000F100A13393078007854513057100A30384
:10DDC000F100253B639D0A00A28A63435005930737
:10DDD000F4FF22876353040001473384E740930A2A
:10DDE0000003A1A06C0081491375F600429503451C
:10DDF0000500118285092380A500850575F6ADB75C
:10DE0000854513057100A303A101FD1CFD3185BFEC
:10DE1000854513055100D531FD1A45BF85451305CC
:10DE20007100A30351017D1CC939E3C989FFFD5A63
:10DE3000FD196398590193090002634F800011098D
:10DE40006DB57C00CE9783C707008545130571002B
:10DE5000A303F1005D31E9BF854513057100A303FC
:10DE600031017D145939D1BFEAF9FFFF12FAFFFFE2
:10DE70003AFAFFFF52FAFFFF6CFAFFFF496D616744
:10DE80006520466C616720253032780A000000006A
:10DE90003031323334353637383961626364656620
:10DEA0006768696A6B6C6D6E6F707172737475768A
:10DEB0007778797A000000003031323334353637E4
:10DEC00038394142434445464748494A4B4C4D4EF8
:10DED0004F505152535455565758595A000000004C
:08DEE000FF000000000000003B
:10E000006F00E2110000000000180118002801282C
:10E0100002280328002901290229032904290529A6
:10E02000062907290829002A012A022A032A042A84
:10E03000052AA62A78E8060056FD0400F002002012
:10E0400076030020C00200208E0200201C02002067
:10E050005EFF0400A6FF04004C010500D803050084
:10E06000C6040500B4FB040072FA040034FB04008B
:10E07000C4FA0400B60A05000C05002034FF0400B1
:10E0800082070500CC9F0600C4A106003CA2060042
:10E09000F66106002A62060056180600960D060074
:10E0A000A6990600B80705004669060004AA0500FF
:10E0B00092AA0500EAAA050046130500921305007E
:10E0C000FC1105002C660500E6600500C26F050026
:10E0D000927305003E7705001A530500B8520500FB
:10E0E000A0560500665305008E5205001253050028
:10E0F00040520500EA53050042540500F253050062
:10E10000F6530500905405004A5405007C54050060
:10E110009459050098590500E6530500EE53050093
:10E120008E540500965905003E550500065B050016
:10E130008685050004860500428605009068050076
:10E14000A8680500E4680500F24C0500104E0500C3
:10E15000864E05001C320500C22C05000843050050
:10E16000402D05006C3E0500C0C9060040C20600F7
:10E170001CC7060022DD060008DC060094DF06004E
:10E1800084DF06008CDF0600CCDF06005AB40600F0
:10E19000000000000000000000000000000000007F
:10E1A0003CE0060004DA06009AD9060000000000F0
:10E1B000000000000000000000000000000000005F
:10E1C00092830600B0710600367506000E730600D5
:10E1D000647D06004E9A0600000000008EB4060022
:10E1E000440C050066630600266906001E6A0600E8
:10E1F0000000000000000000000000008C6C050022
:10E20000C4820600000000000000000000000000C2
:10E21000607106001C0700203E640600B8DF06009F
:10E22000000000000000000088DF06006403050015
:10E23000E2690500C0DF0600688406003685060036
:10E24000B085060062C70600BCDF0600C4DF06001A
:10E25000220D0600C8DF060026110020EC10002069
:10E2600000000000000000000000000000000000AE
:10E27000000000000000000000000000000000009E
:10E280006373B60082801C419105110523AEF5FE33
:10E29000C5BFB72700203727002093878780130743
:10E2A00047D86373F700828023A007009107D5BF8A
:10E2B0004111B7E700E022C480433707200006C6BB
:10E2C000798C23A0E7180F10000011C199E5B7E77A
:10E2D00000E023A08710014545A893073500C20739
:10E2E000C183F19BC207C183130740036366F70232
:10E2F000372700200325079337270020832687929E
:10E300006391A602372700200327079C69D3C20721
:10E31000DD8D0545029765BF372700200325C7928D
:10E32000E1BF035765002DE7035745006362F70619
:10E33000B72600203306F7402148938686936378FA
:10E34000C8028328050003D86600138687001D8F46
:10E350002A9661172312E6002320160123130600D4
:10E3600010C12312F500130788FF2393E60023133F
:10E37000B50083D566002105B387F5402393F600E9
:10E38000B7E700E023A08710B24022444101828019
:10E390000841BDB7B7E700E003A807003707200032
:10E3A00023A0E7183378E8000F10000001E523A050
:10E3B00007118280B727002003AE0793B7270020FC
:10E3C00003A387928146F28763FC670A83A807004C
:10E3D000636BF50A63E9A80A138787006362E50A9D
:10E3E00003D66700216705076319E600372600207A
:10E3F0000347068905072308E6883726002013050A
:10E40000869383D5470003576500239307001306BF
:10E4100086932E97420741832313E5006387C70342
:10E42000372500200325C5926301F50203D5660058
:10E4300009ED83D7460023A016012107BE95A1054B
:10E440002392B6002313E600B6879843630A670257
:10E45000B726002083A6C6926304D70283566700BE
:10E4600085E283D64700835547001843A106AE9640
:10E470002392D70098C383576600A1072313F600A1
:10E48000B7E700E02DB7BE86C6873DBFB7E700E01F
:10E490009843B706200023A0D718758F0F100000EF
:10E4A00001C599C1814711E6B7E700E023A0E71055
:10E4B0008280B386F50003C80600B306F500850721
:10E4C00023800601E317F6FEC5B737E700E01C43DB
:10E4D000B70620002320D718F58F0F10000019C1B0
:10E4E00091C111E637E700E02320F7108280910503
:10E4F00003A7C5FF11057D16232EE5FEDDB737E71F
:10E5000000E01C43B70620002320D718F58F0F101A
:10E51000000001C53307C50011E637E700E02320FE
:10E52000F71082800505A30FB5FEE31DE5FEF5B7E4
:10E53000B7E700E09843B706200023A0D718758FEF
:10E540000F1000008147B306F5008386060099E6A8
:10E55000B7E600E023A0E6103E8582808507E5B798
:10E5600037E700E01C43B70620002320D718F58FBB
:10E570000F10000001C599C1014711EA37E700E01B
:10E580002320F710054582800507E309E6FE3308DE
:10E59000E500B386E5000348080083C60600E305EE
:10E5A000D8FE37E700E02320F7100145828037E7E7
:10E5B00000E01C43B70620002320D718F58F0F106A
:10E5C00000001307F6FFBA952A966317C50037E7D0
:10E5D00000E02320F7108280FD1503C71500050514
:10E5E000A30FE5FEDDB737E700E01C43B7062000C8
:10E5F0002320D718F58F0F10000001C53307C50081
:10E6000019E637E700E02320F71001458280050571
:10E610008346F5FFE397B6FEE31BE5FE37E700E030
:10E620002320F71005458280797126D2B724002077
:10E6300022D403A4C49806D64AD04ECE52CC56CA91
:10E640005AC85EC662C44DC8372A00203729002048
:10E65000B7290020814BB72A002037CBC901130A04
:10E660000A99130989939389C99D8357240099EFC7
:10E670005C44639A0B0023A6F498032CC400228503
:10E68000113B6284B9A823A6FB00C5BF83A74A98A3
:10E6900082971C443307F5406376F50003A74900D1
:10E6A0001D8F2A979306FB3763ECE60623280900A3
:10E6B0008355240003450400970005E0E78060B11E
:10E6C0005C405844B1C70C4403A64900AE97BE86CF
:10E6D00063E4B70063E4C700B386C74014C4A28BE9
:10E6E0003A8441F4B727002093878793984B894653
:10E6F00063FCE604791798CBB25022549254025925
:10E70000F249624AD24A424BB24B224C4561828066
:10E7100063950B0023A6E4988DB723A6EB00B1BF49
:10E7200003274A0219CB63EDA7003385A74083274F
:10E7300009016374F5002328A900A28B404455B752
:10E7400003A74900BA97D5B723A8070075B7B7271D
:10E75000002003A7479D411122C406C63E8411C371
:10E760000297B727002083C7279893F7F70F99E3FD
:10E77000232A049CB24022444101828001114EC6EA
:10E78000B729002083A7499606CE22CC26CA4AC8BC
:10E7900052C456C281C7829723A20996B72400208B
:10E7A000938744C883C7570037240020938444C804
:10E7B000858B1304449681CF83C774001947631671
:10E7C000F70EA3820400EF0030615C4482971C4482
:10E7D00091C3829737240020372900209307849320
:10E7E0000327899803C61700130A849383478493E9
:10E7F00093961700BA9683D60600F9C2834784938E
:10E8000063E8C70C83A74996230C0492639407120C
:10E81000B727002083A74798638E0710B7270020EB
:10E8200083A7079E2328FA00013583C7B4006393AA
:10E83000071083C7940081CF83C7740093F7F70F45
:10E8400099E7A3840400976006E0E780E007B72714
:10E85000002083A7479BF9CF83270A01E1CF83C715
:10E86000740015476368F70CB7270020938707CD1E
:10E8700083C7C700918BDDEFB727002083C7279898
:10E8800093F7F70FC5EB83461A000326899863CCEC
:10E89000D70A6244F240D2444249B249224A924ADB
:10E8A0000561170305E0670043F183C774001D4746
:10E8B000E31FF7F0A3820400EF0010521C4839B7A1
:10E8C000850793F7F70F230CF492E3E1C7F23DB706
:10E8D00086073E978355070023100700034584935E
:10E8E000B727002083A7079613172500B72A002013
:10E8F000BA979C4323900A98829783D70A98034734
:10E90000849393C7F7FF7D8D93171700032789988A
:10E910003E97835707005D8D2310A700834784939C
:10E9200081C78507230CF4920347849383471A0019
:10E93000E37AF7ECF2406244D2444249B249224AB7
:10E94000924A056182801397170032970357070098
:10E9500075F385072DBF37C700408326C720B7074B
:10E96000FCFFFD17F58F2326F72001000100B727D4
:10E97000002093878793C84F832787262326D72095
:10E980006A0593C7F7FF99835D8D8280B7270020C2
:10E9900003A3079F6303030002831305F00F828024
:10E9A0000327851163000712411122C406C683475D
:10E9B000C5008345E5042A8493F7C70F2306F500B5
:10E9C000834697000356C70013958601618563F15E
:10E9D000C508635A05060345870093F6F607A304A6
:10E9E000D700054693E627006314C50093E6170099
:10E9F0002306D4005C4389075CC3A30AB400032543
:10EA000004112E864C430905513483278411034693
:10EA10005401D44303D7C700B296118FD4C32396B1
:10EA2000E7008947A30DF400B727002003476403DC
:10EA300083C7279A6378F7048347C40093E70701E5
:10EA40002306F40081A093E717002306F40075B7AE
:10EA50009376F60F635D050203458700854513E64F
:10EA600027006314B50013E617002306C400A30AA9
:10EA7000D400A30407008547A30DF4008327841165
:10EA80009C43DDF3B240224401454101828093E77B
:10EA900017002306F400A30AD400A30407000325EB
:10EAA00004114C430905DD328327841103465401C8
:10EAB000D44303D7C700B296118FD4C32396E7007F
:10EAC0008D475DBF05458280B727002083A7C7C655
:10EAD000411122C406C6858B2A84DDEB41651305EE
:10EAE00025F5972006E0E78040E05DC18347A5005B
:10EAF0002315F50083270412B5E72320A41223224F
:10EB0000A41285472311F4042320050083476401E0
:10EB100054412316F5000347D4002304E5000547BC
:10EB2000A304E50037270020032787CA13851702AF
:10EB300015811C437D151375F50F9CC25C43DCC227
:10EB40001C479CC65C47DCC61C4B9CCA5C4BDCCAA1
:10EB50001C4F9CCE5C4FDCCE19CD9386060213076A
:10EB60000702C1BF8327441288C38357240423228A
:10EB7000A412850741BFB7270020938787B403D726
:10EB8000870005072394E700B240224441018280B8
:10EB90008347C40023090400054593C747002306A3
:10EBA000F400DDB78347850193F7E70FDDEB83477B
:10EBB0009501C5EB034625018346C50009CA3727E1
:10EBC0000020834565030347379A63E7E50013F7A1
:10EBD000060149CB014709C6C18A0357E51881C61A
:10EBE0008356251936973DCFB727002003D5479E7A
:10EBF0001307C71237460F00B335A702411113069A
:10EC00000624814622C426C206C67D543305A702C7
:10EC100097D006E0E780E07EB727002083C7779A89
:10EC2000B384A700B727002003A787BD8327070960
:10EC300063F387003E84184375FBB727002083A742
:10EC40004798829781476364A400B307A440B24009
:10EC50002244B3B7970093C7170092443E85410101
:10EC6000828081473E858280B727002003A7C7CADC
:10EC70003C5BFDFF010001008280011122CC4AC8EB
:10EC80004EC606CE26CA52C456C25AC00347B50065
:10EC900085472A842E8983290509631AF71E83571D
:10ECA0000508035BC503372A00209306CA9D83DA53
:10ECB0008600130ACA9D63F4671B834605016390AF
:10ECC000E61A03278511631C07180327450A6318F2
:10ECD00007188346F5001D476393E6180355A503FF
:10ECE000330BFB409307204E33056503832444090F
:10ECF00037460F008146130606243305F502B72771
:10ED0000002083C7679AB3549502B3B5AA02BE9494
:10ED1000C204C180231394083385AA0297D006E069
:10ED2000E780206EB307350133B5A7002E953E87E7
:10ED300083264A0019E163E4D7003387D740B384C0
:10ED40005403B7460F009387F623938606242320A7
:10ED5000E900A697B3D7D702DA97636CF70E1D8F39
:10ED60002320E900B729002083A7499883240900BC
:10ED7000829763E1A4123385A4406350050C83A7F6
:10ED80004998372B0020130BCB9D8297032709004E
:10ED90006368E510198D8357E40303578B008E07D2
:10EDA000B387E7021307003293870719B3D7E70247
:10EDB00063EDA70E374A0F00930AFA23130A0A24B9
:10EDC0008357040485072310F4048347041499E34C
:10EDD0002285512A2285971006E0E78000D87DE140
:10EDE000832604098327C40803274B00B6973E8572
:10EDF00063E4D70063E4E7003385E7408347F40129
:10EE0000835464082328A4088507A30FF4008357BC
:10EE10008B00B384F402D694B3D444036363950C9B
:10EE2000B304954083A7499823209900829763EE05
:10EE3000A40A3385A440E34505F8B727002083C71B
:10EE4000779A63E2A708B727002023A087BE014571
:10EE50009DA883264A00B387F6403E9711B7835496
:10EE6000640837470F009307F723B3845403BE9415
:10EE700093070724B3D7F40263E7F900B387F94097
:10EE80002320F900C5B503274A00BA99C5BF23A0BE
:10EE90003501C9BDB727002083A7079EBE94E1BDF9
:10EEA00083274B00998F3E95FDB5A145228597108C
:10EEB00006E0E780A0C3A305A402B727002083A72C
:10EEC000079C81EF7D55F2406244D2444249B249E9
:10EED000224A924A024B05618280894515458297F4
:10EEE000D5B7B3049740AA9435BF83274B00BE948F
:10EEF00089B72DC901116C0022CC06CE2A84B53BFE
:10EF000029CDFD576305F502372700201307079920
:10EF10005453B2479DC62547637FF700D9173EC6B5
:10EF2000B2450345940297F004E0E7808041F24047
:10EF3000624405618280372700200327079EBA9725
:10EF4000F1BF0347770163E4E700998FC9BFB72694
:10EF5000002083A6069EB697CDBF971006E0E780F7
:10EF6000404DF1B78280797126D206D622D44AD09C
:10EF70004ECE52CC56CA5AC85EC683475503034488
:10EF80007513AA843E941374F40F9307400263F63A
:10EF900087001304B4FD1374F40F03AA841383AA27
:10EFA000C413A38B841222865285D68597D006E09F
:10EFB000E7806042058915E503CBD41201498149F8
:10EFC000337B6403930B50024A865285D68597D0D3
:10EFD00006E0E7804040058915C563916903137415
:10EFE000F90F238B8412B250225492540259F249E1
:10EFF000624AD24A424BB24B456182808509E2099E
:10F0000093D989410509E31179FDE1BF832785097A
:10F0100003560504797193D60701BD8EC206C182DD
:10F02000358E1357764093575640898B058B5D8FED
:10F0300093573640918B5D8F93571640A18B5D8F10
:10F0400093171600C18B5D8F9317360093F7070255
:10F050005D8F931756009355860093F707041E069D
:10F060005D8F1376F60F518F93D7554013D63540E9
:10F07000118A898BD18F13D67540D18F13D6154045
:10F08000218AD18F13961500418AD18F13963500AE
:10F0900013760602D18F13965500137606049E054B
:10F0A000D18F93F5F50FCD8FA20745465D8F3307BE
:10F0B000C70222D42A8426D252CC56CA032A8413E9
:10F0C000832AC4135AC806D63697420741839357FA
:10F0D0007740135557400989858BC98F13553740A1
:10F0E0001189C98F135517402189C98F131517002E
:10F0F0004189C98F1315370013750502C98F131580
:10F10000570093558700137505041E07C98F1377A1
:10F11000F70FD98F13D5354013D755401189098B77
:10F12000498F13D57540498F13D515402189498FD3
:10F13000139515004189498F139535001375050204
:10F14000498F13955500137505049E05498F93F556
:10F15000F50F4D8F2207D98FB387C7024AD04ECE05
:10F160005EC662C4B697C207C18313D7774013D572
:10F1700057400989058B498F13D537401189498F2D
:10F1800013D517402189498F139517004189498F5D
:10F190001395370013750502498F1395570093D5C2
:10F1A0008700137505049E07498F93F7F70FD98FD2
:10F1B00013D5354013D755401189098B498F13D585
:10F1C0007540498F13D515402189498F1395150036
:10F1D0004189498F1395350013750502498F1395A1
:10F1E0005500137505049E05498F93F5F50F4D8F56
:10F1F0002207D98FB387C702130650025285D685DE
:10F20000B697BD8E93940601C18033F6C402137B7A
:10F21000F60F97D006E0E780001C05890DED8347C7
:10F22000D41201498149B3849702130C5002C18062
:10F230004A865285D68597D006E0E780C0190589B1
:10F24000937BF90F11C563863403850993F9F90F90
:10F250000509E31F89FD230B6413B2502254925415
:10F260000259F249624AD24A424BB24B224C4561A2
:10F2700082805E8BCDB70111B727002022CC03A47A
:10F2800087C026CA4AC84EC606CEAA8413092500DE
:10F29000854915C083C7140003473400858B630478
:10F2A000F700405CFDB71946930544004A85EFF02E
:10F2B0002FABE31835FF2285F2406244D244424925
:10F2C000B249056182804111B727002022C403A4FE
:10F2D00087C026C24AC006C693042500054901E836
:10F2E0002285B24022449244024941018280A6858F
:10F2F0001305A402974006E0E780C08DE30225FFD6
:10F30000405CF1BF0111B727002022CC03A407C045
:10F3100026CA06CE2AC42EC6854419E40145F24009
:10F320006244D24405618280834791000347140000
:10F33000858B6304F7000044CDB719469305A100FF
:10F3400013052400EFF0CFA1E31795FE0545C1BFDB
:10F35000EFF0EFBF73000000000000009712000004
:10F36000938262890383020023800200630F0300FB
:10F37000F32510342EC0970500009385A5FD7390EA
:10F380001534EF00A0477300203086DCEF00004703
:10F39000E65082800000B726002003A706C80111AE
:10F3A0004AC81C5F4EC606CE998322CC26CA858BDE
:10F3B0003689B7290020ADCF9307000637240020F7
:10F3C0001CDF930744C883C7670013070008930432
:10F3D00044C86319F70083A7C9C79C4393F7070480
:10F3E0002383F400834744C893F7070489CFB727E2
:10F3F000002083A747988297C8CC834744C893F7D7
:10F40000F70B2302F4C883C7440093F707048DE386
:10F410008547A382F400B727002083A7C7CA370710
:10F42000020098C7130700FC2382E4009848F8D331
:10F43000032709C81C5F9183858B95C31C5F93E7E5
:10F4400007011CDFB727002083A7C7CA054723A2EF
:10F450000706B7270020938747C82382E70083A7C2
:10F46000C9C7D8430583058B19C7D843759BD8C333
:10F47000D843799BD8C3F2406244D2444249B2494E
:10F4800005618280093F730020309317D50063DF48
:10F490000700B727002083A7C7CA7D57B8D7B7276B
:10F4A000002093878793D84F0507D8CF937785009F
:10F4B00099CFB7270020938747C803C72700136752
:10F4C00017002381E700130700F82382E7009377F2
:10F4D000150099CBB7270020938747C803C71700AB
:10F4E00013671700A380E700937765008DC7137734
:10F4F0004500B727002059CF03C747C81367170037
:10F500002382E7C8B727002003A707C85C57F19BF1
:10F5100093E717005CD79317F50063D20702B7276C
:10F520000020138787B483460707938787B4C18A6F
:10F53000BDCA8347070793E707022308F706931717
:10F54000E50063D60702B7270020938747C803C7A3
:10F550004700620761876355070005472382E7007C
:10F56000B727002083A7C7CA3707020098C7931799
:10F57000C50063D00702B7270020938787B403C76D
:10F580001707058B29C303C7170713672700A3882D
:10F59000E7068280938747C803C7370013671700C1
:10F5A000A381E70085B703C7070789463D8B63083A
:10F5B000D70003C707078D463D8BE312D7F81147E5
:10F5C0002388E706ADBF03C71707118B79D303C79D
:10F5D00017071367870065BFB7270020B7260020ED
:10F5E00003A6C7CA938746C803C746C8058B11C779
:10F5F00023820700A3820700828003C71700058BC0
:10F6000065FB785275F303C75700EDB73727002025
:10F61000032807C8832788039583858BC1E311C618
:10F6200083270803BD832300F60085CA832707C804
:10F63000985B4607935767016356070093E707C037
:10F64000C207C18303970600C207C18709C7BA97DB
:10F650000947B3C7E7022390F6009DCD8345150007
:10F6600085CDB7270020938747C883C767001387D6
:10F670009500894593F7070485C33A9583470500AC
:10F680000547994593F6F7066398E600E207E18798
:10F69000814563D30700B9452E8582808545EDBF3E
:10F6A000411126C206C622C44AC0B724002035ED47
:10F6B00083A6C4CAAE87F8527DFF372900201309FC
:10F6C00049C82301090037F400E03E85832704D1AF
:10F6D000B285ED9B2328F4D0832704D193E78702DA
:10F6E0002328F4D073005010975006E0E780E00A1A
:10F6F000B727002083A707C8B70680009843558F17
:10F7000098C3D857719BD8D783A7C4CAA30209004E
:10F71000A3000900094798C3832704D193E7870012
:10F720002328F4D07300501005A08D476314F5040E
:10F73000B727002083A707C8B70680009843558FD6
:10F7400098C3D857719BD8D783A6C4CAB7270020BF
:10F75000938747C803C72700058B19E703C73700FE
:10F76000058B51CB23820700B240224492440249C8
:10F77000410182808547E319F5FCB7F700E003A754
:10F7800007D16D9B23A8E7D003A707D11367870292
:10F7900023A8E7D07300501003A7C4CA8177FD17D0
:10F7A0005447F58F5CC70F10000003A7C4CAB70702
:10F7B0000200130600F81CC7B7270020938747C82C
:10F7C0002382C700B727002083A707C89C439D83D7
:10F7D000858B639FA700930760197CD354C737F7C5
:10F7E00000E0832707D193E787002328F7D01DBFC8
:10F7F0009307E01BDDB7F85231FFBDB7B7270020F4
:10F8000083A7C7CA8847D847798D09C988C7B7274A
:10F81000002003A3878963030300028382803727C4
:10F820000020B7260020138606CB130707CD834799
:10F83000D7008345B601484AAE97FD8BB355F50016
:10F84000A300F600A306F700858995E90347170191
:10F85000814613080002B3F7E7020147B355E500FC
:10F8600085899378F70F89C96395D700A30016019E
:10F870008280850693F6F60F0507E31107FF828065
:10F88000B727002083A74798011122CC26CA52C46B
:10F8900006CE4AC84EC68297B7240020938704CD6F
:10F8A0008047014A6301A406938404CD63668506FC
:10F8B000018D37270020930707CB83C7A701135477
:10F8C0005500137AF501130907CB636BF402B729CE
:10F8D00000209389C99DA1378346A90103A884000C
:10F8E00083A54900139756004297158C3A866364A6
:10F8F00007016364B7003306B74090C4E37DD4FCCE
:10F900001604336A4401F24062445285D2444249AB
:10F91000B249224A05618280B727002083A7079E4B
:10F9200033848740229571B7B727002003A7C7CA41
:10F930008967938707F47CD3B727002083A707D074
:10F9400083A60709139656006358060083A6070985
:10F9500013966600634406007453FDF28280000033
:10F96000B72700203727002083A707930327879214
:10F9700001456313F700828083D6670081E683D652
:10F98000470036959C43F5B7B727002083A5079914
:10F990003727002093870799138605222328C792CB
:10F9A00003D74700938785FFB72600204111BA97F8
:10F9B000056523A4F69206C61D05935637006374A9
:10F9C000E500930600203307D600372500202326C4
:10F9D000E59223A0E522E1162312D60023130600A8
:10F9E0001CC3998FE1172312F700231307008D3FE3
:10F9F000B240B7270020239FA79241018280B727FA
:10FA00000020B726002083A7079303A686922A87A3
:10FA1000B305B5406314F6003A8529A8938687009C
:10FA20009C43E369D7FEE377F7FE2E85E3E4D5FE3A
:10FA3000E3F2F5FE828023AC05FE1C4191E7010054
:10FA400001000CC18280BA8703A787FF6DFF23AC3A
:10FA5000B7FE8280184183A785FF6319B7001CC1D8
:10FA6000FD5723AC05FE238FF5FE8280232CF6FE86
:10FA7000C5BF411122C437E400E026C20440370765
:10FA8000200006C6F98C2320E4180F10000009E9B5
:10FA9000232094101545B2402244924441018280B3
:10FAA0000347E5FF9307F00F6306F7002320941048
:10FAB0001145D5B79700FB1FE7800067014523205C
:10FAC0009410D1BF411126C2B7E400E04AC003A997
:10FAD0000400B707200006C622C43379F90023A02A
:10FAE000F4180F10000009E923A02411B2402244A9
:10FAF00092440249410182809565938505D0C98D64
:10FB00002A842105C2054205C18141819700FB1F5E
:10FB1000E780405301CDFD572320050023128500C7
:10FB20002303F50023A024112105C9B723A0241124
:10FB300001456DBF0111B7E700E04AC803A90700FE
:10FB40004EC63707200006CE22CC26CAAA893379B2
:10FB5000E90023A0E7180F10000037250020032438
:10FB600045938144014619E499E8A1654E85EF006B
:10FB7000B00631A88347E4FF6397370395C8A6858D
:10FB800013054593C13D75D0A1654E85C92EF24040
:10FB90006244B7E700E023A0271126854249D244FA
:10FBA000B2490561828091E02286032484FF65BF0B
:10FBB000A284E5BF41114AC037E900E022C4032412
:10FBC00009003707200006C626C2798C2320E918D1
:10FBD0000F10000089E523208910154515A0B727CF
:10FBE000002083C79793AA842E8563F5F400894784
:10FBF00063EE9700BD3DB7E700E023A087100D45F9
:10FC0000B2402244924402494101828083A785FF89
:10FC100099E703C7E5FF9307F00F6308F700913DED
:10FC2000B7E700E023A087104DBF37250020238FC2
:10FC300095FE130545930135A16526850D260145E1
:10FC40002320891075BFB727002023AA079282803E
:10FC5000B727002083A7C79899E33E85828003D702
:10FC600027006316B70003C70700E308A7FEDC47B9
:10FC7000E5B7B9CD011106CE22CC26CA8147C146CF
:10FC800033D7F540058B21C312053E953147330527
:10FC9000E502372700208324079D05443314F40030
:10FCA0002EC642044180AA949C40C8408297B24527
:10FCB00023A0040023A20400A18DF2406244D24498
:10FCC0002E85056182808507E39CD7FA0144EDB754
:10FCD0002E858280BDCD797122D406D626D24AD017
:10FCE0004ECE01444147B3D78540858BB1CF120535
:10FCF000314722953305E502B727002003A9079D68
:10FD00008544B3948400C204C180BE892A99032724
:10FD1000090011C7032549002EC60297B245314795
:10FD20003304E40283A7099D3E941C4489E7232001
:10FD3000090023220900B2502254A58D0259925481
:10FD4000F2492E85456182800504E31EE4F8814472
:10FD5000DDB72E8582804111B7E700E026C28443DB
:10FD60003707200006C622C4F98C23A0E7180F101D
:10FD70000000B727002083A7079B37140020130437
:10FD8000847D91C782971C403E9508C031A0B7275B
:10FD9000002083A74798FDF70840B74703009387E3
:10FDA000D73F3305F502B7A72600938737ECB2405B
:10FDB0003E9508C02244B7E700E023A09710924484
:10FDC000410182800111B7E700E022CC80434AC89C
:10FDD0003707200006CE26CA2A892E86798C23A0D2
:10FDE000E7180F100000131506019305F004418178
:10FDF00032C69700FB1FE780E024AA8419C532466B
:10FE0000CA859700FB1FE780A041B7E700E023A069
:10FE10008710F240624426854249D24405618280BF
:10FE20007971B7E700E022D480433708200006D676
:10FE300026D24AD04ECE52CC56CA5AC85EC662C4EA
:10FE40003374040123A007190F10000005E123A05B
:10FE500087100945B250225492540259F249624A1D
:10FE6000D24A424BB24B224C45618280B7270020D8
:10FE700083A74798BA8A368AB28B2E8BAA89829733
:10FE8000B727002003A7079D3E898144B146C1479B
:10FE9000338CD40233068701104241E6C165938555
:10FEA00005F041459700FB1FE780C01919EDB72702
:10FEB000002083A7079C81C7814511458297B7E73A
:10FEC00000E023A087102D4571B7B727002003A7B6
:10FED000C79821E723A6A798230005008327099D3B
:10FEE00005473317970023260500232475012311A6
:10FEF000E50023225501E29723A0370123A26701E1
:10FF000023A4570163040A0023009A00B7E700E026
:10FF100023A0871001453DBF3E875C47F5FF48C7DA
:10FF200065BF8504E396F4F6B7E700E023A08710E9
:10FF300021450DB7B727002083A7879D411122C413
:10FF400006C6372400201304849389C782975C482F
:10FF50003E9548C84848B240224441018280B7E7F4
:10FF600000E09843B706200023A0D718758F0F1024
:10FF70000000B726002083C696936372D502372609
:10FF800000209316150003258698369583560500A4
:10FF9000D58D2310B50023A0E7100145828023A052
:10FFA000E7100D458280B7E700E09843B7062000D0
:10FFB00023A0D718758F0F100000B726002083C626
:10FFC00096936374D50237260020931615000325F7
:10FFD000869893C5F5FF369583560500F58D231059
:10FFE000B50023A0E7100145828023A0E7100D454E
:10FFF0008280011137E700E026CA0443B7062000DB
:020000040005F5
:1000000006CE22CC4AC84EC652C4F58C2320D7183F
:100010000F100000130705FF1377F70FFD4763E28A
:10002000E70AB146B306D502B727002003A7079D0C
:1000300036971C43D9C71359450005443D893315EC
:10004000A400131405014180AE894A85A2850931B7
:100050002A8A39C9A2854A85B937B727002083A7DC
:100060004798372900201309C99D82978357890033
:100070002A848146B385370313060064B3B7370378
:1000800013850532B335B500BE95EFE04110B307D7
:1000900085003E878326490063E4A70063E4D70018
:1000A0003387D7402324EA00B7E700E023A0971066
:1000B0000145F2406244D2444249B249224A0561B4
:1000C0008280B7E700E023A097100945DDB7011152
:1000D000B7E700E026CA84433707200006CE22CCCB
:1000E0004AC84EC6F98C23A0E7180F100000BD4780
:1000F00063E8A70431473307E502B727002083A749
:10010000079DBA979C438DCF05443314A400420445
:1001100041802E890145A285253EAA8911C5A28567
:100120000145513523A42901B7E700E023A097102A
:100130000145F2406244D2444249B249056182809D
:10014000B7E700E023A097100945E5B779714AD0D9
:1001500037E900E026D283240900B707200006D63D
:1001600022D44ECE52CC56CA5AC85EC6FD8C23202D
:10017000F9180F100000B727002083C79793637802
:10018000F500B727002083AB479863970B00B7E7CC
:1001900000E023A0971099A0B72900209389C99D5A
:1001A000AE8A03AB490083D58900B74736FE9387F3
:1001B00007C83E9BB387C5022A84328A8146B3B5FD
:1001C000C50213850732B337F50013060064BE95E8
:1001D000EFD0F17B6370AB02232099100145B25040
:1001E000225492540259F249624AD24A424BB24BCB
:1001F00045618280829B83D589002A891306006429
:10020000B38745038146B3B5450313850732B3373A
:10021000F500BE95EFD0B177B30725013E8903A75E
:10022000490063E4A70063E4E7003389E740D6852B
:100230002285393C09C923242501B7E700E023A022
:100240009710054569BF936504F0C205C18141451A
:100250009700FB1FE78000DF11E9B727002083A785
:10026000079C95D7A2851145829715B7372700209F
:100270008327C79895E32326A7988547232605005B
:10028000232425012311550123008500A300F50037
:10029000232205005DB7BA87D84775FFC8C7F1BFED
:1002A0007971B7E700E026D284433707200006D6ED
:1002B00022D44AD04ECE52CC56CA5AC85EC662C468
:1002C00066C26AC0F98C23A0E7180F1000002DC188
:1002D0004144B689B28A2E8A2A89B14C372B002034
:1002E000054D130C0003B30B940303270B9D5E977E
:1002F0001C43A5E39375F400B315BD0013554440AA
:10030000C2055686C1811375F50F893539C183271A
:100310000B9DDE9723A0270123A2470163840900D8
:1003200023808900B7E700E023A09710014521A0B2
:1003300023A097100945B250225492540259F24911
:10034000624AD24A424BB24B224C924C024D45611A
:1003500082800504E31984F9B7E700E023A0971031
:100360002145D1BF0111B7E700E026CA844322CC62
:100370004AC84EC63707200006CE2A84AE89328985
:10038000F98C23A0E7180F100000C9332285CE8511
:10039000C1302A8405C5B727002083D5479E1306A0
:1003A00000648146B3872503B3B52503138507325F
:1003B000B337F500BE95EFD0915D48C013351400FA
:1003C000F2406244B7E700E023A097104249D244CC
:1003D000B2490E05056182800111B7E700E04AC805
:1003E00003A9070022CC4EC63707200006CE26CA36
:1003F000AA892E843379E90023A0E7180F100000A2
:10040000EFF01F85AA8419C123110500A2854E852E
:10041000593EB727002083C7879363993701B727D1
:10042000002003D70798598C23908798B7E700E0FE
:1004300023A02711014591E01945F2406244D244BE
:100440004249B2490561828001114AC837E900E09A
:1004500022CC03240900B707200006CE26CA4EC6C8
:100460007D8C2320F9180F1000009307F00263E63B
:10047000A704B147B304F502B729002083A7099D5B
:10048000A6979C439DCB9377F5008545B395F500E2
:10049000C205C1811181893783A7099D0145A697AE
:1004A00023A0070023A2070023208910F240624402
:1004B000D2444249B24905618280B7E700E023A0F7
:1004C00087100945E5B74111B7E700E026C284432C
:1004D00006C622C437072000F98C23A0E7180F10A6
:1004E0000000EFF0EFF619E90145B2402244B7E70A
:1004F00000E023A09710924441018280B72700209A
:1005000083A7479800458297B72700209387C79D08
:100510006368A402D843B74636FE938606C83305FF
:10052000A4403697E372E5FC13070064B335E50297
:1005300003D6870081463305E502EFD0514575B7F4
:10054000D8433A94C1BF411122C426C237240020A7
:10055000B72400201307C49D938484939448584380
:10056000B727002006C683A747981304C49D63924B
:10057000E60882975440B74736FE938707C8B69778
:100580003387A7003A856364F7006364D7003305B7
:10059000D740B7240020938744C8DC53938444C8D1
:1005A00099CBB727002083A607D03707CDFF7D174B
:1005B0009C46F98F9CC611E14840B727002083A7CD
:1005C000479B829719E5DC5085C3EF60215CEF50B3
:1005D000B15ADC5091CBB727002003A707D0B7064C
:1005E00033001C47D58F1CC7B240224492444101BE
:1005F0008280829794485840B387A6003E8563E482
:10060000D700E3E8E7F83385E74061B74111B72742
:10061000002006C623ACA79C0295B240B727002055
:1006200023A8A794014541018280994763E9B70057
:10063000B72700208A0593874796BE9588C1828098
:10064000B727002023AAA79C11C5B727002005477C
:100650002381E7988280B727002023A60798B72731
:10066000002023AC079CB727002023A2079837253A
:100670000020B72700204111238107987146B72732
:10068000002081451305459606C623AA079C22C46F
:1006900026C2372400209700FB1FE78080BF130588
:1006A00084931306800281459700FB1FE78060BE9C
:1006B000EFF08FADB72700209387079903C5C703D5
:1006C00083C7D7031304849385453E958D4733052F
:1006D000F5029947B724002039051375F50F23015A
:1006E000A4003305F502130505249700FB1FE780DE
:1006F000609523A8A49C49C10346240099478145DD
:100700003306F602130606249700FB1FE78060B845
:1007100083A7049D03472400B72400209387072460
:100720000A0723A0F496BA97372700202324F798C6
:10073000EFF06FD1A5218347140083A604963706F6
:100740000500139727003697130646CD10C313876D
:1007500017001377F70F0A073706050036971306B9
:1007600026C710C313873700890793F7F70F8A0747
:10077000A300E400B69790C3B240224492444101E2
:10078000828037270020130787938347170083460B
:10079000270063F0D702B726002083A606961386AB
:1007A0001700A300C70013972700369708C33E859C
:1007B00082809307F00FE5BF1C41638C07104177DF
:1007C0007D8FB706002089476316D7100357450071
:1007D00063020710411126C21946AA849305F00F3F
:1007E000610506C622C49700FB1FE78000B90547D4
:1007F0008D47630AE50C9C4491C7D858994761C757
:10080000985C71C33724002013060004814513054A
:1008100004999700FB1FE780C0A713060004A68574
:10082000130504999700FB1FE780809F93070499A5
:1008300003D7C70009E7130700102396E70003C793
:10084000E70001E705472387E70003D7070101E732
:100850006D472398E70003C7F70001E71547A38713
:10086000E70003C7270101E705472389E70003C71E
:10087000370109E703C7F700A389E70003C757015A
:1008800001CB937637000983238ED702A38EE7022C
:1008900003C7470101E75547238AE70003C76401FF
:1008A00009E71307C003238BE7009C5791C7829782
:1008B000B72700202390A794B72700207D57A38255
:1008C000E7D6513B8147B240224492443E854101E4
:1008D000828089473E85828001114AC837290020DD
:1008E0008327C99D06CE22CC26CA52C456C24EC604
:1008F0008297130A0064B33545031309C99D835ACF
:1009000089008146568633054503EFD05108B72745
:10091000002013878793004FAA8401456306940241
:100920009389879333858440636E9400032549003F
:1009300056868146B335AA023305AA02EFD03105A7
:10094000018D269523AC9900F2406244D24442497D
:10095000B249224A924A05618280011122CC2E843A
:10096000B7E506000A8541469385C55D06CEEFD002
:10097000913B180806043A94B7270020035504FF5A
:1009800083D7679EF2406244AA9737450F0013054C
:1009900005243355F50205618280B727002083D7EF
:1009A000679E51471D45637CF70279471945637877
:1009B000F7021307200315456373F7021307B0040A
:1009C0001145637EF700130740060D456379F70074
:1009D0001307600909456374F70013B5B70F8280E8
:1009E000011122CC06CE2A842EC6EFF0CFB6B24536
:1009F000F240818D33A5A502229562441375F50F4F
:100A000005618280011122CC06CE2A842EC6EFF029
:100A10008FB4B245F240818D33A5A5022295624480
:100A20004205418105618280011122CC06CE2A84D3
:100A30002EC6EFF04FB2B245F240818D33B5A5021C
:100A40002295624405618280B727002013870799A9
:100A500018572DC3411122C426C24AC006C61389A5
:100A600007990297B72700201387879303578700BA
:100A70002A84938487930DCBBA876373A700AA87D0
:100A8000C207C183BA866373E400A286C206C1822C
:100A9000958F5147635AF7008327C90291C3829704
:100AA000EF50F17723948400B240224492440249EB
:100AB0004101828082800111B727002022CC372497
:100AC000002023A8079E93070499DC5706CE26CA68
:100AD000AA851304049981C72AC68297B245C9C161
:100AE0009C410545ADCBDC41BDC783D78500A5C77B
:100AF00083D7A500ADC3B72400201385C49D5146FC
:100B00009384C49D97F0FA1FE780807123860400C8
:100B1000B727002083A6C79D372700202322D79818
:100B2000034774011DE39387C79D03D5870093078F
:100B3000805737460F003305F50213060624814619
:100B40008145EFD0C164A30BA40037150500130540
:100B5000858D6D3C0145F2406244D244056182803E
:100B6000B7270020938787933707002023AE07001D
:100B70001307676EB727002023AEE79C3787320044
:100B80009387C79DFD56130727A1D4C398C7238613
:100B90000700B7C7004023A4D7269DBF011122CC70
:100BA0003724002093070499884706CE26CA4AC8EE
:100BB00001E90545F2406244D24442490561828020
:100BC000130404995C58F5D7185C65D77000854507
:100BD00082971844B247E30EF7FC0355C40093050F
:100BE000E004B724002097F0FA1FE780A0451387A0
:100BF000849308D3938484934DDD0356C4009305F6
:100C0000F00F014997F0FA1FE780A0688347E400DE
:100C10009050634DF900328597F0FA1FE780C0507D
:100C2000014523A0040223A2040269B78355C4002E
:100C30000844185CB3872503898105093E9508C2DD
:100C40000297E9B701114EC6B72900209387099989
:100C50009C4726CA4AC852C406CE22CC56C25AC0A5
:100C60002A8AAE843289638D071E9389099903A766
:100C70004903630407121307F01F6362A7123724A6
:100C8000002013078493832A070213048493639A32
:100C90000A0803D5C9009565938515E097F0FA1FFA
:100CA000E780403A08D02A866DC983D5C90083A75A
:100CB000490303A589008981829783A78900832A34
:100CC00004025CD089476316FA08C1476397F40CA5
:100CD00083D5C9009147938505FCB3C5F5028A0504
:100CE000D69503C725009307A0056314F70A83D799
:100CF00005006390470B4A852686910597F0FA1FF9
:100D0000E78000521C505685639357130145F2400B
:100D10006244D2444249B249224A924A024B056196
:100D200082805850E380E7FA03D5C9009565938522
:100D300025E097F0FA1FE780E030AA8A39CD83D505
:100D4000C9002A8683A7490303A589008981829760
:100D500095BF8D47631BFA00C1476390F40483D5A8
:100D6000C900938545FDF199A5BF91476318FA0025
:100D70006395440383D5C900A115F5B79307001007
:100D8000631DFA00A14763EA970083D5C900C11526
:100D9000D9BF1C5056856390570D29458DBF9D6A5C
:100DA000637C5509930A05E01947B3CAEA0203D7E1
:100DB000C900372B0020B38AEA02BE9A93078B93AF
:100DC000DC53130B8B936395570103240B021DE037
:100DD00003D5C9009305E00497F0FA1FE780802649
:100DE0002A8445DD83D5C90083A749032A868981E2
:100DF0005685829791451307A00589819397250011
:100E0000A29783C627006393E60483D60700639CFA
:100E1000460385058A052686A2954A8597F0FA1F1E
:100E2000E780004083270B02E38287EE228597F05C
:100E3000FA1FE780602FD9BD21677917E36FA7F408
:100E4000B30A5541ADB783C5370045BF83270B02B1
:100E5000E38587F4228597F0FA1FE780E02C35BF01
:100E6000B727002083A587958DD991479306A005C4
:100E70008983139727002E9703462700E31FD6F098
:100E800003560700631C460185078A072686BE9520
:100E90004A8597F0FA1FE780A0388DBD8347370059
:100EA000C1BFB727002093870799984729C3985F48
:100EB0001DCF8546631DD502411122C43724002071
:100EC00013048493105006C619CE83D5C70048502A
:100ED00089810297085097F0FA1FE780E0242320C9
:100EE000040223220402B240224441018280828013
:100EF000011122CC372400209307049956C283AAFB
:100F0000870026CA4AC84EC606CE52C42A89AE8475
:100F1000B28913040499638C0A1C1C5C99EB294563
:100F2000F2406244D2444249B249224A924A05619F
:100F300082805C58EDD79307F01F63E8A70C372A2F
:100F4000002093078A939C53130A8A93B9C70844D5
:100F500083274A02639FA70489476317F906C1479D
:100F6000E39FF4FA0355C4009147130505FC33458C
:100F7000F5029317250003250A022686CE853E95A5
:100F80009307A0052301F50023102501110597F013
:100F9000FA1FE780E028014561B70355C4009305B7
:100FA000E00497F0FA1FE780E0092320AA0245F148
:100FB000BDB78355C4005C5803260A028981829715
:100FC0001C442322FA0249BF8D47631CF900C14724
:100FD000E397F4F40355C400130545FD9377C5FF6B
:100FE00059BF91476318F900E39B24F30355C400EC
:100FF0002115EDB793070010E313F9F2A147E3E0E1
:1010000097F20355C4004115D1BF9D676378F5067B
:10101000930705E01947B3C7E7020357C400372A0F
:101020000020B387E702BE9A93078A939C53130A62
:101030008A93A1CF83274A026395570703250A02A3
:1010400091461308A0059305F00F93D72600139738
:1010500027002A97034627006316060783580700D0
:1010600003463700639C2805B306D64063C6960442
:1010700085078A072686CE853E9511BF2167791799
:10108000E36FA7E8B307F54049BF0355C4009305D4
:10109000E00497F0FA1FE780E0FA2320AA0259F94A
:1010A000BDBD8355C4005C5803260A02898156855C
:1010B000829723225A0359B72310B70093160601CB
:1010C000C18261B70356C400B3859600910513062B
:1010D00006FCE3F6C5E413863400719A1106B29655
:1010E0002301070123102701A301D70051B7372A95
:1010F000002093078A939C53130A8A93A9C303255C
:101100000A0291461308A0059305F00F93D7260015
:10111000139727002A970346270063140605835870
:1011200007000346370063982801B306D640E3D191
:1011300096F42310B70093160601C182C1BF034580
:10114000E4008357C4009305E0043305F50242052B
:10115000418197F0FA1FE780E0EE2320AA0245F1D3
:101160007DBB0356C4008345E400B385C5023386C6
:1011700096001106E3E5C5DAB9BF0145828083C751
:1011800005002300F50083D72500A300F50083D7D1
:101190002500A1832301F50083C74500A301F500C5
:1011A00011458280B727002023A60780B72700209B
:1011B00023A40780828029C1411126C206C622C409
:1011C000AA8401458DC52E84B7E5060022854146D7
:1011D0009385C55E97F0FA1FE780800483C70400FB
:1011E00005452306F40083C71400A306F400B240AB
:1011F000224492444101828001458280011122CC27
:1012000026CA06CE0947AA8432846381E504414692
:101210008147639BC500638FE6006397B6000DA806
:1012200041478147638EE600F2406244D2443E85E6
:10123000056182808A852285BD3F41468A8519A83D
:101240008A85953F41468A85228531A0E39AB6FC7E
:101250002E86A285268597F0FA1FE780A009AA8727
:10126000E1B7B727002023A4A7808280B7270020FA
:1012700023A6A7808280011122CC0354650006CEEC
:1012800026CA4AC84EC641C083298500AE842A8832
:1012900003C9090081471317890161876355070254
:1012A000B147054563FA87045114420403552800E9
:1012B000418033878900A2864E868545EFA0900C39
:1012C000B337A00085077D141355690042040589D2
:1012D0001379F90341802380F400A380A4002381C3
:1012E000240123928400014719C01387190098C470
:1012F00009476383E7000145F2406244D244424912
:10130000B249056182800545C5BFC167F917630A07
:10131000F502D94763F7B702011122CC2EC606CEDB
:101320002A84EF703055B2456368B5002285624467
:10133000F24005616F90E078F24062440545056136
:10134000828005458280C167F9176314F5006F70CC
:101350007052411106C6EF90806511E15D45B240C3
:101360004101828091476394F50283470500230081
:10137000F6008347250003471500A207D98F2311E4
:10138000F6008347350001452302F60082801145AF
:1013900082804111814522C426C206C6AA84052541
:1013A0002A8409E9B727002083A7878081C7F945E8
:1013B000268582972285B240224492444101828050
:1013C00039714ED656D25AD006DE22DC26DA4AD8F9
:1013D00052D4AA8A2E8BB28941EF36C6AD379145D9
:1013E000EF70105BAA844D492DC9B246054A23808F
:1013F00034010544630A0B00B68513851400029B73
:101400000505131405014180E20993D9894163D38D
:101410000902C1455685EF90C067654905E93386E5
:101420008400A2852685EFA000472A8905E13104C2
:101430004204418091472C085685231CF10026CE9A
:10144000231D8100EF8010702A8901C963070A00FB
:10145000268597F0FA1FE78020CDF25062544A8526
:10146000D2544259B259225A925A025B2161828067
:10147000BA84014AADBF011122CC26CA4AC84EC661
:1014800006CE2A893284B689253FAA840DE1B72782
:10149000002083A7C78081CF05476317E40003C4FA
:1014A000090005041374F40FA2854A858297F2405F
:1014B000624426854249D244B24905618280AE86A3
:1014C000B7150500014705469385E5176DB783D726
:1014D00005002300F50083D70500A183A300F500D4
:1014E0000945828083D705002300F50083D70500D6
:1014F000A183A300F50083D725002301F50083D73E
:101500002500A183A301F5001145828083D7050042
:101510002300F50083D70500A183A300F50083D73E
:1015200025002301F50083D72500A183A301F50041
:1015300083C755002302F50083C76500A302F500A9
:1015400003D58500190542054181828083D70500B6
:101550002300F50083D70500A183A300F50009450A
:10156000828083D705002300F50083D70500A1837F
:10157000A300F50083D725002301F50083D72500BC
:10158000A183A301F5001145828003D5450006051E
:1015900042054181828083D705002300F50083D76F
:1015A0000500A183A300F50003D525000905420528
:1015B0004181828083D705002300F50083D7050091
:1015C000A183A300F50083D725002301F50083D76D
:1015D0002500A183A301F50003D5450011054205AF
:1015E0004181828083C705002300F5000545828084
:1015F00083D70500411122C406C62300F50083D716
:1016000005002E841105A183A30EF5FE83D72500C6
:101610009505230FF5FE83D7D5FFA183A30FF5FE14
:1016200003C6F5FF97F0FA1FE78080BF034544002B
:10163000B24022441105410182808947639CF50034
:1016400083471500034705000145A207D98F2310E2
:10165000F60082801145828003D70500D94763FEDA
:10166000E702011122CC06CE2EC62A84EF7090200C
:10167000B24683D70600636DF50022856244F240CE
:10168000B7150500014709469385E54C05610DBB7B
:10169000F240624409450561828009458280914794
:1016A0009DC583460500FD15C2058547C18163922E
:1016B000F60213D725008D89914791E9914701CB17
:1016C00005052301D6002310E60048C281473E8568
:1016D000828009479147E39CE6FEC94733D7F5026C
:1016E000B3F5F502D1BFAE86B71505000147114627
:1016F0009385454EF1B193F7350091EB8981914780
:1017000089C52310B60048C281473E858280914733
:10171000EDBF03C745008947631AF702011122CCC8
:101720002A84C84506CEAE86014719C52EC69D45FA
:10173000EFE0EFACB2462A8722856244F240B7154B
:10174000050019469385C55005619DB909458280FC
:1017500099E1114582808347050005472311F60072
:10176000E379F7FEFD1593F5F50F33D7F502B3874F
:10177000E702E390F5FE050548C22310E6000145A7
:10178000828083C745000947AE866385E7004147ED
:101790006399E700B7150500014721469385055F6A
:1017A00005B1094582802310B60091E1014548C288
:1017B00001458280AE86B71505000147294693850D
:1017C000C554FDBE2310B60091E1014548C2014554
:1017D0008280AE86B71505000147314693852556B0
:1017E000C5B62310B60091E1014548C2014582808B
:1017F00003D74500854763FDE702011122CC2A8407
:10180000884106CE0DC12EC68545EFE04F9F2A8741
:1018100022856244B246F240B715050039469385E9
:10182000A558056171BEF240624409450561828098
:101830000945828091479DC5034705008D46914724
:1018400063F2E602FD15C205C181B3C6E5023308A5
:10185000D7026399050105052310D6002311E60080
:1018600048C281473E85828083C745000947AE86CE
:101870006385E70041476399E700B7150500014715
:1018800041469385055F2DBE09458280B335B00082
:10189000139525008280011122CC26CA06CE03C7EB
:1018A00085008547AA842E8449466310F702613C6F
:1018B0008357240049151306200963C8A700F24086
:1018C0006244D244094505618280034794008547FC
:1018D0006314F70013660604484011C58D4532C6EF
:1018E000EFE0EF913246A2866244F2402A872685D5
:1018F000D244B7150500938565590561D1B48D476C
:1019000063FFB7028347150003470500F115A207DF
:10191000D98F2310F6008347350003472500C20501
:10192000A207C181D98F2311F6002312B60089C501
:10193000110508C60145828023240600E5BF114534
:101940008280011122CC2A84884506CEAE8611C53C
:101950002EC69545EFE0AF8AB2462A8722856244BB
:10196000F240B715050059469385455B056189BC72
:10197000B335B000139525008280AE86B7150500FB
:10198000014761469385455E25BC8547114563F453
:10199000D7028347160083450600A207CD8F231088
:1019A000F7009387E6FF2311F70089476386F60067
:1019B000090650C30145828023220700E5BF014785
:1019C000814679468145EDBA83D705002300F500AD
:1019D00083D70500A183A300F5000945828083C752
:1019E000250005472300F50003D505006397E700B0
:1019F0000A050505420541818280C9473305F50284
:101A0000CDBF03D505000A0542054181828083D7F9
:101A100025002300F50003D5050083D725003305F5
:101A2000F502050542054181828003D505008280CB
:101A300003D50500828003D50500828083D7250069
:101A40002300F50003D5050083D725003305F502F3
:101A5000050542054181828083D705002300F500FA
:101A600083D70500A183A300F50083D725002301B8
:101A7000F50083D72500A183A301F50003D5450018
:101A8000110542054181828083D705002300F500BE
:101A900083D70500A183A300F50003D52500090520
:101AA00042054181828089471145639BF600834747
:101AB0001600834606000145A207D58F2310F700C4
:101AC000828003D70500D947AE8663F9E700B725C2
:101AD000050001470D469385859C71BA09458280B2
:101AE00011456393A602834716008346060001450D
:101AF000A207D58F2310F7008347360083462600C0
:101B0000A207D58F2311F700828083C725000547E0
:101B1000FD1793F7F70F6361F70483D705008DCFA7
:101B2000011122CC2A84C84106CE15C12EC6894592
:101B3000EFD0FFEC2A8722856244B246F240B725F7
:101B4000050015469385E59D05616FF0DF92F24033
:101B500062440945056182800945828095471145A7
:101B600063F9D706411122C426C24AC006C683477C
:101B70001600BA8403470600A2073284D98F239047
:101B8000F400834736000347260093054400A2076C
:101B9000D98F2391F40089472382F40009461385E5
:101BA0005400368997E0FA1FE78080679307A9FF02
:101BB0002394F4009947631BF90023A60400B24064
:101BC0002244924402490145410182801904C0C463
:101BD000FDB7828083D705008DCF011122CC2A84E6
:101BE000C84106CE15C12EC68545EFD05FE12A87D4
:101BF00022856244B246F240B72505001D46938512
:101C000025A005616FF03F87F240624409450561F8
:101C100082800945828099476395F604894741117E
:101C200006C62302F7008347160083460600B285E6
:101C3000A207D58F2310F70083473600834626007E
:101C400003464700A207D58F130557002311F7005D
:101C5000910597E0FA1FE780A05CB2400145410181
:101C60008280D14711456394F600C1474DBF828001
:101C700083D705008DCF011122CC2A84C84106CE1E
:101C800015C12EC68945EFD09FD72A872285624489
:101C9000B246F240B725050025469385E5A00561CB
:101CA0006FF06FFDF240624409450561828009458D
:101CB000828089471145639BF6008347160083465F
:101CC00006000145A207D58F2310F700828001117D
:101CD00022CC2A84C84106CEAE86014719C52EC63D
:101CE0008545EFD0DFD1B2462A8722856244F24093
:101CF000B72505002D469385A5A205616FF0AFF7C6
:101D000011456393A60283471600834606000145EA
:101D1000A207D58F2310F70083473600834626009D
:101D2000A207D58F2311F7008280011122CC2A84CB
:101D3000C84106CEAE8611C52EC68545EFD03FCC34
:101D4000B2462A8722856244F240B725050035460F
:101D5000938505A305616FF00FF293F71600114507
:101D600089EB89476387F60085822312D70010C369
:101D700001458280011122CC2A84C84106CE15C1BA
:101D80002EC68545EFD0BFC72A8722856244B2465A
:101D9000F240B72505003D46938565A305616FF0C8
:101DA0008FEDF240624409450561828083D70500CA
:101DB0008DCF011122CC2A84C84106CE15C12EC672
:101DC0008945EFD0DFC32A8722856244B246F240BC
:101DD000B725050045469385C5A305616FF0AFE9BA
:101DE000F240624409450561828009458280854749
:101DF00063FCD7022304A700A304B700834716009F
:101E000083450600A207CD8F2310F7009387E6FFD6
:101E10002311F70089476386F600090650C3014580
:101E2000828023220700E5BF114582800147814659
:101E30004D4681456FF02FE48D47114563FBD70276
:101E40008347160083450600A207CD8F2310F700B5
:101E50008347360083452600A207CD8F2311F70064
:101E60009387C6FF2312F7006386A600110610C7EA
:101E70000145828023240700E5BF011122CC2A847A
:101E8000884506CEAE8611C52EC69545EFD03FB724
:101E9000B2462A8722856244F240B72505005D4696
:101EA000938585A505616FF00FDD85471145639723
:101EB000F6008347060001452300F70082800147B2
:101EC0008146654681456FF00FDB011122CC2A84E3
:101ED000C84106CEAE86014719C52EC68D45EFD046
:101EE0001FB2B2462A8722856244F240B725050018
:101EF0006D46938585A805616FF08FCC011122CCCA
:101F00002A84C84106CEAE86014719C52EC68D4526
:101F1000EFD0FFAEB2462A8722856244F240B72551
:101F200005007546938585A805616FF06FC901119D
:101F300006CE2EC6EF80D02301C9B245F24003552C
:101F4000250005616FC0102EF24049450561828071
:101F5000B7270020A38C0782B7270020238C078295
:101F6000B727002023A00782B727002023A20782DB
:101F7000B727002023A40782B727002023A60782C3
:101F8000B727002023AE0780B727002023AC0780A7
:101F9000B7270020239A07A013064038938747A14C
:101FA0002391C70271761307400B130606B82391DD
:101FB000E7002392C70211671D46930600059305AB
:101FC000000A1305007D2392E7002393C7024147CF
:101FD0000546130810F82395E7002396E700239998
:101FE000E700239AE700239BE700239CE700239464
:101FF000E7022393B7002394B7002397D7002398D1
:10200000D700239DA700239E0700239F070023904E
:1020100007022395C7022396070323970702930815
:10202000F007239807022392E7042393E704239FF2
:10203000E7042390E7062391E7062392E706239916
:1020400017031307C01C239AC702239BC702239CB4
:102050000702239D0702239E0702239F0702239066
:1020600007042391C70423940704239507042396A8
:10207000C7042397D7042398D7042399A704239A46
:102080000704239B0704239C0704239DD704239E56
:10209000D7042393A70623940706239507062396C0
:1020A00007062397B7062398B70623990706239AAE
:1020B000E7067D57239B0706239007092391E7082E
:1020C0008280011126CAAA84214522CC06CE2E8404
:1020D00032C636C43AC2EFD0FF9E1DC9A24612478F
:1020E0003246930700FD2300F5009947A3009500B1
:1020F0002301F5002303D500A303E5002312C50047
:10210000AA8522856244F240D24405616FD09FAA1D
:10211000F2406244D24405618280B727002023A4A4
:10212000A7828280B727002023A6A7828280011180
:1021300022CC4AC806CE26CA2A890144B3048900A3
:102140006368B400F2406244D2444249056182802F
:102150002EC6EFD05FC093170501C183A183B2459E
:102160002380F4009307140093F7F70F850463F9B5
:10217000B700CA9709042380A7001374F40F7DBF2A
:102180003E847DBF411122C4372400201304449FA4
:1021900003556400C16706C6FD17630FF500B72736
:1021A000002003C687B3B725002093850583EF8001
:1021B000E05AFD572313F400B240224441018280CB
:1021C00009C925151375F50F1335850E134515002F
:1021D00082800145828023900500C9C6797122D48E
:1021E00026D24ECE52CC5AC806D64AD056CA5EC661
:1021F0003684328AAE892A8B814463F34407B3075D
:10220000940083C70700138914004209939A0701B9
:1022100093DA0A011359090163840A04CA976341D6
:10222000FA04B307240183CB07005E85513F0DC933
:102230009387FAFF2390F90063906B03130519004D
:102240002295B250225492540259F249624AD24A1B
:10225000424BB24B45618280D694C204C18071BFAB
:102260000145C5B701458280011122CC37240020E9
:1022700026CA4AC84EC69307449F06CE2E89D0CBA5
:102280008CCBC8C7AA8441469305F00F4A8597E0D6
:10229000FA1FE780800E85491304449F63193503B4
:1022A0000848C145693541469305F00F268597E0FA
:1022B000FA1FE780800C05496315250348446244F2
:1022C000F240D2444249B249C14505618DB541460B
:1022D00081454A8597E0FA1FE780200AE31535FD1E
:1022E000C1B741468145268597E0FA1FE780E0089F
:1022F000E30625FDF2406244D2444249B2490561F9
:102300008280411122C43724002026C24AC0AE84F4
:102310002A891306000281451305449F06C697E0EB
:10232000FA1FE78000F79307449FA3812701B7278F
:102330000020238E97B2EFC02071854719C18147D5
:102340004945230AF49EB240224492440249410185
:102350008280814781CD19C98547631BF50083C7FA
:10236000550093E707FCA382F50085473E858280F0
:1023700089476317F50083C7550093F7F703E5B75F
:102380000D478547E314E5FE03C755001377F703B0
:1023900013670704A382E500D1BF81478DC105C142
:1023A00003C755009306000C85471377070C630895
:1023B000D700930600048D476303D70089473E8505
:1023C0008280411122C4005D06C626C21DC8AA84AF
:1023D000085009C597E0FA1FE78000D5485009C5A5
:1023E00097E0FA1FE78040D4085409C597E0FA1F28
:1023F000E78080D3228597E0FA1FE780E0D223AC04
:102400000402B240224492444101828019E9B72774
:10241000002083C7679F91C73725002013050581DA
:102420008280372500201305C5A08280B7270020B1
:1024300003C5679F8280B727002003A507A082807D
:10244000B727002003A547A08280B727002083A7D5
:1024500087A088438280B72700209387479FD44B6B
:102460009842050798C203C537009307F00F63052C
:10247000F50091656FD0BFAE8280011122CC06CEEF
:102480002E8432C6EF80605F9147B2456310F5023B
:10249000B727002083A7C78295C303A30700630F54
:1024A000030022856244F24005610283B7270020C1
:1024B00083A7478281C703A34700D5B7F240624490
:1024C000054505618280011122CC2A84035545000F
:1024D00006CE26CA4AC84EC6EF8040383DC92A8972
:1024E000834405008349C500E93D4A85EF80101803
:1024F00003554400EF80A053372900201309898336
:1025000083470900B9CB639A9704B727002083C596
:1025100097832685293C19E12300090003554400CF
:10252000EF80A0559147631FF500B72700209387E0
:10253000479F8356440003D767006395E6007D57A5
:102540002393E700F2406244D2444249B249056114
:10255000828081499304F00F45B79307F00FE38F12
:10256000F4FA8346640003564400034524004E8772
:10257000A685813E65B779715EC6AA8B2E8552CC41
:1025800056CA5AC806D622D426D24AD04ECEAE8AD1
:10259000328B368AEF80802C7DC1045D2A89E5C0AC
:1025A0009C50614599C3130540039C5481C7510554
:1025B0004205418163050A00710542054181DC50F5
:1025C00081C75D0542054181EFD0CFCF2A8445C93F
:1025D0006146814597E0FA1FE780A0CBB72700202E
:1025E00083C947A46394090083490900930700FD48
:1025F0002300F400A947A30074012301F40023037E
:1026000064018C50231254011305840191C908C43C
:102610007146930A440397E0FA1FE78060C056852D
:102620008C5491C948C45146930A450197E0FA1F5A
:10263000E78000BF5685630C0A0008C87146D28542
:10264000930AC50197E0FA1FE78080BD5685CC50FC
:1026500099C548C85D4697E0FA1FE78060BCA2852F
:102660004E85EFD02FD52254B2509254F249624A8F
:10267000D24A424BB24B4A850259456199B3B25096
:10268000225492540259F249624AD24A424BB24B06
:102690004561828001114EC6AA892E854AC806CEA0
:1026A00022CC26CA2E89EF80601B21C9B7270020C3
:1026B00083C447A499E0834405001945EFD08FC037
:1026C0002A8405CD8145194697E0FA1FE78060BC52
:1026D000930700FD2300F400B947A3003401230150
:1026E000F40023122401A2856244F2404249B24917
:1026F0002685D24405616FD0EFCBF2406244D244CC
:102700004249B2490561828039715ECEAA8B2E851D
:1027100026DA4ED652D456D25AD006DE22DC4AD819
:10272000AE84328BB68A3A8ABE8942C6EF800013E5
:1027300021CD2A894145EFD0EFB82A8431C54146E1
:10274000814597E0FA1FE780C0B4B727002003C592
:1027500047A419E103450900930700FD2300F40095
:10276000BD472301F400B247A30074012312940073
:1027700023046401A304540123054401A305340187
:102780005CC4A285EFD00FC3F2506254D2544259B8
:10279000B259225A925A025BF24B216182807971BE
:1027A00026D2AA8439454AD04ECE06D622D42EC689
:1027B000B2893689EFD00FB121C1B2459307000D20
:1027C0002310F500B1472A842312B5002301F50038
:1027D000CE851905194697E0FA1FE78060A4230605
:1027E0002401A2852254B2500259F24913F5F40F84
:1027F000925445616FD00FBCB2502254925402598A
:10280000F24945618280411126C2B7240020938499
:10281000449F03C7340006C622C44AC09307F00F82
:10282000630CF7042A893945EFD0CFA92A8429C53A
:10283000930700FDB72500202300F500A300250124
:10284000230105009385C5A00D05194697E0FA1FE1
:10285000E780009D83D78400A28503C5340023153B
:10286000F40083C714002306F4002244B2409244CB
:10287000024941016FD00FB4B24022449244024950
:102880004101828001115AC02A8B314526CA4EC6A9
:1028900052C456C206CE22CC4AC8AE84B28A368A08
:1028A000BA89EFD02FA23DCD2A842685EF70107B08
:1028B00011C50347C500A1476314F704B7270020DB
:1028C00003C9779F930700FD2300F4009D47A300F1
:1028D00064012301F40023129400231354012314F0
:1028E000440123153401A2856244F240D244B24926
:1028F000224A924A024B4A85424905616FD08FAB0A
:10290000B727002003C9D7B3E31E0BFAB72700206F
:1029100083A7878D9C47DDD7CE865286D6852685B0
:1029200082974DB7F2406244D2444249B249224AAA
:10293000924A024B05618280011122CC2A842145F2
:1029400006CE2EC6EFD00F9821C1B245930700FDE9
:102950002300F500C5472301F50083C73500A30117
:10296000F50083D745002312F50083C765002303D4
:10297000F50083C77500AA85A303F500228562448C
:10298000F24005616FD00FA3F2406244056182807E
:10299000397162CC2A8C594526DA4AD84ED652D49F
:1029A00056D25AD05ECE06DE22DCAE8432C636C4A3
:1029B000BA8B3E8BC28A468A83590104034941047B
:1029C000EFD04F9025C93246930700FDA246230061
:1029D000F5009547A301C500A30085012301F5007B
:1029E0002A8419461105A9C2B68597E0FA1FE78027
:1029F000208323066401230A24012315740123176D
:102A000054012318440123193401A2856254F25061
:102A10004259B259225A925A025BF24B624C2685B5
:102A2000D25421616FD00F99814597E0FA1FE7805A
:102A30004086C1B7F2506254D2544259B259225A18
:102A4000925A025BF24B624C21618280411122C496
:102A5000372400201304449F8347240006C626C25F
:102A60008DCBB7240020AA8519461385048197D001
:102A7000FA1FE780E07A0345240093850481EFF094
:102A80005F8D2244B24013850481924441016FB0AE
:102A9000707CB24022449244014541018280411140
:102AA00026C2B72400209387449F06C622C44AC08A
:102AB00003C737009307F00F9384449F6304F70420
:102AC0002A892945EFD00F802A840DCD930700FD78
:102AD0002300F500A147A30025012301F50083C7CA
:102AE0002400B725002093850581A301F500194630
:102AF000110597D0FA1FE780A07203C53400A285A4
:102B0000EFD04F8B03C724008D476311F702B7271F
:102B1000002083A7878299CB03A387006308030063
:102B20002244B2409244024941010283B24022440D
:102B30009244024941018280797122D406D626D27C
:102B40004AD04ECE52CC56CA09445DCD2A8903558F
:102B50000500AE895144EF707050AA8455C53727DF
:102B60000020930787B383C747008546BA8AFD17BD
:102B700093F7F70F494463F9F6080347C500A147E7
:102B80006314F700639209089C5C4544B5EF9165B6
:102B9000938545711305C00297D0FA1FE780804ADC
:102BA00088DC2A8A4D442DC11306C002814597D086
:102BB000FA1FE780006E8357090093064A003685A6
:102BC0002311FA0071469305490036C697D0FA1FC3
:102BD000E780006589472300FA0003C5C400B246B8
:102BE0000356090083C58AB3611513351500EF80BC
:102BF000506D2A8463860900CE852685EF80A05615
:102C000001C42685EFF0EFFB2285B2502254925486
:102C10000259F249624AD24A45618280B7270020B0
:102C200083C7C7B30547FD1793F7F70F6378F70816
:102C3000894751C6011122CC26CA4AC84EC652C481
:102C400006CEAA89368AB2842E89EF7030412A8452
:102C5000D14729C9485509C597D0FA1FE780C04C0C
:102C6000F1452685EFD00F9648D4CD4705CD834654
:102C7000C40021478147639FE600630D0A000347B4
:102C8000A5010356050193062501AA854E85EF800F
:102C90002055AA8703474400630F090013676700A4
:102CA0002302E400F2406244D2444249B249224A3B
:102CB0003E850561828013674700DDB7C9473E85C1
:102CC00082809307000463EBA700B7270020938757
:102CD00047A106053E9503550500828041657D1597
:102CE0008280011122CC2A842E8526CA06CEAE848B
:102CF000EF70D0361DCDB7470F009387F7230945F6
:102D000063E4870281450A85414697D0FA1FE78030
:102D10004058A685231081000A8541802301810047
:102D2000A3010100EF809045F2406244D244056166
:102D300082804945D5BFB7270020238DA7B2828066
:102D40006F805052797152CC2A8A328522D426D291
:102D50004AD04ECE56CA5AC85EC606D662C4AE8B9C
:102D6000B28A368BBA843E89C2894684EF70102FAE
:102D700015C92A8C63140A0213774B008347450058
:102D800015CF93E727012302FC008DEC631C090299
:102D9000639A090205E8ED9B2302FC00832B8C0358
:102DA000639F0B06B250225492540259F249624A70
:102DB000D24A424BB24B224C45618280F59B93E74D
:102DC0000701D1B793E747002302FC0001CC1C4860
:102DD0004146A2852324FC0213058C0197D0FA1FDB
:102DE000E780004463910B02D5D80325CC0209C5C6
:102DF00097D0FA1FE7804033F1452685EFC09FFC4E
:102E00002326AC0261BFE30B09F80325CC0209C5F8
:102E100097D0FA1FE7804031F1454A85C5B79DC478
:102E200083A70B0299EB916593853571714597D016
:102E3000FA1FE780202123A0AB0203A50B0219C5CE
:102E40007146A68597D0FA1FE780803D6388090206
:102E500083A74B0299EB9165938525715D4597D0CA
:102E6000FA1FE780201E23A2AB0203A54B0219C55F
:102E70005D46CE8597D0FA1FE780803A1DC483A7B0
:102E80008B0299EB916593851571514597D0FA1F87
:102E9000E780401B23A4AB0203A58B0219C5514652
:102EA000A28597D0FA1FE780A0372254B2509254DF
:102EB000F249B24B224CCA865A860259424BD685F9
:102EC0005285D24A624A45616FF0EFEA011126CA83
:102ED00052C406CE22CC4AC84EC62A8AAE84EF70AF
:102EE000F01725C5AA893945EFC0DFBD2A8431CD49
:102EF000B727002003C947A46314090003C90900C8
:102F00009307000D2310F400AD472301F4009385CF
:102F1000690013053400194697D0FA1FE780403046
:102F200093F71400858085882306F400A306940097
:102F300023154401A2856244F240D244B249224A98
:102F40004A85424905616FC0FFC6F2406244D244DF
:102F50004249B249224A0561828001114EC652C4DB
:102F600056C206CE22CC26CA4AC8AA8A2E8AB2895E
:102F7000EF70D00E2DCD2A891305C002EFC09FB48B
:102F80002A8435C5B727002083C447A499E0834429
:102F900009009307000D2310F400E9472301F40012
:102FA0009305690013053400194697D0FA1FE7808E
:102FB0002027D285231554011305C400414697D01C
:102FC000FA1FE780E025CE851305C401414697D05E
:102FD000FA1FE780E024A2856244F2404249B249E8
:102FE000224A924A2685D24405616FC0BFBCF24096
:102FF0006244D2444249B249224A924A05618280DF
:10300000411122C43724002013048481084006C6DD
:1030100019C597D0FA1FE780201123200400B24081
:10302000224441018280011106CE22CC26CA4AC820
:103030002EC6EF70B00239CDB245B727002003C9C4
:1030400047A40CD5AA84631409000349050041452F
:10305000EFC05FA72A841DCD9307000D2310F50054
:10306000A5472301F50083C754009385640011052B
:10307000A30FF5FE194697D0FA1FE780601A9C54FB
:10308000A285F2405CC46244D2444A85424905614B
:103090006FC05FB2F2406244D2444249056182800F
:1030A0001D71A2CC86CE2A842EC6EF70207B05CD62
:1030B0008346C5001147AA8749456392E6029C5F93
:1030C000B24599C383C56701B7D605002308B1008F
:1030D0009386A6A7100889452285EF70907FF64059
:1030E0006644256182805145DDBFB727002083C734
:1030F000C7B30547FD1793F7F70F637AF7048947BE
:1031000021CA411122C426C24AC006C6B2842E89F1
:10311000EF70C0742A84D14705C56308090083474E
:10312000450093E727002302F5004146A6851305D5
:10313000840197D0FA1FE780A00E9C481CD48147D9
:10314000B2402244924402493E8541018280C947EF
:103150003E858280797122D406D62A842EC6EF70ED
:10316000E06F01CDB2452285230EB1006C08EF70EF
:10317000107CB2502254456182805145DDBF6F7092
:103180009004C1671387E7FF6395E502B727002026
:1031900083A7478291EB494582804945B24022444A
:1031A000924402494101828003A30700E30503FE24
:1031B0000283411122C426C24AC006C6FD172A89CD
:1031C0002E84B284639AF502B727002083A7478232
:1031D00091CF9C4381CF829711E9B7270020238CA0
:1031E0002783B7270020A38C97824DBFA6854A85E9
:1031F000EFE0FFD345F5D5B72E85EF70206651DDA2
:10320000834705000D45E39B27F922852244B24000
:103210000249A685924441016FB0D0009307000493
:1032200063E2A7064111C16722C406C626C2FD1784
:103230002A8409456382F502C547AE846313F4020C
:103240002E85EFB0B00537250020130545A10604F3
:103250002A94231094000145B24022449244410133
:1032600082809307A0036316F4002E85EFB0407CA4
:10327000D9BF9307B003E318F4FC13F5F50FEFB0D3
:10328000607BD1B709458280011106CE2AC6EFE0E6
:103290003FCCEF10C01CEFA0910EB7270020938702
:1032A000479F130700F02391E70023820700B72709
:1032B00000203245138787B3FD562301D700F24023
:1032C000238CA7B2954505616F50F06659719397AD
:1032D0000501A6D286D6A2D4CAD0CECED2CCD6CA2A
:1032E000DAC8DEC6E2C4E6C2EAC06EDEC187AE84DA
:1032F00063D3075237240020034584B337290020C5
:10330000372A0020EFC01F83AA8C22CCB72A0020C6
:10331000B72B00201304499F372C002063930C0225
:103320002165258DB650265496540659F649664AAD
:10333000D64A464BB64B264C964C064DF25D65611F
:10334000828083C70C001307200A639CE70083492F
:10335000340003D52C00C1656686FD15EFF0EF91B2
:103360009DA26247130787B38349270013071009FB
:103370006398E71683C71C001547639FE7006685BF
:10338000EFF06F946685EFC0CFEEE24703C587B3D9
:10339000EFC04FFAAA8C59B73947639BE71603D59C
:1033A0004C008567A5076316F50483A58C0003CB45
:1033B0000500631D0B00850591C9372500201946BE
:1033C0001305C5A097D0FA1FE78080E50347499F02
:1033D00085476317F71063080B00230A099E5A8577
:1033E000EFF06FC245B78947230AF99EEFB04066F8
:1033F00051BF896713872700631CE50403AB8C006A
:1034000063000B0E83470B0089EF83472B000347B4
:103410001B00A207D98F2314F40083473B00A300AD
:10342000F4000347499F8947631CF70A83470B0051
:1034300091C7230A099E03450B005DB7834514001D
:10344000035584008D47230AF99EEF50D051E5B70C
:1034500095076319F50083A78C0003C50700EFF0FB
:103460000FE40DB7F9771387A7FF2A974207418327
:10347000914663F1E6049387A7FCAA97C207C1832C
:1034800071476371F70289671387B7006310E5041A
:1034900083A70A82E38807EE9C43E685E38407EE70
:1034A000829715A0370700181307F770B357F70076
:1034B000858BA9CB83278A82E38607EC9C43E38331
:1034C00007EC66858297E31F05EA19A81387C700F2
:1034D0006311E50283A78C0083C70700E38407EA32
:1034E0009307F00FE380F9EAE6854E85EFC08FEC95
:1034F00069BDB9076318F50083274C82E38407E8A8
:10350000DC4361BF896793871704E303F5F8C9BFFC
:103510003D476399E70403D54C0089671387D700BB
:10352000E30CE5FC13879701E308E5FCCD07E319FD
:10353000F5FA03576400C167FD17631DF700832781
:103540004C82E38107E4DC43E38E07E20965E6850C
:103550004D05B9B7B727002083A7C782E38407E2E8
:103560009C43DDB71307E003E39CE7F683C72C0019
:1035700005476398E70E83C76C0037270020930D3B
:103580008781E1E783A70D00D5CF03CB0700A149D1
:1035900003C57C00138D8C00EA85EFE01FE083C734
:1035A0004C01A383AC0083D80C0103D8EC0003D7F3
:1035B0004C002A8603C53C003EC283D72C01EA8614
:1035C000DA853EC0CE87EFF0AFBC83C73C0095E7FD
:1035D000DD4783D80C0103D8EC0083C67C0083D57B
:1035E0004C003EC283D72C016A873EC0CE87054679
:1035F0005A85EF70805FA381AC0083A70D0081C75F
:103600001145EFF0FF9F138B8B8303450B00E30BFA
:1036100005D6B727002083C59783EFE05F91E303CA
:1036200005D683C63C0093071003638AF60003D6D1
:103630004C0083450B004E873685EFE09FA8238C16
:103640000B8289B3034B340099B783278A82034BDB
:103650003400914995DFDC4385DF81450145829740
:1036600005BF29476398E70A83C76C003727002006
:10367000930D8781A5EF83A70D00B5C703CB070086
:10368000A14903C57C0093868C0093772500BDCBB0
:1036900013761500138E4C0183C70C0283D8CC011E
:1036A00003D8AC0103D74C0003C53C003EC283D70E
:1036B000EC01DA8572CE3EC0CE87EFF06FAD83C7E6
:1036C0003C00724E9DFBDD4783D8CC0103D8AC0192
:1036D00083C67C0083D54C003EC283D7EC01728741
:1036E0003EC0CE8729B7034B340059BF83278A8257
:1036F000034B34009149D1D7DC43C1D78145014503
:10370000829741B7B68536CEEFE03FC9F2462A86AA
:10371000368E59B70947639CE70083A70A82E38383
:1037200007C6DC43E38007C666858297A1B92D47AB
:103730006398E70083A70A82E38607C49C47DDB746
:103740000D476397E70066868D4503D54C0039B178
:1037500019476395E7069305610213051031EFA041
:10376000A14A2C1013052031EFA0014A03D66C00AA
:103770008357810203D54C0063E8C70083D68C00D1
:103780000357610263F7E60093050002EFB00030D3
:10379000D5BE6374E6002393EC0063F4D700239452
:1037A000FC0003D7CC0083D6AC0003D68C0083D5B5
:1037B0006C0001488147EFB0202DE9B61D47E38139
:1037C000E7D231476395E7006686B145BDBF35470F
:1037D0006398E70083A70A82E38607BADC4799B7B4
:1037E0004947639DE70083278A82E38B07CEDC434A
:1037F000E38807CE814505458297DDB14D47E391CA
:10380000E7CE83278A82E38D07CCDC43E38A07CCAB
:10381000E6850945D5B793F7150089CFB72700206E
:1038200083A7078289C7DC4399C30145829713C5E3
:103830001400CDBC93F7250091CFB727002083A7B4
:10384000878291C7DC4381C781450545829713C5AF
:103850002400C9BC93F745000145E38507ACB727B1
:10386000002083A7C781372400201304449F91CFF1
:1038700085472302F400B727002083A7878291C7DA
:10388000DC4381C781450545829748442C10EF7081
:10389000507B2810EFF08F9BB727002083D767A3BA
:1038A00081CF130600643386C702B727002003C503
:1038B00087B39145EFC09F8913C54400A5B441115A
:1038C00022C4372400200325C48106C619C597D019
:1038D000FA1FE7806085232E0480B2402244410114
:1038E00082805971A2D4372400208327C48186D6D0
:1038F000A6D2CAD0CECED2CCD6CADAC80545638D00
:10390000070C9305F1041305F041EF807113930543
:10391000F1041305F041EF80B112B727002093871F
:10392000479F83C727000347F104B337F00011C353
:1039300089070327C4813EDE03453700930547000E
:10394000EFE03FA10327C4812ADC0D458345270012
:103950002EDAEFF00FB72AD81145EFF08FB6032417
:10396000C4812AD665450347A400034BB4003AD46A
:10397000EFF02FB5AA846945EFF0AFB42A897145FD
:10398000EFF02FB4AA896D45EFF0AFB32A8A7545E1
:10399000EFF02FB3AA8A7945EFF0AFB2E204625894
:1039A000F2572257B2564256D2551375F50F93FA75
:1039B000FA0F137AFA0F93F9F90F1379F90FE184DB
:1039C0002ACC56CA52C84EC64AC426C25AC0930808
:1039D00044000545EFB0400DB650265496540659A4
:1039E000F649664AD64A464B65618280011122CC6F
:1039F00006CE26CA8D472E846315F50603C735000B
:103A0000B7240020E94703D545009384449F6316FB
:103A1000F70083D764006382A706EF60306409C5AE
:103A2000835764002317F5000357A40083568400CE
:103A3000035664008355440003453400EFE09FE4DF
:103A40000357440083D764006309F7008547F240B9
:103A50006244D2443E8505618280FD572393F40081
:103A6000F5B78967CD07631DF50083C7250031478A
:103A70006385E7004547E39BE7FCEFE0AFF0F9B76C
:103A8000B1476319F500B727002003C5D7B3EFE0AE
:103A9000BFEA6DBF41677D178147E31AE5FA83C628
:103AA00055004947E395E6FA83C5450003552400D0
:103AB000300023140100EF60B04649BF411122C419
:103AC000372400208347A48326C206C64AC01307B2
:103AD000E00FAE846386E7041307F00F1304A4839A
:103AE0006387E7021145EFB0FFFD15C1930700FDA5
:103AF0002300F50089472301F5008547A3009500C1
:103B0000A301F500AA8503450400EFC0AF8AF95769
:103B10002300F400B24022449244024941018280D1
:103B20002A891145EFB01FFA75D5930700FD2300D0
:103B3000F50089472301F500A3009500A3012501A5
:103B40002244B7270020B24092440249AA8503C507
:103B5000B78341016FC00F8679714AD037290020A1
:103B60008327C98122D406D626D24ECE52CC56CA3D
:103B70004544D5EFB7240020938784B383C747001B
:103B80004944958BCDC7B72700202E8A9165A38D18
:103B9000A782AA8993857571314597C0FA1FE7807E
:103BA000604A232EA9804D4459C123003501A3004A
:103BB00005002946D285090597C0FA1FE7804066AF
:103BC0008327C981914603C7270063EDE60835EBDB
:103BD0004D472381E70003C72700136707012381AF
:103BE000E700930571001305F041EF80616583479D
:103BF0007100F1EBB727002003C7679F8D4763145F
:103C0000F70CEFE05F832C00EF70B0432800EFE08B
:103C1000FFE34545EFF0EF8A014411C91306006444
:103C20003306C50203C584B39145EFC02FD2228568
:103C3000B250225492540259F249624AD24A456122
:103C4000828085466314D700754761B7894663143F
:103C5000D7004947BDBF8D466314D700414795BF84
:103C6000554785BF9546CA8A630ED70099466316A5
:103C7000D70009472381E70031A01D466314C7021E
:103C8000238107006545EFF0CF839307F007E30A30
:103C9000F5F403A7CA818347270093E707042301AC
:103CA000F70081B721466314C7000547E1B72546F1
:103CB0006315C7002381D700F1B7A9460544E3186F
:103CC000D7F6114745BF31392A8435D1CD3E85B766
:103CD000011126CAB724002083A7C48122CC06CEB6
:103CE0004AC84944B1C783C707000D446392A7047B
:103CF00037290020034589B38945EFC0EFED03451F
:103D000089B3B72700209145239E0782EFC0CFECEF
:103D100083A7C48101478146A38087001306F10071
:103D2000854785450145A307F100EFA0505B2A8434
:103D30002285F2406244D2444249056182800111E9
:103D400006CE22CC26CA4AC88547631EF50637240C
:103D500000201304C48383570400A9CB3727002015
:103D60000347879F21E71307B003636CF702B7246B
:103D7000002003C584B38945EFC00FE60356040055
:103D80009307006403C584B33306F6028945EFC088
:103D9000EFBB23100400F2406244D2444249056163
:103DA0008280938747FC2310F400F5B7B7270020E3
:103DB00083A7C781EDD36244F240D244424903C590
:103DC0000700056131B7B724002083A7C481E1D77C
:103DD00037270020130987B383474900918BC5DF3C
:103DE00089476313F5062D452EC6EFB0BFCD2A8453
:103DF0005DD1B245930700FD2300F500E547A30020
:103E000005002301F50083C7350015051946230F6A
:103E1000F5FE83C745009505A30FF5FE97C0FA1F71
:103E2000E7800040034559009307F00F6316F50043
:103E300083A7C48103C50700A2856244F240D2442F
:103E4000424905616FB01FD7034587B38945EFC06D
:103E5000AFD86244F240D2444249B7270020239EA3
:103E6000078205616FF0BFA549458280B727002012
:103E700083C7C7B3958B638F07129307C01C63FC7E
:103E8000C70009458280F2406244D2444249B249A7
:103E9000094505618280B727002083A7C781638B0E
:103EA0000710B72700209387A78303C807001307CD
:103EB000E00F6311E810011122CC4AC806CE26CAD1
:103EC0004EC62380A700130586004205368932843A
:103ED0004181ADC991659385657197C0FA1FE780EF
:103EE0006016AA894DD1B724002003A54484938489
:103EF000448409C597C0FA1FE78000231385890011
:103F000023A0A9002286814523A0340197C0FA1F6F
:103F1000E78020389C402286CA85884397C0FA1FD4
:103F2000E78000309C40A286F240239287006244E2
:103F3000D2444249B249984305468D45054505613D
:103F40006FA0703991659385557197C0FA1FE7800E
:103F5000600FAA890DD9B724002003A5C4849384D7
:103F6000C48409C597C0FA1FE780001C1385890027
:103F700023A0A9002286814523A0340197C0FA1FFF
:103F8000E78020319C402286CA85884397C0FA1F6B
:103F9000E78000299C40A286F24023928700624479
:103FA000D2444249B249984305468D4505450561CD
:103FB0006FA0B032494582809307C01C63FCA70004
:103FC000094582800945F2406244D2444249B249DF
:103FD0000561828045CD011122CC2A8421054EC67F
:103FE0004205AE8991659385657141814AC806CEC7
:103FF00026CA97C0FA1FE780E0042A8961D5B72452
:10400000002003A544849384448409C597C0FA1F03
:10401000E7808011130589002320A90022868145AD
:1040200023A0240197C0FA1FE780A0269C40228687
:10403000CE85884397C0FA1FE780801E9C4023925C
:104040008700B727002083A7C7818DCFB72700201F
:1040500083C7C7B3958B8DCBB727002083A7478431
:1040600099CF984383D647006244F240D2444249F4
:10407000B24905468D45054505616FA0D02501472C
:104080008146DDB7014581B7494535BFB7270020D7
:1040900083A7C78195C7B727002083C7C7B3958B70
:1040A00095C3B727002083A7478481CB984383D645
:1040B000470005468D450545C9B701478146D5BF2F
:1040C00001458280494582809307C01C63FCA7009C
:1040D000094582800945F2406244D2444249B249CE
:1040E0000561828045CD011122CC2A8421054EC66E
:1040F0004205AE8991659385557141814AC806CEC6
:1041000026CA97C0FA1FE780E0F32A8961D5B72451
:10411000002003A5C4849384C48409C597C0FA1FF2
:10412000E7808000130589002320A90022868145AD
:1041300023A0240197C0FA1FE780A0159C40228687
:10414000CE85884397C0FA1FE780800D9C4023925C
:104150008700B727002083A7C7818DCFB72700200E
:1041600083C7C7B3958B8DCBB727002083A7C784A0
:1041700099CF984383D647006244F240D2444249E3
:10418000B24905468D45054505616FA010150147EB
:104190008146DDB7014581B7494535BFB7270020C6
:1041A00083A7C78195C7B727002083C7C7B3958B5F
:1041B00095C3B727002083A7C78481CB984383D6B4
:1041C000470005468D450545C9B701478146D5BF1E
:1041D00001458280494582809307C01C63F4A70093
:1041E00009458280797122D44ECE06D626D24AD095
:1041F000AE892A842DC1210591654205938575718B
:10420000418197C0FA1FE780E0E32A8909456306E8
:104210000908B724002003A584849384848409C5F5
:1042200097C0FA1FE78040F0130589002320A900FA
:104230002286814523A0240197C0FA1FE7806005EC
:104240009C402286CE85884397C0FA1FE78040FDB8
:104250009C4023928700B727002083A7C781014590
:104260008DCFB727002083C7C7B34945958B95C726
:104270006C001305D030EF903119B247014593F728
:10428000070F81CFB727002083A787848D45054579
:10429000944303D64700EFA0D004B2502254925466
:1042A0000259F24945618280B727002083A74784DD
:1042B00091CF03D647008C43411106C697C0FA1F21
:1042C000E78000F6B24001454101828009458280C5
:1042D000B727002083A747848DC7B727002003A7EF
:1042E000C784894705C3035647000C43411106C6DE
:1042F00097C0FA1FE780C0F2B24081473E85410176
:10430000828089473E858280797106D622D426D262
:104310004AD04ECE52CC8D4763FCA7008944B250A0
:104320002254268502599254F249624A456182809C
:10433000372900200347499FC144E312F7FE930742
:10434000F5FF9309499F93F7F70F8546AE842A84BA
:1043500003CA29001309499F63EAF6068DE19945CE
:104360002800EFD0DFDCB729002003C589B39145D1
:1043700023018900EFC04F8635E481444DB71946CB
:104380008145280097C0FA1FE780A0F019462C004D
:10439000268597C0FA1FE780E0F549F11946930595
:1043A000F00F280097C0FA1FE780A0EE19462C00F6
:1043B000268597C0FA1FE780E0F32DF11946A68500
:1043C000280097C0FA1FE780A0E571BFE31DE5F85C
:1043D00003A5C9002C00EF70C046AA8449D52381EB
:1043E000490135BF2800EFE06FE6AA840DED930583
:1043F00071001305F041EF70B16483447100B5FCA6
:104400008D47E31CF4F64545EFE0BF8B3DD5B7770C
:104410001800938707A03306F50203C589B39145B9
:10442000EFB05FF4EDBD23014901D5BDB7270020F2
:1044300083C7C7B3918B8DC3372500204111130566
:10444000058406C6EFD01FCEB240B72700207D57A7
:10445000239DE79E4101828001456FD0BFCCB727E5
:1044600000207D57A38DE782B72700207957238D41
:10447000E782B7270020238C07A8B7270020239EB8
:104480000782B727002023A20784B727002023A68E
:104490000784B727002023A4078437470500B727E0
:1044A00000209387078E1307876798C33747050057
:1044B0001307E7D3D8C3374705001307278E98C7DC
:1044C000B7470500372700209387C79E2320F7842E
:1044D0008280411126C2B724002083A7C48106C66A
:1044E00022C48DCF2A840D45EFB0CFDDAA8505C14A
:1044F000930700FD2300F5008D47A30085002301ED
:10450000F50083A7C48103C50700EFB0AFEA19C463
:104510002244B240924441016FF06FBAB24022444B
:10452000924441018280797152CC372A002083273E
:10453000CA814AD006D622D426D24ECE56CA0149C6
:10454000B1C703C91700B72400208547AA899384FF
:10455000449F6307F90483C74400054985EB0D4573
:10456000EFB04FD6AA8505C1930700FD2300F500E3
:104570009147A30035012301F5008327CA8103C5B4
:104580000700EFB02FE3EFF08FB30549B25022548C
:104590004A8592540259F249624AD24A4561828060
:1045A000B727002083A74784D28A85E30145EFE03F
:1045B0004FF12A8601CAB727002003C587B3894572
:1045C000EFB0DFB883A7CA8181A8944303D6470020
:1045D0009305E1000545EFD01FC069D98347050069
:1045E000858BE9D70545EFE0CFED9307B0032A842B
:1045F00063F0A704B727002003C587B35D661306E1
:1046000006708945EFB01FD6B7270020130444FC7D
:10461000239E87828327CA810947A380E70083C737
:10462000440081C72382040095B74E855D35B9BF2C
:10463000130600643306C502B5BF411122C42A84A3
:104640000D4506C6EFB00FC805C5930700FD230052
:10465000F500CD472301F500A30085002244B727CC
:104660000020B240AA8503C5B78341016FB08FD443
:10467000B24022444101828083564500011189677E
:1046800006CE22CC26CA138667002A876399C60005
:104690001C47014583C50700EFF04FC23DA81386B4
:1046A00087006397C6001C47054583C50700EDB723
:1046B000138697006395C602B727002083A7C7819A
:1046C000014595C71847034507006311050E0547C7
:1046D000A380E7000545EFA02038054509A813860B
:1046E000A700639BC6001C4703C507002D3DF24091
:1046F0006244D2440561828013866703E38AC6F868
:1047000013867703E381C6FA138687036392C60A8A
:104710001C45372400201307E00F83C4070083479C
:10472000A4831304A483638EE7021307F00F638648
:10473000E7021145EFB00FB9AA8505C1930700FD47
:104740002300F5008947A30095002301F500A3018C
:10475000050003450400EFB0EFC5F9572300F4004E
:10476000ADBFB727002003A7C7813E84014541D3D1
:104770008DEC85447D4523059100EFE08FD4231611
:10478000A10013050002EFE0CFD38327C481A30566
:10479000A1001307B100A380970074001306A100C5
:1047A00085450545EFA0A0330DBF26851D3335B7E0
:1047B00013869703E389C6F21386E7036397C6005F
:1047C0001C45094583C50700C1BD9387F703014513
:1047D000E39FF6F01C4703C5070005E96C001305CD
:1047E000D030EF906142B247414793F7070FE3861D
:1047F000E7EE9305B10013056031EF90E14003450A
:10480000B1008545EFA0202EC9BD053DF9B5B727FC
:10481000002083C7C7B3411106C6958B99CB3725B6
:1048200000201305058EEFD05F8F4D45B24041014A
:1048300082800145EFD07F8E0145CDBF03C70500C3
:10484000937625009377D70F99C2936727001318A3
:1048500085011358884113F7F7076354080013E7DD
:104860000708937685009377770F99C2936787003F
:104870001377050293F6F70D19C393E60702238019
:10488000D500634508009377A50281CB83470600D6
:1048900093E7C7002300F60082807DFD8347060072
:1048A000CD9BCDBF2D456319071403C805000947EB
:1048B0006310E814C84103471500034505002207AB
:1048C000498F42070D654187930825A0630B170B9D
:1048D000011122CC26CA4AC84EC606CEBE89B6846D
:1048E00032842E8963CEE800930705A0630DF7029A
:1048F000130515A06300A706239004000545B5A085
:10490000930745A06309F7086348F706130565AAEE
:10491000E314A7FE85472390F600DC4583C7070014
:104920002300F60091A0C84597C0FA1FE780809940
:10493000420541814E86637335012A862390C40067
:10494000420641828325C900228597C0FA1FE7806D
:10495000208D19A8DC4583D707002390060123008A
:10496000F600A183A300F6000145F2406244D24460
:104970004249B2490561828099472390F600194661
:10498000D1B785472390F600DC45014583C7070072
:104990002300F6008280DC45A9CB21472390E60066
:1049A00003D707002300E60003D707002183A300F5
:1049B000E60003D727002301E60003D72700218361
:1049C000A301E60003D747002302E60003D7470010
:1049D0002183A302E60003D767002303E60083D701
:1049E0006700A183A303F60041B723900600ADBF83
:1049F0002390060005458280828083C80500894790
:104A00006394F816DC41797122D406D626D24AD0B6
:104A10004ECE52CC56CA03C8170083C707002E8457
:104A200022083368F80042088D6713580841138341
:104A300027A0630C68102A8A3A89B684B285634C31
:104A40000301138707A0630BE802938717A0630194
:104A5000F80A854711A8138737A06303E80C13876A
:104A600067AA8D47E317E8FEB250225492540259C8
:104A7000F249624AD24A3E8545618280484432C644
:104A800097C0FA1FE7800084420541819D47E36D8E
:104A900025FDB72A0020938A2A8583C70A00B30917
:104AA0009900B24563D43701B5477DBF4844268697
:104AB000C2094A9597B0FA1FE780807603C60A00BC
:104AC000484493D9090105063306364181454E9580
:104AD00097B0FA1FE780E07BB727002083A74785C0
:104AE00099E3814751B79C438145E5DF52853DA05D
:104AF000AD47E31B09F6E39916FB8347160083468F
:104B000006005844A207D58F2310F700B7270020CE
:104B100083A74785F9D79C438545E1D78297D1B7CD
:104B2000AD47E31309F49947E390F6F84844194672
:104B300097B0FA1FE780C06EB727002083A747858C
:104B4000CDD39C43D9DF8D4555B7AD4711FF854780
:104B5000E39CF6F40347060093070008E3E6E6F05B
:104B6000DC452380E700B5BF85473E858280B727B7
:104B7000002023AA0784B7270020A3890784B7272A
:104B8000002023890784B7150020B707A00093856C
:104B9000457E938707059CC1B707E803DCC137F65C
:104BA0000600B71700209387076F1306C6C1D0C34E
:104BB000B71E002037F606000947938EFE7D1306C8
:104BC00006BF371E00202380EE00130ECE7DD0C717
:104BD00023AED70137230020B71800203718002054
:104BE0003715002037F60600B7FE06008546130687
:104BF00006C02300EE009388087E23AEC70313038C
:104C000003851308E87D1305D57D938E8EC037FE8E
:104C100006002380E8002380E7002388E700238044
:104C2000E7022388E7022380E7042300E8002384C7
:104C3000D70023950700D0CB238CD700239D0700F6
:104C400023A2D7032384D7022395070223A60702B2
:104C5000D0DB238CD702239D0702231003002300FF
:104C6000D500130E8EBF23A2C7052388E70423AE09
:104C700017052380E7062388E7062380E708B7F8AF
:104C8000060037F706001307C7BF938888C123A221
:104C9000E7082384D7042395070423A66704F0CBF1
:104CA000238CD704239D070423A217072384D70648
:104CB00023950706ECD7F0DB238CD706239D070648
:104CC00023AE07072384D7082395070823A6A70840
:104CD00037570500B7170020938707781307478ACF
:104CE00098C3375705001307A79FD8C323A407000D
:104CF0008280A54763ECA710B7E706009387C75FDC
:104D00000A053E951C41011122CC26CA06CE4AC88E
:104D1000B2842E8482879307800F63F9B7006145C0
:104D2000F2406244D2444249056182803719002032
:104D30009307096FC8571309096F09C997B0FA1F7C
:104D4000E780803EB72700202389078413061400DC
:104D5000916593850571328532C697B0FA1FE78059
:104D6000602E2326A90245DD3246814597B0FA1F01
:104D7000E78020520325C9022286A68597B0FA1F34
:104D8000E780004AB727002023898784014549BF6F
:104D90008947E396F5F803570600B72700202398C4
:104DA000E784EDB7A147E39CF5F6371500202146CF
:104DB000A6851305457E97B0FA1FE7806046F9B7D0
:104DC0008547E39EF5F4B71500209385056FD04D18
:104DD0009385850203C50400EFF05FA645BF8547B4
:104DE000E39FF5F2B71500209385056FD05D93859D
:104DF0008504CDB78547E394F5F203470600B7175E
:104E00000020A38EE77C59B7094519BF0945828068
:104E100005476302E5044111AA8706C62E8581CFA6
:104E200011476383E70425476388E7048947B24055
:104E30003E8541018280B717002083A5C77189474D
:104E4000FDD5B727002003C6278597B0FA1FE78056
:104E5000203D8147E9BFB727002083D707852390EE
:104E6000F50081473E858280B71500202146938555
:104E7000457EEF90416BF1BFB717002083C7D77D08
:104E80002380F500F9B7B72700209387378503C73C
:104E9000070015E305472380E700058909CDB7160C
:104EA000002037150020938606784146A545130556
:104EB000056F6F30406D01458280011106CE22CC16
:104EC0000546638CC50211460944639EC5023EC671
:104ED0003AC436C2EFD0EFC22A8492462247B24784
:104EE0001DE13E86BA853685EFD00FB8EFF03F92D0
:104EF000EFF0CFD3EF60F06F39A0EFD08FC02A84EE
:104F000019E1EFF0DF902285F24062440561828072
:104F100079714ECEAE896C0022D426D24AD006D604
:104F20002A89B284EF00707A2A840DE1CE854A8501
:104F3000EFC05F882A8419E93245B7160500268735
:104F40009386667A2D468145EF10C0122285B250B5
:104F5000225492540259F2494561828079714ECEB1
:104F6000AE896C0022D426D24AD006D62A89B284D1
:104F7000EF00B0752A840DE1CE854A85EFC0BF9160
:104F80002A8419E93245B726050026879386C68804
:104F90004D468145EF10000E2285B25022549254A6
:104FA0000259F24945618280397126DAAE844C009B
:104FB00022DC4AD84ED652D406DEAA893289368AF5
:104FC000EF00B0702A8431EDA6856303090283D710
:104FD00004002C002314F10083D724002315F100D2
:104FE000930720302316F100930780022307F10076
:104FF0004E85EFC00FF92A840DE55946A6851305A5
:10500000A1002304210197B0FA1FE7806021124517
:10501000B716050052879386067525462C00EF10BB
:1050200060052285F2506254D2544259B259225A34
:1050300021618280797126D2AE846C0022D44AD05C
:105040004ECE06D6AA893289EF0030682A840DE157
:10505000A6854E85EFC0EFF72A8419E93245B716C9
:1050600005004A879386467C3546A685EF1080006A
:105070002285B250225492540259F24945618280ED
:10508000BD47638CF50663E9B702A5476387F5065C
:1050900063EDB7009947638CF5049D47638FF50472
:1050A0009547638CF50401458280B5476387F50415
:1050B00063E1B704AD47F5B7DD47638EF50263EAF8
:1050C000B700C947638BF502D9476386F502C54728
:1050D000C9BFF5476383F50263E4B700ED47D1B775
:1050E00093072005638BF5009307200D5DBF4845AE
:1050F00082800841828008458280484182809307EF
:10510000F00F630EF506011126CAAA8413050002EA
:1051100022CC4AC84EC652C456C206CE3A89B68977
:10512000B28A2E8AEFA01F9A2A844D4515C893078C
:1051300000FB2300F400A3005401231144012302C7
:10514000340113058400614663050902CA8597B0DE
:10515000FA1FE780E00CA2852685EFA0BFA50145D8
:10516000F2406244D2444249B249224A924A05611D
:105170008280814597B0FA1FE780A011E9BF0945F9
:105180008280011122CC06CE2A842306B100A30618
:10519000C100EF50A06C15C18346C500B7270020A1
:1051A0002147938787B3639EE60003C567007800B5
:1051B0009306E0070146A2859937F24062440561F3
:1051C000828078009306E0070146A28503C5570058
:1051D000E5B7930700643306F6026FB06F8C05C91C
:1051E0000347050085469307270093F7F70F63F001
:1051F000F602411122C42A843A8506C6EFB0CFA434
:10520000FD572300F400B240224441018280828095
:10521000035705009307000B6313F702834745000C
:105220004947639CE7000347150185476399E700F9
:105230000355250085456F3090646D47C5BF82805A
:1052400001112314B1006C0022CC26CA4AC806CE34
:105250002A89B6842315C100EF0030472A840DE166
:105260002C004A85EFC02FC82A8419E93245B716A9
:10527000050026879386E66915462C00EF00905FAF
:105280002285F2406244D2444249056182807971AC
:10529000930720302314B1002315C1002316F10019
:1052A0002C0093078002014606D62307F100EFF099
:1052B000BFCFB25045618280C177797185073EC406
:1052C000894726D22316F100AE84930780024C0052
:1052D00022D44AD006D62A892307F100EF00F03EF7
:1052E0002A840DE12C004A85EFC00FD82A8419E9E1
:1052F0001245B726050026879386468345462C002F
:10530000EF0050572285B250225492540259456101
:105310008280B28605466FF03FC9797126D2AE848D
:105320006C0022D44AD04ECE06D6AA893289EF002C
:10533000D0392A840DE1A6854E85EFC0EFB12A84CD
:1053400019E93245B71605004A879386A6630D46CC
:10535000A685EF0030522285B25022549254025951
:10536000F249456182807971930720202314B100AE
:105370002315C1002316F1002C009307800201467B
:1053800006D62307F100EFF03FC2B250456182809C
:10539000011122CC06CE2A842EC632C436C2EF506A
:1053A000E04B0DCD0345C500B7270020A1469387EC
:1053B00087B312472246B245631CD50003C5670078
:1053C000B2862E86A2856244F24005616FF03FD31B
:1053D000B28603C557002E86A285F5B7F240624417
:1053E0000545056182806FF0BFB26FF07FB26FF04C
:1053F0007FC46FF03FC479714ECEAE896C0022D469
:1054000026D24AD006D62A89B284EF00102C2A84EC
:105410000DE1CE854A85EFC0AFBD2A8419E932453A
:10542000B716050026879386267E3D468145EF0008
:1054300070442285B250225492540259F249456177
:105440008280B28601466FF03FB6011122CC2E84D5
:105450006C0026CA06CEAA84EF003027DD47630A17
:10546000F500930710102314F400A2852685EFC0E1
:105470008FC2F2406244D2440561828023940500C9
:1054800083D7850099E36FF07FAD09458280FDB732
:10549000B727002003C7E788854763F9E7020111B2
:1054A00022CC2E846C0026CA06CEAA84EF00F021FE
:1054B00009E9930700102314F400A2852685EFC0A4
:1054C0008FBDF2406244D24405618280594582809A
:1054D000B727002023ACA7848280B727002023AE03
:1054E000A7848280011122CC26CA06CE2A84AE84EB
:1054F000EF50C036A6852285EFB03FE10DE9228549
:1055000023169100EF5080351DC18346C500B72793
:1055100000202147938787B36390E60203C56700A5
:1055200078009306F0070146A285EFF05FBDF240D8
:105530006244D2440561828003C55700D5B701118A
:1055400026CA06CEB68422CCDD4663E2B608D9462A
:1055500063FED50AA5466381D50A63EEB604954677
:10556000638CD50899466387D50A054441687D1840
:10557000631606093AC6EFB01FDD33068540324791
:1055800042064182420441803305C4004205BA8587
:10559000418132C6EF30D03FAA8749C181C432462B
:1055A0002390C400B30580406244F240D2443E855B
:1055B00005616FA0CFC4C5466380D504C9460D44BC
:1055C000E395D5FAC167FD17E31EF6FA65B7F54610
:1055D0006380D50463E4B600ED46D5B79306200595
:1055E0006388D5029306200DE391D5F8C167FD17B6
:1055F0000D446319F600BDBF09448DBF9306200D0D
:10560000E392D5F8310642064182ADBF15445DBF35
:105610000D444DBFC167FD171D447DB7F240624484
:10562000D24405618280011122CC26CA06CE03C66F
:1056300045002E841307000281469945AA8401374C
:105640002AC629CD8357040003464400930554001D
:105650002310F100835724002311F10089472312FE
:10566000F100930780022303F10097B0FA1FE7804F
:1056700020BB834744008A8526852314F100EFC0B0
:105680004F892A8411C5324597B0FA1FE780C0A917
:105690002285F2406244D244056182804D44CDBFF0
:1056A0005D7186C6A2C4A6C2CAC04EDE8947630623
:1056B000F600C14709446319F6040144B1C52E89B7
:1056C0004C0832C6B689AA84EF0030002A843246DC
:1056D00005EDC1778507CA851305D1013ECC230EA0
:1056E000C10097B0FA1FE780A0B32C082685253F9C
:1056F0002A8419E95245B71605004E879386666FCE
:105700001D462C08EF0010172285B640264496440B
:105710000649F25961618280797122D436844AD077
:105720004ECE52CCB2892E8A3A8981461307100296
:105730002286D94526D206D6AA8411352AC629C181
:105740002286CA85231481002312410123133101CB
:1057500097B0FA1FE780C0AC4C002685EFC06F9E63
:105760002A8411C5324597B0FA1FE780E09B228555
:10577000B250225492540259F249624A45618280E1
:105780004D44F5B7011122CC26CA06CE4AC8DD47E2
:105790002A84AE84638DF5028147035504006C00B2
:1057A0002306F100EFC06F9D0545638DA4080345F6
:1057B0008400B165938505B8EFA0BF83E547230159
:1057C000F400B7270500938707975CC09DA803479F
:1057D00055013149B2863306270318499C42329756
:1057E0001043E31BF6FA83D7460003564700E31540
:1057F000F6FA8C46084797B0FA1FE780A0AF49DD5C
:105800008347540103474401850793F7F70FA30A21
:10581000F40063FFE702B387270318480355040029
:10582000BA97984783D6470003D6270083D5070049
:10583000E5353DF103458400B165938505B8EFA0DA
:105840004FFB5945F2406244D2444249056182808F
:105850008347640199B7011122CC26CA06CEDD47E1
:105860002A84AE84639BF50603550500EFB0BFADF7
:105870000356C40183562401035744016D162A962A
:1058800042064182B307D640C207231EC400C1832B
:1058900063F0E7089305C5FF3308F740635BB80280
:1058A000BA96918EC206184C835504010355040024
:1058B000C1823E97953515E103458400B165938516
:1058C00005B8EFA00FF35945F2406244D244056198
:1058D00082806D1593160501F9B7814703550400C1
:1058E0006C002306F100EFC04F890545E38EA4FC50
:1058F00003458400B165938505B8EFA08FEFE547B8
:105900002301F400B7270500938707975CC065BFA4
:105910008547E9B7397126DAAE842C0022DC4AD8F3
:105920004ED606DE2A89B2894D232A8421ED4A8586
:10593000EFB07FA183D644006D1563C5A600931612
:105940000501C182984403D6240083D504004A850A
:10595000EFF09FDC2A841DE53146A6850808230662
:10596000010097B0FA1FE780A08B83D7240022455F
:10597000B72605004E879386E68F5D466C00231E92
:10598000F100CD2D2285F2506254D2544259B259C1
:105990002161828041B7BDBF797126D206D622D45B
:1059A0004AD04ECE52CC56CA5AC88944C5C159CEE7
:1059B0002E842A89BA8A368B328AEFB0DF98930513
:1059C00044008147711503D705006352A70A850774
:1059D00093F7F70FB105E318FAFE8A854A85F5219A
:1059E000AA842DE531453305AA029165938515708A
:1059F000CD4497A0FA1FE780E064AA8921C9314607
:105A00003306CA02A28597B0FA1FE7806081184466
:105A10008356440003562400835504004A85EFF062
:105A2000BFCFAA841DED0245B726050085475687DE
:105A30009386E68F5D464C002302F1004EC4230698
:105A40004101A3060100230761012D25B250225414
:105A5000268502599254F249624AD24A424B456124
:105A600082804E8597A0FA1FE780006CC5B7ED4491
:105A7000F1BF79714ECE37F60600AE89C16526D2E8
:105A80000147AA848946130646C2FD15054522D45E
:105A900006D64AD0EF10301A054431CD2A891307B3
:105AA000300281461146F5452685EFF05FA92AC6EA
:105AB000554431C18357A900CE8601462314F10015
:105AC00091472315F10085472300F500B2472C00CC
:105AD0002685A38007003247FD572301F700324790
:105AE000A301F700EF10F00A2A8411C5324597A0F0
:105AF000FA1FE78060632285B25022549254025903
:105B0000F24945618280411106C6EFF06FD719C591
:105B1000B240410117A3FA1F67000361B24041017F
:105B20008280011106CE2AC6EFB0CFE73245B727F3
:105B3000002023AC0784B727002023AE07849145BB
:105B4000B7270020A38CA7B2EF30E05EF2400561DA
:105B50006F20F0387971939705014AD006D622D488
:105B600026D2C187014963DE070AB727002003C593
:105B700097B32E89EF901FFC2A844DC1034705007F
:105B80009307000A6319F70885474C08A305F1003D
:105B9000EFB06FEEAA840DED834761017147637921
:105BA000F708138717FE1377F70F9306000263F8C1
:105BB000E608858BD5CBB727002083A78785994436
:105BC00081CB035524001306B1004C088297AA84A8
:105BD0008347B10099C7084409C597A0FA1FE78019
:105BE000A05495E05247B7070001938707F07D8FD7
:105BF000B707120093870710630FF700034761018F
:105C0000ED47631AF700035524008545EF30204720
:105C1000CD476388F4002285EF90BFE5A167334943
:105C2000F900B25022544A8592540259456182804B
:105C30003707301405073357F700058B3DDB37274F
:105C400000200327C78549D70347510151F3230695
:105C5000F10099472308F100035524006C00231735
:105C60000100EFB0DF85ADB7B727002083A7C78558
:105C70009DC3035524001306B1004C08829729D90F
:105C8000AA8483475101A9F7834761012308910042
:105C90002306F100D1B79944EDB7397122DC26DA39
:105CA00006DE4AD84ED652D456D25AD0A5472A84B8
:105CB000B2846399F5108347450203570600835A5F
:105CC000260085072302F5029307F7FFB387FA0240
:105CD0005442C207C183B69703C9170083C70700A0
:105CE0008346C50022093369F90085476390F602AF
:105CF00033075703231006008149014A130B35016E
:105D0000931A070193DA0A0163E15907C167FD1786
:105D10006302F90C83570401637EF90A05094209FD
:105D20008346C4001359090123172401054703556D
:105D300004009305E400639FE6002315F100930738
:105D400020302316F100930780022314210123073A
:105D5000F1002C00EFB0FFA203458400B1659385EC
:105D600005B8EFA00FA95945BDA083D62400DC409B
:105D700083452401ED1613865900C206C1823E9662
:105D80005A85EFB0AFC705C9630C3A01C84003D6C6
:105D90002400B3053501529597A0FA1FE7804048CB
:105DA00083D724003E9A83D70400420A135A0A017B
:105DB00085072390F40083D72400BE99C20993D9A4
:105DC000090199B703474600A9476310F7028347C3
:105DD000450281CF0145F2506254D2544259B25922
:105DE000225A925A025B2161828083462401130960
:105DF000340137F506004A8689451305C5C1EFB061
:105E0000EFBF19C10545C1BF8346240137F5060020
:105E10004A868945130505C2EFB04FBE65F5834636
:105E2000240137F506004A868945130545C1EFB0C0
:105E3000EFBC69F98346240137F506004A86894597
:105E4000130505C0EFB08FBB55FD03C74400BD4728
:105E5000E3EAE7FAA56793874712B3D7E700858B94
:105E6000D5D38347440285072302F40203D92400D3
:105E700071BDB727002003C607B4B727002003A7CA
:105E8000078681476315F600814636858280BA868B
:105E900013078702835587FDE389A5FE850793F7DE
:105EA000F70FCDB7011106CE2EC6E13701CD8347DE
:105EB000A500B245138717006396E50093F707F82E
:105EC0002305F500F24005618280011106CE2EC641
:105ED0004D3705C5B24591C188C183478500130779
:105EE000E00F5D456388E7001307F00F014563830A
:105EF000E7005945F240056182800945E5BF41113F
:105F000022C42A84210506C626C24AC0EFF02FAD5E
:105F100083472400A51793F7D70F91EB0347C400DD
:105F200085476310F7061C4881443149A9E3FD57B2
:105F300023010400A304F400230204021305C40097
:105F40002244B2409244024961468145410117A36F
:105F5000FA1F67000334B38724033E95084509C53B
:105F600097A0FA1FE780401C850493F4F40F834741
:105F700044010848E3E1F4FE97A0FA1FE780C01A45
:105F80007DB7084C75F965B7411122C4416406C656
:105F900026C29307E4FF630CF500AA8491EDD13D7E
:105FA00019E51305F4FFF13519C123109500B2402E
:105FB000224492444101828085476394F504EFF0C6
:105FC0005FEB2A846DD5FD572310F50083478400CD
:105FD0001307F00F6384E7021307E00F638BE700FA
:105FE000834624000345940001475146A685EFF0FF
:105FF0000F9122852937FD572304F400230504005F
:106000007DB78947E395F5FA8545EF40902845F13E
:106010002685EFF01FE62A8455F951BF39C9034799
:1060200085009307F00F6306F704011122CC06CE1A
:106030002A848346250083550500034595000147C2
:106040005D46EFF0CF8B03472400E1476319F7006B
:10605000035504006C0023060100EFB01F92F957AE
:106060002304F4002285EFF09FE9F24062440561C9
:10607000828082809307F00F6306F706011122CC1D
:1060800026CA2A844EC6AE84B689AA8593068500A0
:10609000376505004AC852C43A89328A1305C501DA
:1060A000794606CEEFF0EF92A304240123014401C8
:1060B0002322340185C01305C4006244F2404249E2
:1060C000B249224AA685D2446146056117A3FA1F48
:1060D00067000315F2406244D2444249B249224A61
:1060E000056182808280B72700202382A786828074
:1060F0009547639CF506834745028546850723023D
:10610000F50283570600584203462600FD17C207D2
:10611000C1836318D6048A07BA9703C7170083C7D9
:1061200007002207D98F0357E50063F9E7044111FF
:1061300006C622C485072316F5002A849305C500E8
:1061400003550500EFB02FDA03458400B165938550
:1061500005B8EF901FEAB2402244D9473E8541017D
:106160008280C946B387D70245BF83464600294788
:1061700085476396E6000347450211C381473E8584
:1061800082809D476392F506834745028356E5006A
:1061900085072302F502835706005842FD178A0738
:1061A0003E978347170003470700A207D98F01478F
:1061B00063F6D704411106C622C485072A84231634
:1061C000F5009305C50003550500EFF0CFC5034565
:1061D0008400B165938505B8EF90BFE1B2402244D9
:1061E00059473A854101828083464600A9470547C1
:1061F0006396F60003474502133717003A858280FD
:10620000411122C406C626C2B5472A84639BF50401
:1062100083474502B28485072302F5020355050032
:10622000EFB06F9283D704001307F5FF014563C5F4
:10623000E7020357E400035504009305C400BA972E
:106240002317F400EFB0EFD803458400B1659385C0
:1062500005B8EF901FDA5945B240224492444101FB
:106260008280034746009D470545E317F7FE034537
:10627000440213351500CDB7C547639EF506835715
:10628000060003572600FD17B387E70203474502C0
:1062900005072302E5025842C207C1833E978347A0
:1062A000370003472700A207D98F41677D17639501
:1062B000E70081473E858280138717002316E5009B
:1062C0000357E500E3F7E7FE411122C49305C5003B
:1062D0002A840355050006C6EFB00FD90345840094
:1062E000B165938505B8EF90DFD0B2402244D9471D
:1062F0003E85410182808346460029478547E39BCE
:10630000E6FA0347450255F775B7011122CC26CAB4
:106310004AC852C406CE4EC683C7250015472A8AEE
:10632000AE8432843689639DE7043686A28526854D
:10633000EFF01FDCAA8955E985476318F40A034783
:106340004900A9476301F70203C594004A878546BF
:106350000146D285EFE0BFDA19E585454A85EFE0D1
:106360003FD21334150083C6240003C594000147AF
:106370006946D285EFE0BFD82685EFF05FB851A01F
:106380001D476398E7003686A2852685EFF07FDFFC
:1063900055B725476398E7003686A2852685EFF036
:1063A000DF8F49BF35476398E7003686A28526858B
:1063B000EFF01FE541B745476398E7003686A285B1
:1063C0002685EFF07FEBBDB75D47639FE70003C70E
:1063D000C50085473686A2852685631DF702EFF046
:1063E0006FBA8547631BF5048549A5476317F40217
:1063F000835709009DE30544E38709F6D947E39DE8
:10640000F9F62285F2406244D2444249B249224A16
:1064100005618280EFF02FC4E9B703C594004A8775
:10642000A2860146D285EFE09FCD71F5A2854A850F
:10643000EFE01FC513341500C1B70544D9B7397152
:1064400022DC06DE26DA4AD84ED652D456D283D77C
:1064500005001944B1E783C925002A89328A938748
:1064600059FE93F7D70FAE84DDE7B727002083C628
:1064700047861307F00F938A478619446382E60222
:10648000F5476394F904EFF0DF9EAA8921C1034622
:10649000A5000DCE93178601E18763DD0700014457
:1064A0002285F2506254D2544259B259225A925A19
:1064B00021618280F5454A85EFE0BFCC83C7A90002
:1064C00093E707F82385F900D9BF814983D64400B3
:1064D000904483C5140003C504003800EFB0EFCA30
:1064E0002A845DFD83C6240003C50A0038000146E6
:1064F000CA85EFE0DFC02A8445F5B24799C323007F
:106500000A0083C724007547E39BE7F8E38909F88D
:106510002385F90071B7EFF0DF95AA8A49D1854745
:106520006391F90A83D5440088443000EFA09FE3CB
:106530002A843DF503C72A00C54763F2E70ADD4711
:106540006301F70CB727002003C59A0083C797B3F0
:10655000639CA70A014403C72A008D47631FF70401
:106560008357810003D7CA0063F4E7002396FA003B
:1065700083D5CA004A85EFE0FFF6B727002083D70E
:10658000079A6D47637BF70283D5CA005D47637640
:10659000B7021387350091056349F7001307B00F61
:1065A000BE856374F7009305B00F1166C20513062C
:1065B0000629C1814A85EF8060475685EFF03F94F8
:1065C000C5B5834725001144E39C37ED5C41E38961
:1065D00007EC83D5440088443000829791BFB727E9
:1065E00002009387072AB3D7E700858BA1DF03C694
:1065F00024003400D6854A85EFF03FD12300AA005D
:1066000045B583A70A01DDB783C6240038000146DB
:10661000CA85EFE0DFAE2A841DFD83C52400280073
:10662000EFE01FA605D923000A0035B7011122CCDF
:106630003724002006CE26CA4AC84EC652C4930943
:1066400084B303C589009307800291653305F50281
:1066500093856570372900209304098697A0FA1F57
:10666000E780409E03C68900930780028145330678
:10667000F60288C097A0FA1FE780A0C19C404D4554
:10668000A1C3930484B3130909860144130A800249
:10669000FD5983C78400636DF40237650500130557
:1066A000E543EFE0FFE237650500130545EAEFA09B
:1066B0005FBB37650500130585F8EF40A034014541
:1066C000F2406244D2444249B249224A0561828082
:1066D000B30744030325090061468145050413748B
:1066E000F40F3E95231035012301050023143501D5
:1066F0002305050023020502310597A0FA1FE78054
:1067000040B941BF01458280B727002083C617B436
:10671000814763E5D70001473A8582802E8791053E
:1067200003D6C5FFE30AA6FE8507E5B70DCD83476F
:1067300025000547890793F7F70F6376F7024111A4
:1067400022C406C62A848355050003453500014747
:10675000F9465D46EFE0BF9AF9572311F400B240C5
:106760002244410182808280B727002003C717B4EA
:10677000FD56814763E3E70082802310D5002301A3
:10678000050085071105FDB70145828037160020F9
:106790001306B67F930700022300F6003717002088
:1067A000FD57230DF77E37170020A306F77E371716
:1067B00000202306F77E8545B7170020239CB77E6F
:1067C000B727002023930786B727002023A8078632
:1067D000B727002023A00788B727002023AA078611
:1067E000B7160020B7F706009386067F938707C188
:1067F000DCC2B727002023840786B71700209387C1
:10680000C77809472380E6002380E7002388E70054
:106810002380E7022388E70237F70600130747C003
:10682000D4C7D8DBB7F606000D47238CE702938662
:1068300006C037270020D4CB0327C78637F50600CC
:10684000B7F606001305C5C1938646C2C8C32384A4
:10685000B70023950700238CB700239D0700D0CFF6
:10686000D4D3238407022395070223A60702239D7E
:106870000702D8DFB7170020377705009387C77C5A
:106880001307479423A00700D8C323A407008280DE
:10689000411106C6EFF05FE711C503452500B24080
:1068A000410182800145E5BF411122C426C24AC090
:1068B00006C6AA842E893284EFF01FE511E94165EE
:1068C000CA857D15EFF05FE4C54711C5231095001B
:1068D000230185008147B2402244924402493E850B
:1068E0004101828029E789483547639316050111E4
:1068F00006CE22CC26CA034716000346060093C7DD
:10690000F7FF2207598EF18F32C68DE7C4452A84DE
:10691000A685EFF0FFF732460147630FA6002285F8
:106920006244F240A685D24405616FF0FFF72D471F
:106930003A85828013070008F2406244D2443A85C7
:106940000561828083C8050009486395080303A890
:1069500045008347180003480800A207B3E7070172
:10696000C2070D68C18713082890639507018947FE
:106970006FF05FF705458280011122CC37140020AB
:106980001304D47E0347040006CE26CA4AC84EC666
:106990009307F00F6300F704AA892945B2842E8972
:1069A000EF904F9205C99307100B2310F5002302B7
:1069B0000500231135012313250123149500AA8511
:1069C000034504006244F240D2444249B2490561A1
:1069D0006F904F9EF2406244D2444249B2490561F1
:1069E00082804111B727002026C2AE8483A5C786C6
:1069F00022C406C62A84EFF0BFE9098909C92285A5
:106A00002244B240A685924441016FF08F86B24085
:106A100022449244054541018280411122C426C28C
:106A20004AC006C6AA84130445001309850B835780
:106A300004009DC3084409C59790FA1FE780C06E03
:106A400022853146814597A0FA1FE7808084310472
:106A5000231A04FEE31D24FDB2402244FD57239077
:106A6000F4000249924441018280B727002003C606
:106A700017B4B727002003A7878781476315F6005F
:106A8000814636858280BA861307870B835587F443
:106A9000E389A5FE850793F7F70FCDB7B727002049
:106AA00083A7078889CB03D747006314A7008847CB
:106AB00082809C43C5BF01458280411106C6F93FD3
:106AC00009C50845B240410182800145E5BF011179
:106AD00026CA9384450022CC4EC606CE4AC852C46C
:106AE00056C25AC0268781490144814681473D45A7
:106AF0000356070055CED9E20354470083572700B9
:106B0000B286A297C207C18385093107E392A9FE25
:106B100025C82E8991659385457022859790FA1F27
:106B2000E78040522A8B29CD814A014A8C4485C591
:106B300003D6440033054B019790FA1FE780406E5F
:106B400083D7440088443E9A420A135A0A01979018
:106B5000FA1FE780605D63890A003146814526851A
:106B60009790FA1FE780E072850AB104E3E03AFDEE
:106B70002326690123148900054521A0630DD60051
:106B80000145F2406244D2444249B249224A924A03
:106B9000024B0561828003562700E313F6FE03567D
:106BA00047003294B2974204C2074180C183A9BF13
:106BB0000545E37835FDA9BFB727002083A74787A0
:106BC00099E30145828098470357A7006315A70002
:106BD0001385470082809C43E5B7411106C6E93F13
:106BE00011C503550500B240410182800145E5BF52
:106BF000411106C6D13711C503452500B2404101F8
:106C000082804145E5BF411122C42A842E8506C6F3
:106C1000C537AA8505462285EF307047954763053D
:106C2000F500BD476313F5002145B2402244410100
:106C300082804111B727002022C406C603A44787DB
:106C400081469387478729C018440356A7001840F8
:106C50006317A60285CA98C22E8581C9214693056D
:106C600044009790FA1FE780A05B22859790FA1F57
:106C7000E780804B0145B240224441018280A286D8
:106C80003A84D1B798C3C9BF0545F5B73727002067
:106C900083270788014613070788A9C703D8470039
:106CA0009443631CA802011106CE22CC26CA0DCA49
:106CB00014C2AA843E852E849790FA1FE780C046AE
:106CC0002C002685EFF0FFF601E519C0B2471CC085
:106CD000F2406244D244056182803E86B68775BF29
:106CE00014C3C1BF05458280411122C42A8409050D
:106CF00006C6EFE0CFCEFD57A301F400B240224418
:106D000041018280B727002003C717B4B7270020AE
:106D100083A7C7872A86050781463E8583D7070054
:106D20006388C700850693076500E3E8E6FE014532
:106D30008280411122C4416406C626C29307E4FF43
:106D4000630EF500AA8485E1EFF0DFFB01E913058E
:106D5000F4FFEFF03FFB19C123109500B24022442D
:106D600092444101828085476394F504EFF09FF9D6
:106D70002A846DD5FD572310F5008347240013079F
:106D8000F00F6384E7021307E00F638AE70003450F
:106D900034000147F9465146A685EFE04FB62285FB
:106DA000EFF09FF4FD572301F400230204007DB7A8
:106DB0008947E395F5FA8545EF30B04D45F12685D5
:106DC000EFF05FF42A8455F951BF1D71A6CACEC6F3
:106DD00086CEA2CCCAC8D2C4D6C2DAC05EDEAE8429
:106DE00083C52500F947AA896397F504EFF09FF161
:106DF0002A8411ED01442285F6406644D644464972
:106E0000B649264A964A064BF25B25618280834743
:106E100025000547890793F7F70FE37DF7FC034546
:106E200035000147F9460146CE85EFE04FAD22859A
:106E3000EFF09FEBC1B703AB0400B70700019387E6
:106E400007F037071200B377FB0013070710B28A69
:106E50000149638AE7022EC6EFF0DFEA2A89B245CC
:106E60001DC10346450005C293178601E187E3C3B0
:106E700007F84E85EFE0EFB08347490093E707F846
:106E80002302F90085BF371A00200347AA7F930722
:106E9000F00F130AAA7F1944E30FF7F4E147E3EC7C
:106EA000B7F493D71500FD1713973700B7E706001F
:106EB00093874762BA9703A80700E30E08F283ABF3
:106EC0004700E38A0BF2420B135B0B0163050B00D7
:106ED000C947E392F5F283D64400904483C5140079
:106EE00003C50400380802982A84E31605F02C082C
:106EF0004E85829B2A8421C983C71400E39D07EE37
:106F000083C72400230AA10039472308F1006399AD
:106F1000E70262478347170003470700A207D98F9C
:106F20000C084E852319F100EFA06FD9E30405EC9E
:106F300014080546D9454E85EFE08FC52A8465BD06
:106F400083578101F1BF83C624009147E384F6EAA9
:106F500003450A0038080146CE85EFE04F9A2A849F
:106F6000E31B05E883C524002808EFE06F9119C1F1
:106F700023800A009840B7070001938707F07D8FB0
:106F8000B707120093870710E306F7E6E30409E664
:106F900083C724002302F900B9BD011106CE2EC615
:106FA000EFF05FD601CD83474500B2451387170048
:106FB0006396E50093F707F82302F500F2400561B8
:106FC0008280B727002003A7478719E3014615A849
:106FD0001C4703D8A700636B050183584700B3869D
:106FE00008016355D5008146639416011843F1BF2B
:106FF0003E86C10703D3A7FF6317A30099C123905F
:107000000501328582808506C206C182F1BF3971D1
:1070100052D42E8A4ED69305E101AA89528522DCEC
:107020004AD856D206DE26DA328936C63AC4BE8A35
:10703000EFF03FF9054435C5AA840355E101394411
:10704000EFF0DFA539CD03284500630C0804224783
:10705000B246D6874A86A6854E8502982A8431E1B3
:107060009307E00F638FFA0203C704008947631A8E
:10707000F702D8408347170003470700A207D98FBC
:10708000C2070D67C18713072790639CE7008347FA
:10709000190003460900D285A2075D8E4E85EFF0E8
:1070A000BF8D2285F2506254D2544259B259225AAD
:1070B000925A21618280797122D4035425004ECEE8
:1070C000AA89228556CA06D626D24AD052CC5AC898
:1070D0005EC662C4AE8AEFF05F9901E92285EFA037
:1070E0001FDE594429E90144B9A003C78900854737
:1070F000AA840144631AF702AA8513858900EFF078
:107100001F9D29CD03D7640083D68400D04483D546
:10711000440003D52900E147EFF07FEFD9472A84E7
:107120006318F50223A604002685EFF01F8F49C0DF
:10713000D947E30AF4FA2285B250225492540259F4
:10714000F249624AD24A424BB24B224C456182809C
:1071500061DD83D744002390FA00F9B71389440016
:10716000014AB94B594C3D4B83550900D5DDE147E8
:1071700063067A010357C90011C3D9470357290091
:10718000835649000326890003D52900EFF03FE824
:107190002A846319850123240900050A3109E315AE
:1071A0006AFD59B77DD9835709002390FA00F5B7D6
:1071B00003D529002DB701112317C1009307E00F54
:1071C0001306E1000147894606CEEFF05FE4F24086
:1071D00005618280797122D42A840355850026D2E4
:1071E000AE849305210106D64AD0EFF09FDD6308F7
:1071F000050E834785002AC693F707028DCF0355F6
:107200002101EFF09F8BAA87B24501ED83578400DF
:1072100039452390F400B2502254925402594561EA
:107220008280035524004946829711C58357840004
:107230002390F400CDB7035924004A85EFF0FF8274
:1072400011ED41657D15EFF05F8219E583578400EC
:1072500025452390F400C1B72310250113074500ED
:107260008147BD46035607002DE63147B387E70245
:10727000130984003146CA8591073E959790FA1FFD
:10728000E78000FA3146CA8548089790FA1FE780E0
:1072900020F90356C4000355240041478146DD45CB
:1072A000EFE0EFA92ACE19E58357840045452390E6
:1072B000F40095B70C480356C4009790FA1FE78076
:1072C00020F6035524004C08EFA03FBB29D55945B3
:1072D00099B785073107E397D7F8254581BF05455D
:1072E000B1B7797122D42A840355850026D2AE84A1
:1072F0009305E1014AD006D63289EFF09FCC51C503
:107300008347850093F70702A9E703471401930712
:10731000200519E3834744008356A4005044835555
:107320008400035524000147EFF07FCEAA8721E9AE
:107330008347140199E703552400EFA03FAFD947D5
:1073400011E18147B2502254925402593E85456161
:1073500082802AC60355E101EFF02FF6AA8705C9FE
:10736000B2450355240049468297AA8759DD035741
:1073700084002390E4000347140161F7E1B7594703
:10738000E317E5FE230009006DBF8547CDB7B94778
:10739000F9BF397122DC4AD84ED652D406DE26DA3D
:1073A000AA892E8A32C63689EFF0DF95094415C5C1
:1073B000834725001307E00FAA845D44638FE7002D
:1073C0001307F00F5944639AE700324605E2D2856D
:1073D0004E85EFA0BFB22A8415CD2285F2506254AB
:1073E000D2544259B259225A2161828003550A006F
:1073F0009305E101231F0100EFF0BFBC0355E1013C
:10740000EFF00FFFAA8505464E85EF3040482A84ED
:107410005DDDE1B79307F00FE301F9FC3765050087
:10742000938624007946A6851305C572EFD07FDACE
:10743000A38124015DB73971B727002026DA83A420
:10744000478752D45AD05ECE62CC06DE22DC4AD8C0
:107450004ED656D266CA2A8BAE8B328C368A99E0CB
:107460008149B9A0804483DC44000149835AA400C7
:10747000631499018440E5B78357A400A28963F897
:10748000670105094209135909014104D5B7E3EA27
:10749000FBFE630C0A00834504004840D2866286E6
:1074A0003AC6EF90BFD5324769DD19C323105701A3
:1074B000F25062544E85D2544259B259225A925ACD
:1074C000025BF24B624CD24C2161828003D70500F3
:1074D00083D62500854763E9E60439C7411183C691
:1074E000450026C237F506009384550022C426863F
:1074F0002E841305C5C1894506C6EF903FD0C1470C
:1075000011CD8346440083552400035504000147F0
:107510002686EFF05FF2814711E1A947B24022448D
:1075200092443E85410182803E8582802E860355AD
:10753000060083D52500854763E2A50205C1834681
:10754000460041110147150606C6EFF0DFEE814700
:1075500011E1A947B2403E85410182803E8582808B
:107560002E860355060083D52500854763E2A502D4
:1075700005C18346460041110147150606C6EFF0D6
:107580009FEB814711E1A947B2403E8541018280CE
:107590003E85828039714ED683D7250083D9050078
:1075A00006DE22DC26DA4AD852D456D25AD05ECE33
